:020000040800F2
:1000000000A00020E90301082DBE00081DF400082F
:100010002BBE000829BE000827BE00080000000013
:1000200000000000000000000000000025BE0008E5
:1000300023BE00080000000021BE0008BF550008D4
:100040005104010851040108510401085104010838
:100050005104010851040108510401085104010828
:100060005104010851040108510401085104010818
:1000700051040108252F00085F2A000851040108D7
:1000800051040108510401085104010851040108F8
:100090008DBE0008510401085104010851040108F3
:1000A000A9BB0008E9BB000899BB000811BC000807
:1000B000D9BB0008C9BB0008B9BB0008510401083E
:1000C00051040108510401085104010851040108B8
:1000D00051040108D5BD0008C9BD0008510401083C
:1000E000CD5500085104010869EB000851040108CE
:1000F0005104010851040108510401085104010888
:100100000000000000000000000000005104010891
:100110005104010851040108510401085104010867
:100120005104010851040108510401085104010857
:100130005104010851040108000000000000000003
:100140005104010851040108510401080000000095
:10015000000000000000000000000000000000009F
:1001600000000000000000005104010851040108D3
:100170005104010800000000000000000000000021
:08018000000000005104010819
:100188002DE9F04F2DED068B6B4D6C4B2B60A1B01C
:1001980000236B600DF068FF18B90DF087FF0AF0B7
:1001A800AFFD0AF06BFE664B664C1A7842F001020E
:1001B8001A70654A4FF47001C2F88810002208923C
:1001C8000992226842F4803222600493236803F47F
:1001D80000330993089B01330893099B1BB9089BBB
:1001E800B3F5A04FF2D1236813F4003318BF0123ED
:1001F8000993099B012B69D0DFF84C81534BC8F850
:100208000C30636AAB60636A514EDFF870A1DFF8A7
:10021800709143F080736362636943F4FC0320AF19
:10022800636103238DF8323041F6FF7327F8503DA0
:100238004FF09040394602F089FE4FF6FF73304682
:100248003946ADF8303002F081FE4248394602F0B6
:100258007DFE4148394602F079FE4048394602F0B1
:1002680075FE39463E4802F071FE384609F024F81A
:100278000C9B3C4AB3FBF2F33B4A3C4913603C4BB2
:1002880000221A603B4B5960F02188F823109A60CD
:1002980007221A60DFF8EC80DAF80830C8F8003076
:1002A80099E80300636987E8030043F480236361E6
:1002B8004FF48053B3610C980DA902F047FED8F8AB
:1002C800003013F0080F564629D163E02A4B12225A
:1002D8001A606368636063686360636843F480639B
:1002E8006360636823F47C136360636843F4881372
:1002F8006360236843F0807323602268114B920186
:10030800FBD55A6822F003025A605A6842F002028A
:100318005A60636803F00C03082BFAD16CE79AF86B
:100328009031012B36D8044A9AF89131926812F02C
:10033800805A00F0DB872DE03808002029A6000845
:10034800D02600200010024000ED00E00005FA056C
:100358000004004800080048000C0048001000484D
:100368000014004840420F00881100203F19010086
:100378008C11002010E000E000200240481C002002
:100388003C3A0108781B0020C34B002283F89121D6
:100398000AF010FF642005F004F94FF48C72BF488E
:1003A800002112F042FAE369BD4A43F00703E36112
:1003B800A36943F4E123A361636943F4C023636140
:1003C80002F1E00E937BD07B4FEAD30C03F00701D8
:1003D800536803EB8C038900D3F820C04FF00F0A51
:1003E80088400AFA01F12CEA01011962196A1032EF
:1003F800084372451862E5D10022AA4900235354E4
:1004080001320E2AF9D1DFF8CCA20AF11A02FF2133
:1004180099540133072BF6D1A34AA44B1360DFF894
:10042800B8B2A34A0393032111705846002124222D
:1004380012F0FBF914228BF800209E49039BD8F890
:10044800008001228BF8182096F805B081F800B0DA
:10045800A3F5F171CAF824109749A3F591730B60BD
:10046800964B03EBCB0318F0200F5B78CAF82830C3
:1004780018BFCAF828200023914A40F2DC5122F81C
:1004880013100133082BF7D1384600211C2212F033
:10049800CCF9BBF10E0F04D00BF0EF0BBBF1080F3A
:1004A80002D101238DF84030022007F035F818B149
:1004B8004088003018BF0120C8F340038DF836305B
:1004C800C8F380138DF83830C8F340338DF83030D6
:1004D800C8F3C03300F001008DF8333018F400631E
:1004E8008DF8350004D096F884315F1E7B427B413D
:1004F8008DF83430C8F300438DF83930AB6AB6F85C
:100508004401ADF84400003318BF01238DF83A3098
:10051800C8F300538DF83B30B6F84631ADF83E309D
:1005280018F4805FB6F8523118BF5B48ADF83C301C
:10053800C8F380438DF83730B6F850311CBFB0F897
:100548004C01ADF84400B3F5FA7FADF8423084BFF2
:100558000023ADF844305B4896F8D43185F82C3048
:10056800002385F82D3043709DF8403008F00101D4
:10057800002BC8F3C0028DF831108DF832200CBF63
:100588000023022301B902B1013309EB83094FF0BB
:10059800000AD9F808309A1E1A3303920593039B70
:1005A80033F8022F03934FF6FF739A4200F0358118
:1005B800110A0229CBB202D19DF8301003E00129BB
:1005C80004D19DF83110002900F022819DF83A10DD
:1005D800D2B261B19DF8401049B99DF8381009B1FF
:1005E800111F01E0A2F10801012998BF04232C4F33
:1005F8009DF83B104FEA02194F4431B19DF8401065
:1006080019B9043A032A40F2EC80012B66D1FF2382
:1006180085F8743085F87530214BC5F8847003EB84
:1006280009024FF00008517B50688DF82A1002F13A
:10063800080B1289ADF828200AA9022285F87880CB
:1006480006938DF82B2085F83080C5F83480C5F8DE
:100658003880C5F83C80C5F8708085F8768085F8C4
:10066800778002F073FC069B9BF8021053F8090090
:10067800424602F09DFB38460CF094F8124B1349A1
:10068800C5F88830124BC5F88C30C5F890803846CC
:100698000A1D0BF03BFBBBE0481C0020C4110020E6
:1006A80030580108440800206C2300203A1E00201E
:1006B800851100201403002058130020485B01080E
:1006C800D810002065080020A1270008C0080020D5
:1006D800812800083808002070230020022B46D10A
:1006E8005FFA8AF21C2101FB02FC05EB0C089D4A0B
:1006F80088F879A0012188F8781002EB09014FF0F9
:10070800000B91F80DE0486888F87AB001F108020A
:100718000989ADF8281088F882B00AA9C8F8847049
:10072800CDF81CC08DF82AE006928DF82B3002F027
:100738000DFC8C4B069A53F8090091785A4602F042
:1007480037FB38460CF02EF8DDF81CC08649874A7E
:10075800C8F888206144864AC8F88C20C8F890B048
:1007680038460A1D0BF0D2FA0AF1010A50E0032BB1
:1007780035D19DF83730DFF82C82DFF82C923BB169
:1007880098F82EB0384608214FF6FF7200231AE079
:10079800BDF8422098F82EB0BDF84430B2F5FA7F83
:1007A8000BD97449B1FBF2F23846082192B202F033
:1007B800F6FB714B49F82B000AE07049B1FBF2F2E5
:1007C8003846012192B202F0EAFB6D4B49F82B0042
:1007D800C36098F82E30013388F82E3018E0042BC7
:1007E80016D195F82D80BDF83C20644B93FBF2F2AE
:1007F8003846BDF83E30012192B202F0D0FB95F8A0
:100808002D3005EB88080133C8F8580185F82D30DC
:10081800039B059A93427FF4C2AE95F82D2085F884
:100828007821584A584B92F800E0AEF11702002799
:10083800022A1F709C461AD86B6A3B44D3ED007A93
:10084800F5EE407AF1EE10FA02D1AB6A63BB26E00E
:100858004E4A07EB02080FCB88E80F009CF80030DF
:1008680010370133C02F8CF80030E5D1EDE7484B45
:1008780013F83E908CF8009003EBCE03D3F804A055
:10088800BAF1000FE1D04F45DFDA404A3B0103EBF4
:10089800020853440FCB013788E80F00F3E73D4FB8
:1008A8003B68DD0425D41DE03B4B3C4A13F83E0071
:1008B800107003EBCE035D68002DF0D00023834257
:1008C800EDDAC3EBC3016A18DFF8E080D2F80090D4
:1008D80041F8089001EB08079188B9809279BA71BC
:1008E8000133ECE70EF0EF03082BDFF8C48020D1CA
:1008F80022E09CF80020012AF4D9294B03EB0212CC
:10090800103210339342EDD053ED047AB6EE007AEC
:1009180067EE877A43ED047A53ED057A67EE877AB6
:1009280043ED057A53ED037A67EE877A43ED037A50
:10093800E7E7BEF10E0F0BD198F8003043F0100333
:1009480088F80030BEF1180F34D104F0FFFF31E011
:1009580098F8003023F0100388F80030BEF1190F22
:10096800F2E700BF30580108C0080020B52E000883
:100978007927000800127A00A128000840420F00D9
:100988009128000814030020C01100205002002004
:10099800485B0108781B0020F03E0108E4120020A3
:1009A800580200203808002090110020E51200208D
:1009B8001811002004F0AEFF3B68DFF84093C34DE8
:1009C80058035EBFC24B01221A70049B049A1B781D
:1009D80043F0040313704FF48063ADF828301123FB
:1009E8008DF82A3063694FF0020A43F480230AA97C
:1009F8008DF82BA04846636102F0A8FAB54BB64AB9
:100A08001A60002004F0E6FDB44B1D60636943F4EE
:100A180080236361E36943F40013E361236B23F0EC
:100A280010032363236B43F010032363D9F82030AA
:100A380023F07063C9F82030D9F8203043F0806380
:100A4800C9F82030D9F8203023F07043C9F8203095
:100A5800D9F8203043F08043C9F82030032300241C
:100A68008DF82D30484640230AA98DF82E408DF880
:100A78002F400A938DF82CA008F08CFD802348465F
:100A88000AA90A9308F086FD2B6823F001032B605E
:100A98002A68934B13402B60924B2B612B6843F0D1
:100AA80001032B60AC60EC60AC60AB688E4C43F427
:100AB8000043AB602B682B606B6823F0784323F40A
:100AC80000436B602B6843F001032B60B4F8583186
:100AD800002B40F08D84B4F95A21002A40F0888414
:100AE800B4F95C21002A40F0838400210C227F485D
:100AF8007F4E11F09AFE002114227E4811F095FED7
:100B08007D4B002201201A7006F028FF337843F04D
:100B180002033370794B4FF480529A610A25DFF84B
:100B2800DC91B9F814309BB283F48053A9F81430DF
:100B3800192004F036FD012004F04CFD192004F0C2
:100B480030FD013D002004F045FD15F0FF05E6D11C
:100B58004FF48053C9F81830694B9FED6A8AD3F86F
:100B68000090DFED698A99F80C3000EE103AB8EE83
:100B7800C00A20EE080A0AF069F8644B83ED000AFF
:100B8800634B4FF06E521A605A4BD3ED047A614BA7
:100B980067EE887AB7EE007AC3ED007A99F80030EC
:100BA80007EE903AF8EEE77A5B4BC7EE277AB0EE9D
:100BB800680AC3ED007A77EE677A584BC3ED007A7E
:100BC800574B83ED027AC3ED008AC3ED018A554B7A
:100BD80083ED027AC3ED008AC3ED018A0AF036F884
:100BE800B0EE408AB0EE680A09F0D0FF20EE006A45
:100BF80068EE086A66EE007A4B4BE6EE887AFF21CB
:100C08001B2220EE087AC3ED007A67EE007AF0EE38
:100C1800675AD7EE085AE7EE087A28EE468AC3EDF7
:100C2800015AA6EE808AC3ED027A83ED038A3F4B10
:100C38001D703F4B184611F0F8FD3E4ADFF8F8E00A
:100C480012680570012112F0020F8EF800101FBF04
:100C5800417003218EF80010022118BF81705107DE
:100C680041BF9EF800104D1C8EF80050032548BF68
:100C7800455412F00A0F73460ED09EF80020042146
:100C88008154511CC9B205254554D11C0232D2B237
:100C98008EF800100621815439688D0641BF1A78F4
:100CA800551C1D70072548BF85540A0608D51A78B3
:100CB80009258554951C0132D2B21D700A25855428
:100CC8006579082D3AD00E2D41D137E00054004007
:100CD80080070020D8260020B55400089C1000206A
:100CE800FFE0CF00300E5000481C0020A824002050
:100CF800D02600205C130020701300200004004858
:100D08005414002035FA8E3C0000000050140020D6
:100D1800081400200C140020681400205814002027
:100D28006C1400205C14002040140020C61300201E
:100D3800B1100020A4100020B01000201A7802F191
:100D4800010E83F800E04FF00B0E00F802E01A786D
:100D580011F0040F4FF00C0C00F802C002F1010E64
:100D68001CBFDFF8D0C202325FFA8EFE83F800E0C3
:100D78001FBF8CF80020954A4FF0100C02F80EC0E7
:100D88001A7802F1010E5FFA8EFE4FF0120C11F480
:100D9800806F83F800E000F802C00ED094F80CC20F
:100DA800BCF1000F09D0DFF88CC202328CF80020A9
:100DB800864A4FF0130C02F80EC01A7811F4007F1F
:100DC8004FF0140C00F802C002F1010E1CBFDFF84E
:100DD80064C202325FFA8EFE83F800E01FBF8CF80F
:100DE80000207A4A4FF0150C02F80EC0182D13D1C6
:100DF8001A784FF0160E00F802E002F1010E5FFAC1
:100E08008EFE4FF0170C00F80EC002F1030E0232EE
:100E1800D2B283F800E085540D0341BF1A78551CFF
:100E28001D70192548BF8554CA0541BF1A78511C41
:100E380019701A2348BF835400219822644811F07E
:100E4800F4FC0BF01CFF634B634A1A60634BB4F865
:100E58004E111980624900230B808B7061490A602A
:100E6800614A1370B4F8962190B2604921F81300D2
:100E78000133122BF9D13B68DD0458BFB4F89C014B
:100E8800C8801B0740F1078194F89031062B00F2C7
:100E9800FC80DFE803F004070E3D5979790045F23C
:100EA800F05201E042F6F822514B1A800BF09DFFF8
:100EB800EAE007EE902ADFED4F6A4D4BB8EEE77A8D
:100EC800DFED4D7AE7EE267A42F6F8211980002305
:100ED800FCEEE77A494A17EE901A42F823100133DC
:100EE800122BF7D1464A47491160474A40201370F0
:100EF80006F0FAFB002800F0C88001234FF0070C29
:100F080090F90000414A8DE808104021404BB6E0B6
:100F1800374B42F6F8221A80394B3E4A1A603A4B50
:100F2800102240201A7006F0DFFB002800F0AD8088
:100F380001234FF0000E90F90000374A8DE8084071
:100F480040214FF4E1339AE0294B42F6F8221A8007
:100F58002B4B324A1A602C4B082240201A7006F09C
:100F6800C3FB002800F091800123002590F90000C0
:100F78002B4A8DE8280040214FF4E13306F08CF924
:100F8800284BC3F87C017CE0194ADFF8AC90DFF805
:100F9800ACC0DFF8ACE0244D244842F6F8211180BB
:100FA80019490C22062B0A704CD0002389F800300E
:100FB8008CF800308EF800301B232B701C4B02700D
:100FC80005221A704FF4E13549E000BFB110002046
:100FD800B01B0020880A0020D01D00208C0A0020A9
:100FE800A426002074260020230A0020782600204A
:100FF800CE010020CDCCCC3F0000B0C4801600202C
:10100800640000209D8C000864230020098F0008DC
:10101800A0860100898C00085D8E0008718C00088C
:10102800118E0008380800200E1700200B1600202B
:101038000F170020B01000200C1600200D170020FC
:101048000C170020002189F800108CF800108EF889
:10105800001002702121BF4A2970BF4D1370BF4B89
:10106800BF4A1A60402006F03FFB70B101210023FF
:10107800BC4A90F900008DE80A0040212B4606F092
:101088000BF9003018BF012028B9082009F006FE26
:10109800B24BB54A1A603B68B44A13F4804F1FBF7D
:1010A80012211170AD49B24818BF086042F201011F
:1010B800194003F0010003F4005581B1AD4944F62D
:1010C800206EA1F800E025B108211170A349AA4DAE
:1010D8000D6020B10C211170A049A8480860117852
:1010E800043951701A065ED5A548A64DDFF8ECA262
:1010F800C0F880A14FF000094946152200F5C270DA
:10110800DFF8DCB285F80190C5F80490C5F80890BE
:1011180011F08BFBAAF105034846CBF800300AF022
:10112800A9FB994B02201B68EB6006F0DDFA18B9A1
:10113800802009F0B3FD2EE06B7890F805E0934924
:101148000C2202FB03125278724504D00133DBB241
:10115800042BF4D900236B70DBF800306A781B7815
:1011680090F90000002B4FF00C0303FB021314BF8F
:101178004FF0030E4FF0010E00225B78CDF800E02F
:101188000192022106F088F8814B18600028CFD020
:1011980001200AF06FFB7F4B18687F4B00F5C57282
:1011A8001A600AF015FC3B685B055DD5744D7B4BF6
:1011B800D5F89CA1C3F800A0042006F095FA0421F4
:1011C800C5F8A00106F06AFA754B85F8A401082055
:1011D800C3F800A006F088FA724BDFF8089218608E
:1011E800082106F05BFA002185F8A5012C22484663
:1011F80011F01BFB8E227C2389F801204FF07D0B18
:10120800E02289F8003089F8032089F82BB0DFF84C
:10121800D89103932C220021484611F006FB039B2A
:1012280089F800308A2389F801301020A02389F832
:10123800033089F82BB0C5F8A8A106F055FA10219B
:10124800C5F8AC0106F02AFA85F8B0012020C5F8E7
:10125800B4A106F049FA2021C5F8B80106F01EFA33
:1012680085F8BC010BF07AFE3B684F4A13F4002363
:1012780018BF0123137004F06EF94C4B18606379A2
:10128800052B02BF4A4B4FF4C8721A80494B4FF4E2
:101298007A721A8098F80030474A43F0080388F8B1
:1012A8000030137823F0020313703A6840F6020303
:1012B80013406BB1414B424A1A60424B03221A70E9
:1012C800414B01221A70414A00231380404A13807F
:1012D800A3683B603F4B01221A70337863F07F03A9
:1012E800337021B0BDEC068BBDE8F08F013B092BB4
:1012F8003FF650A8D9F81800386039464FF09040AA
:1013080001F024FE4FF0904308229A613C2004F03B
:1013180048F996F891319A45BFF636A82E4A4FF00B
:10132800904B4FF4805108239161782006910592E3
:10133800ABF82830039304F029F9059A0699039B22
:1013480011857820CBF8183004F020F90AF1010A49
:10135800DFE700BF0F17002090D0030064000020D3
:101368008D8B0008F18C000835F3000864230020F9
:10137800D18C0008CE01002029F30008E18C000878
:10138800380800207C010020181B00205C3601086A
:1013980060180020E8100020D80A00208C070020E0
:1013A800C807002010080020D2240020A001002037
:1013B800DA130020EC260020F3260020C8170020AE
:1013C800C21D0020A4240020F80000207010002076
:1013D8007210002080070020000400483A1E0020F8
:1013E8009C01002098070020CC07002035FA8E3C8D
:1013F8001BB208EE103AB6F95A315FED047A344A56
:1014080009EE103AB6F95C31B8EEC88A08EE903A9F
:1014180028EE278AB8EEC99AF8EEE88A0021B0EEDD
:10142800480A29EE279A68EEA78A117009F00EFC7F
:10143800F0EE409AB0EE480A09F0A8FBB0EE408AF8
:10144800B0EE490A09F002FCB0EE40AAB0EE490A33
:1014580009F09CFBF0EE40AAB0EE680A09F0F6FB32
:10146800B0EE409AB0EE680A09F090FB60EE296A87
:1014780068EE097AF0EE665AE7EEAA5A154B29EE9D
:10148800296A28EE007AC3ED035AF0EE465A2AEE8E
:10149800400AE7EE6A5AE6EEAA7AA6EE6A7A29EEDA
:1014A8000A9A83ED010A28EE4A8A2AEE290A83ED70
:1014B800009AC3ED02AAC3ED045A83ED058A83EDB1
:1014C800067AC3ED077A83ED080AFFF70EBB00BF63
:1014D80058000020A41700202DE9F04F804D814CC2
:1014E8002A68DFF82C9202F59C432DED028B2033FD
:1014F80023607D4B1F7887B0C7B17C4909688A4251
:1015080040F21181013F1F700DE1D9F80030784891
:10151800072E98BF995D774B88BF31461B6898475F
:10152800032E0AD904EB46060137B080704B1A78AF
:10153800FEB2B2421A46E8D820E0D9F8002006F1F7
:101548000E0302EB83039988DA880028EAD04FF467
:101558007A73401A5843531A90FBF3F040F6C903C4
:1015680000F57A70984205DC40F2EE239842B8BF45
:10157800184601E040F6CA0080B2D3E75E4B1B680C
:1015880042F2010803EA080894F82830B8FA88F803
:101598004FEA581833B9B8F1000F05D0514B93F8FA
:1015A800293002E0012300E0434692F800A094F8B5
:1015B8002B20DFF860B10F210327B2FBF7F707EB09
:1015C800470784F82A10D71BD9F80010FFB2002665
:1015D80056454FDA1BB1494830F8160000E0184666
:1015E800B1F814E0864503D8B1F816E0864515D25F
:1015F800F0B20292019100930DF09AFE032EDCBF27
:101608004FF0010E94F82AC0009B0199029ADEBFA0
:101618000EFA06FE2CEA0E0E84F82AE0B8F1000F46
:1016280020D194F874E02BF81700BEF1000F06D112
:10163800022A17D92B484FF0010E80F874E0BBF846
:1016480000E0BBF802007044BBF804E07044DFF827
:10165800C8E080B22EF8160000B24FF0030E90FBDF
:10166800FEF080B2DFF8A4E00BF1060B2EF81600AE
:101678000136ADE794F82A202148224BA2F10F0E3B
:10168800DEF1000242EB0E0284F88E206AB11E4A97
:101698001268570109D40268D9689A60521AC82A90
:1016A8003CD9012283F8212038E002689868DA6082
:1016B8005B68121A9A4288BF124B4FF0000184F8F7
:1016C800281088BF83F821100026564526DAF0B284
:1016D8000DF02EFE0D4B23F816000136F5E700BF7E
:1016E800D4260020F8090020A02600209C260020EF
:1016F8006423002064000020781B0020FC090020DF
:10170800181B0020A4260020AC10002078260020FA
:1017180074260020240A00206E0A002094F82B303A
:10172800013384F82B308F4B1A6812F4805F984687
:1017380005D08D4B1B68DE0701D40DF09CFBD9F852
:101748000020937A2BB3013B8849127B31F8133080
:101758001AB1C3F53B6308339BB21BB2A3F57A7386
:10176800B3F57A7FA8BF4FF47A7323EAE37307EEE1
:10177800903A9FED7F7A7F4AF8EEE77AC7EE877A4C
:101788009FED7D7A67EE877AFCEEE77A17EE903A5E
:101798001380D8F80030794F13F4807F00F003816C
:1017A8002A68774BDFF8DC919A4205D999F802202C
:1017B80012B9012289F8022099F80220002A00F0C3
:1017C800F280704A3E7892F82150674A681E454276
:1017D80011684541002DC1F38063C6F3800600936C
:1017E800924614BF4FF0000B4FF0030B99F82020DE
:1017F800052A00F2D280DFE802F0034D527584A179
:10180800002E3AD0D4F89000B4F8941006F00FF8EF
:10181800012809D15C495D4A09681268C9886420B1
:1018280000FB0122C9F81020009B6BB1564A1268D0
:1018380012794AB10DF056FD032289F820204FF4A1
:101848007A72C9F81C20D1E7002D40F0A6804F4AD3
:10185800D9F8101010684B4A88420AD901920DF045
:1018680041FD019A032182F8201040F6B831D16178
:10187800BCE7012182F82010B8E7009B4FF4806094
:1018880013B109F0FBF901E009F0E8F90022C9F801
:10189800102082E0002D46D10DF024FDA6E725B1E9
:1018A800052289F82020012000E0284666B1D4F8F6
:1018B8009020D1892D4A1180518091803249096840
:1018C8004988D1804FF0020B304A1168D9F81420AA
:1018D800914201D8002E5DD147F23052C9F81C2040
:1018E800032221E03A7842F002023A700DF0C3FA7E
:1018F800264AD9F81C1012680A44C9F8182004228C
:1019080012E0224A9DB11168D9F81820914244D9B1
:101918001F4A12781AB9DAF80020D1073DD43A786C
:1019280022F002023A70052289F820205EE7126848
:10193800D9F81C100A44C9F818202EE01249134A95
:1019480009681268C988642000FB0122C9F81020C0
:101958004FF48060002289F8202089F8032009F0DC
:101968007DF943E7781B0020AC1000207826002082
:1019780000007A440C11002000C07F44F3260020A8
:10198800404B4C00A426002070260020181B002085
:101998000200002000287FF429AFBBF1000F02D01D
:1019A800584605F09FFF8A4D05F5C470B5F84E11ED
:1019B80005F03DFF834668B90DF086FC854BC3F8FA
:1019C80000B0C3F804B0C3F808B0834B00221A6013
:1019D8005A609A603B785A0736D5D8F80030DB064B
:1019E80032D57E4B1B78DE062ED47D4B1B7893B107
:1019F80095F8E031BBF1000F15D17BB1794B1A682E
:101A0800D4F898309B1A002B08DA0DF034FA764B8C
:101A180083F89CB018E0BBF1000F0DD1102005F041
:101A280061FF01230EE03BB16E4A12684FF47A71F0
:101A380001FB0323C4F8983094F89C3023B105F0D7
:101A48003BFF002384F89C30002295F8DEA195F82E
:101A5800DF11B5F898E1B5F89AC11346634E0096C0
:101A680036F912009B087045C4BF63F07F03DBB2F0
:101A780001326045B8BF43F04003042AEED194F820
:101A88009D2059489A4205D190F89E20F92A04D8F9
:101A9800013200E0002280F89E2084F89D30504BEF
:101AA800534E1A789946E2B93368D80708D5BBF17E
:101AB800000F16D13B78D90713D50DF059F810E06F
:101AC8003B785A070DD5484B93F828304BB1494B12
:101AD800DB7833B911B10DF0CEF902E0BBF1000F9C
:101AE800F9D094F89E30404ADFF820B1142B40F02A
:101AF800A88099F800301AF1000A18BF4FF0010ABF
:101B08006BB392F89D305F2B11D13B7803F004033F
:101B180003F0FF0113B10DF0AEF908E00B200291BC
:101B2800019205F0DFFE019A029982F89E10BAF13F
:101B3800000F14D094F89D307D2B10D13B7803F022
:101B4800040303F0FF0213B10DF095F907E00B2031
:101B5800019205F0C7FE244B019A83F89E203B783A
:101B680003F0040303F0FF01002B6AD194F89D30C1
:101B78001D4A572B11D1204B4FF47A721A80D8F88E
:101B880000301B0601D509F085FF1C4B1B6813F0BC
:101B9800080356D11A4A138053E0D8F800004007CA
:101BA80036D55A2B34D1174B187820B11970164BEB
:101BB80001221A7045E092F89F3083F0010382F801
:101BC8009F300BB10C2000E00D2005F08BFE38E0B3
:101BD800481C00202C150020A815002018110020F2
:101BE80002000020181B0020F80900207826002099
:101BF800AC100020A4260020EC260020A410002011
:101C0800041100200514002006140020E81000200C
:101C18005D2B00F0E0845B2B00F0FE845E2B00F06F
:101C2800FD84562B01D109F0C5FA99F80030002B34
:101C380000F0A58494F89D306F2B40F09A840CF046
:101C480097FFD8F800305A0732D594F89F30A3B1DF
:101C58003B785B0711D5009BB3F90620B5F898319E
:101C68009A420ADD336813F0010301BFAD4A3221FD
:101C78001180AD4A08BF82F89F303368D8030AD56F
:101C8800AA4B1A782AB9AA4A127812B9A54A322157
:101C9800118001220BE0A64A13784BB13B7803F080
:101CA800040303F0FF011BB9A24B117001221A7043
:101CB800DBF800A0002333600AF17B090AF1CB0BA3
:101CC80099F8002099F8013019F8010C9A420BD2C2
:101CD800494605F075FD38B119F8022C012303FABD
:101CE80002F233681343336009F10409D945E7D197
:101CF800914B1B7843B1914B914E1A6812F0020F29
:101D0800994640F03F8336E30AF1CA060AF5897915
:101D18003278737816F8010C9A4225D2314605F0CC
:101D28004FFD08B3B37896F804E0864A96F803A006
:101D38007D480C21013B01FB0E4103EB4303134497
:101D4800D1F8A4209A420FD0C1F8A430002390F80B
:101D5800D020C1F8A830012303FA0EF322EA0303C6
:101D680081F8A0A080F8D03006364E45D0D1764B09
:101D78001E68764B1B68029394F828300393744BC3
:101D8800009300230193009B1B68002B00F0E8825E
:101D980093F800A0BAF1000F00F0E282009A0299CD
:101DA80052688A1A002A0CDB01F5FA7200994A6017
:101DB800019901228A4094F8D01021EA020284F89D
:101DC800D020039A002A00F0CB82009A597812F8A2
:101DD800042C0432D2B2002940F081825D4931F9E5
:101DE8001210B5F8962102F1C800814202DD93F87D
:101DF80002B015E0C83A914203DA9978C1F1000BB4
:101E08000EE0019A0123934094F8D02022EA0303BC
:101E180084F8D030029B009A03F5FA7353609FE26E
:101E280094F8D030019A1341D90700F19982BBF197
:101E3800000FCCBF0220012005F078FD0AF1FF3326
:101E4800DFF8E490132B00F28382DFE813F014002C
:101E5800250037004B0064008B00EE005101B801EB
:101E6800E601160281024B005A008B00EE00510178
:101E7800C0002301880196F80090D944B9F1FA0FFF
:101E8800A8BF4FF0FA0929EAE979304686F80090A8
:101E980005F07CFC01200FE096F80190D944B9F1D7
:101EA800640FA8BF4FF0640929EAE979304686F83B
:101EB800019005F06BFC02204946DBE196F803A08F
:101EC800DA44BAF1640FA8BF4FF0640A2AEAEA7A42
:101ED80086F803A03046D9F8D41005F00DFC03208D
:101EE8005146C7E1717959446429A8BF642121EAA0
:101EF800E17171710D2005F0CBFCBAF10D0F00F006
:101F08002782317959446429A8BF642121EAE17103
:101F180031710E20AEE1B179594481F30801B171F4
:101F28000520A7E1EC130020F80900200414002084
:101F38000514002006140020F5260020AC1000200F
:101F4800A4100020C43A010814110020181B002016
:101F58009C0A00207826002000007A440000C8422D
:101F680000000000D9F8D8301A78022A20D107EEEC
:101F780090BAB8EEE70A5FED077A93ED097A80EE3A
:101F8800270A30EE070AB5EEC00AF1EE10FA07D4B8
:101F9800B4EE670AF1EE10FAC8BFB0EE670A01E0C6
:101FA8001FED110A83ED090A0F2005F05BFC0AE01A
:101FB80099785944C829A8BFC82121EAE1719970C4
:101FC8000F2005F065FCBAF10F0F00F0C181D9F8B8
:101FD800D8301A78022A1ED107EE90BAB8EEE78AEE
:101FE8005FED227A93ED080A88EE278A38EE000A18
:101FF800B5EEC00AF1EE10FA07D4B4EE670AF1EEB6
:1020080010FAC8BFB0EE670A01E01FED2B0A83ED96
:10201800080A122056E159785944C829A8BFC8218E
:1020280021EAE1715970122024E1D9F8D8301A78E0
:10203800022A20D107EE90BAB8EEE70A5FED397AA6
:1020480093ED0C7A80EE270A30EE070AB5EEC00A47
:10205800F1EE10FA07D4B4EE670AF1EE10FAC8BF31
:10206800B0EE670A01E01FED420A83ED0C0A10206A
:1020780005F0F8FB0AE0197B5944C829A8BFC82114
:1020880021EAE1711973102005F002FCBAF1100F72
:1020980000F05E81D9F8D8301A78022A1ED107EEEE
:1020A80090BAB8EEE78A5FED537A93ED0B0A88EEA3
:1020B800278A38EE000AB5EEC00AF1EE10FA07D406
:1020C800B4EE670AF1EE10FAC8BFB0EE670A01E095
:1020D8001FED5D0A83ED0B0A1320F3E0D97A59440A
:1020E800C829A8BFC82121EAE171D9721320C1E02B
:1020F800D9F8D8301A78022A22D107EE90BA1FED03
:102108006A0AF8EEE77A87EE800AD3ED0F7A30EEA6
:10211800270AB5EEC00AF1EE10FA09D45FED717A1C
:10212800B4EE670AF1EE10FAC8BFB0EE670A01E034
:102138001FED750A83ED0F0A112005F093FB0AE0E5
:10214800997D5944C829A8BFC82121EAE171997528
:10215800112005F09DFBBAF1110F00F0F980D9F8B4
:10216800D8301A78022A20D107EE90BA1FED860AD5
:10217800B8EEE78A88EE008A93ED0E0A38EE000A78
:10218800B5EEC00AF1EE10FA09D45FED8C7AB4EE20
:10219800670AF1EE10FAC8BFB0EE670A01E01FED5A
:1021A800900A83ED0E0A14208CE0597D5944C82901
:1021B800A8BFC82121EAE171597514205AE0D9F85D
:1021C800D8301A78022A1ED107EE90BAB8EEE78AFC
:1021D8005FED9E7A93ED0A0A88EE278A38EE000AA8
:1021E800B5EEC00AF1EE10FA07D4B4EE670AF1EEC4
:1021F80010FAC8BFB0EE670A01E01FEDA70A83ED29
:102208000A0A09205EE0D9785944C829A8BFC8211C
:1022180021EAE171D97009202CE0D9F8D8301A7870
:10222800022A1ED107EE90BAB8EEE78A5FEDB57ABA
:1022380093ED0D0A88EE278A38EE000AB5EEC00A3B
:10224800F1EE10FA07D4B4EE670AF1EE10FAC8BF3F
:10225800B0EE670A01E01FEDBE0A83ED0D0A0A2001
:1022680030E0597B5944C829A8BFC82121EAE17147
:1022780059730A2005F00CFB6AE0D9F8D8301A78AF
:10228800022A22D107EE90BA1FEDCD0AB8EEE78AEE
:1022980088EE008A93ED100A38EE000AB5EEC00AFF
:1022A800F1EE10FA09D45FEDD37AB4EE670AF1EED5
:1022B80010FAC8BFB0EE670A01E01FEDD70A83ED38
:1022C800100A0B2005F0CEFA42E0D97D5944C829FE
:1022D800A8BFC82121EAE171D9750B20CAE70129F5
:1022E80036D19878BD4B33F91230B3F5617F05DBF1
:1022F80040F633029342A8BF134601E04FF46173DE
:10230800BAF10C0F24D14FF4966292FBF0F0B44A64
:10231800A3F5617393FBF0F35FFA83F913784B45E8
:1023280016D0B9F1040F34BF4B4602231370AD4ADF
:102338000AFB035303F2E663136008F07BFD504683
:10234800494605F0A5FA09F10100C0B205F0EEFA18
:10235800019A0123934094F8D020134384F8D03095
:10236800019B01330193009B0C330093019B042BC9
:102378007FF409ADBFE4D8F80030DA0510D59A4BE0
:10238800DB786BB133689B070AD5984B1B8813F031
:10239800010A0AD10CF098FF012008F06FFC04E054
:1023A800012008F05BFC012300E00023D9F800209D
:1023B80050070DD563B1012008F050FC8B4B1B88EA
:1023C800990708D40CF080FF022008F057FC02E0BF
:1023D800022008F043FC33689A0609D4D9F8003083
:1023E8001B0540F194804FF4807008F047FC92E0A0
:1023F8007F4BDFF8F8A11B7813F0020F53D07D4B09
:102408001B78042B4FD9D9F8003013F4007B0FD078
:10241800BAF80030DE063AD4102008F02FFC20204D
:1024280008F01CFC7448011D09F088FA02232AE010
:10243800BAF8006006F01006B6B22EB1102008F007
:102448000DFC012684F8DCB0D9F80030580512D507
:10245800D4F8E03069495A89B1F90030002BB8BF87
:102468005B42934207DAB1F90230002BB8BF5B42F6
:102478009342C0F2FA80BAF80030990608D52020B5
:1024880008F0ECFB002384F8DC30012600E000268D
:1024980094F8E430BBB90E2005F024FA584B012219
:1024A80083F8E4200FE0BAF8003003F03003002B83
:1024B80094D0102008F0D2FB202008F0CFFB002396
:1024C80084F8DC3001E0002E88D04E4B002003F168
:1024D800280603F150044C4A002122F810104B4AF8
:1024E800596022F810100432716022F8101000228E
:1024F8001A609A603260B26022606160A260143330
:102508001436143400287FF469AF0120E3E74FF450
:10251800807008F0A3FB6B79082B01D00E2B02D139
:10252800402008F09BFBD8F800305A0540F1B380F2
:1025380095F80C321BB93B7813F0040F03E0D9F877
:10254800003013F4002F0BD0314B00221A703C20BE
:102558000AF090FC002800F09E800BF07DFAF6E768
:102568000AF0FCFC07B0BDEC028BBDE8F04F0AF0A6
:1025780086BBBAF1000F02D07E2B3FF460AB94F813
:102588009D30972B05D1234B4FF4C8721A80FFF763
:1025980058BBA72B06D1164A137843F004031370CF
:1025A800FFF74FBB0022BB2B059201D1022303E0AA
:1025B800B72B04D14FF6FE73ADF816303EE0BE2BB4
:1025C80001D1022304E0BD2B7FF43BAB4FF6FE7331
:1025D800ADF8143032E0012021E000BF7826002059
:1025E8007C24002014110020A4260020A81000201C
:1025F8001811002019110020301100201415002096
:10260800F8090020E00A0020EE260020580B0020E0
:1026180069230020DA130020022000E003205FFA7B
:1026280080F909F1FF3385F8E43608F069FB08F012
:1026380025FC484605F07AF9FFF703BBDBF80030C4
:10264800BDF81410B3F858200A44A3F85820BDF870
:102658001610B3F85A200A44A3F85A2008F0AAFD25
:10266800002384F89E30FFF7ECBABAF800309B06D6
:102678003FF50EAF202008F001FB0948094B011D6A
:102688001A685B684360026009F058F9064B012636
:1026980083F8DC60FCE607B0BDEC028BBDE8F08F88
:1026A800381100201C110020F8090020026BC168B5
:1026B800034610B5406942B11A6C8C1A013A005DA4
:1026C80008BF0A46C0B21A6410BD1A6A805C01329B
:1026D8008A4228BF0022C0B21A6210BD436B13B1F0
:1026E80090F844007047836A406A1B1A5842584160
:1026F8007047036B13B15B68016C01E0C369016A41
:102708008B423CBFC2689B18581AC0B27047836A94
:102718008169426B1944D160416A99429DBF016940
:10272800CB1A5360CB1A96BF0023536083624FF0D5
:10273800000380F84430136888BF816243F00103C6
:1027480013607047436A8269D154436A026901334E
:10275800934228BF00234362436B1BB11B68DB070E
:1027680005D4D4E7026D136843F080031360704703
:1027780010F80A3C0133DBB20A2B84BF10F8131C93
:10278800044A00F80A3C82BF002322F8113000F8FE
:102798000A3C7047EC160020334A136C90681944C1
:1027A800081A40F68C23984270B513469160D060A1
:1027B80051603BD9127893F945108A4210460BD1E3
:1027C800111F082908D893F84610182901D8013193
:1027D80003E083F8442002E0002183F8461093F9CF
:1027E80044402149A24219D191F84740B4B10C3173
:1027F8000024944206DA1D4D51F8046F25F8146040
:102808000134F6E70C2805D01849002421F81040B7
:102818000130F7E7164801780131017083F8452047
:10282800002201211A7083F8471070BD92F84710F2
:10283800C9B1A0F2EF2440F2DA518C4208D81178DD
:102848000B2905D80B1D0131117042F8230070BD0A
:10285800002283F84720074B03F13002002143F898
:10286800041F9342FAD170BD68080020EC160020BE
:102878006C01002074080020024A136C01331944CB
:102888001164704768080020024B53F820301B6819
:102898001960704790110020064B53F820301A68D1
:1028A8001B89A1F57A7159434FF47A7391FBF3F1BF
:1028B8001160704790110020F0B5046D8668236898
:1028C80023F0010323608379054613F0020F407952
:1028D8000CBF4FF0000E4FF4005E13F0040F14BF4E
:1028E8004FF48067002710F0010F14BF0421002166
:1028F8008307206820F001002060626822F44052BB
:102908004EEA02026260226822F4B05323F00C03FC
:1029180048BF41F008013B430B432360A36895B0CF
:1029280023F44073A360684606F0C6FC284B9C421B
:1029380001D10C9B0EE0274B9C4201D10D9B09E075
:10294800254B9C4201D10E9B04E0244B9C420CBFBA
:102958000F9B109B2268A879170448BF5B00B3FB44
:10296800F6F206FB1233B3EB560F236828BF013289
:102978001E0441BF4FF6F073C2F34201134041EA0F
:1029880003026B7992B213F0020FA28100F00101E9
:1029980014BF4FF400320022DC0748BF42F48032F3
:1029A8002B6D11B159680A4302E0596821EA020205
:1029B8005A609A6801074CBF42F0080222F00802E8
:1029C8009A601A6842F001021A6015B0F0BD00BFA3
:1029D800003801400044004000480040004C0040DE
:1029E800417169E7816067E7026D036B70B5044662
:1029F800D5699BB9A90611D5C36A1BB1908C80B261
:102A080098470BE0E169928C40694E1CD2B2E661AE
:102A18004254E169E268914228BFE361616BA1B960
:102A28002A0612D5636AA26A9A42236D09D0501CFD
:102A3800A669A062B25C1A852369984205D3A1628F
:102A480003E01A6822F080021A602B0742BF236D48
:102A580008221A6270BD0D4B0D484FF400525A609F
:102A68000C4A11684FF6FE730B401360426B1168F5
:102A78004FF6FE730B401360426A836A9A4200D095
:102A880045E6012380F84430704700BF000002404B
:102A9800AC1A0020440002402DE9FF471D46B24B06
:102AA8009DF8306098428846174640F08680AF4BC4
:102AB800AF4A1A60AF4A5A6102F580729A614FF4C0
:102AC8008072DA601A61AC4A1A63143A5A63A2F542
:102AD8004842203ADA6404329A649F601865A74B2A
:102AE8009A6942F480429A615A6942F001025A6135
:102AF80002238DF80C30032316F0010A8DF80D30EF
:102B08004FF000038DF80E3014BF02230123310764
:102B18008DF80F301BD54FF090444FF40079CDF865
:102B280008908AF001038DF80E30636A23F0F003F1
:102B38006362636A43F070036362204602A906F089
:102B480029FDBAF1000F28D1C4F8189025E0AA078A
:102B580010D504A94FF4007341F8083D4FF0904098
:102B6800436A23F0F0034362436A43F0700343620D
:102B780006F010FDEB0710D504A94FF4806341F867
:102B8800083D4FF09040436A23F470634362436A00
:102B980043F4E063436206F0FDFC0E238DF8043035
:102BA8000022012301A88DF805308DF806208DF844
:102BB80007306E4C09F0D8FD75E0714B984240F033
:102BC800F380704B6A4A1A604FF48072DA601A61B7
:102BD8006D4A5A6102F580729A61684A9F60186569
:102BE800D36943F40033D36102238DF80C300323F7
:102BF80016F0010A8DF80D304FF000038DF80E30F5
:102C080014BF0223012334078DF80F301AD55F4C07
:102C18004FF02009CDF808908AF001038DF80E30A6
:102C2800236A23F470032362236A43F4E0032362D4
:102C3800204602A906F0AEFCBAF1000F24D1C4F870
:102C4800189021E0A8070ED504A9202341F8083DD3
:102C58004E48036A23F470030362036A43F4E003F3
:102C6800036206F097FCE9070ED504A9402341F852
:102C7800083D4648036A23F070630362036A43F021
:102C8800E063036206F086FC26238DF804300022F8
:102C9800012301A88DF805308DF806208DF807303E
:102CA80009F062FD374CC4F82C80012384F84430C5
:102CB80000232362E361A36263626571A760A67162
:102CC8002046FFF7F9FDEA0729D5206B00B3D4F8B1
:102CD8004C80E668676906F063FA236B216D1A6811
:102CE80022F4FF4222F0700242F48552B6B21A6012
:102CF8005E60C3F80880DF601A6842F001021A605B
:102D08008A6842F040028A605B689BB2236406E0EE
:102D1800236D20221A621A6842F020021A60AB075B
:102D28003BD5606B002833D0A66C256906F038FACD
:102D3800636B1A6822F4FF4222F0700242F4845254
:102D480042F010021A60ADB200225D609E60DA6047
:102D5800196841F0020119605A605A60226D93683F
:102D680043F08003936018E000380140AC1A00205B
:102D7800003B0108600B0020580002400010024090
:102D880000440040581A0020600D0020000C004844
:102D9800226D136843F080031360226D136843F0BB
:102DA80001031360204600E0002004B0BDE8F0876E
:102DB8003D4B1B78012B30B514BF00240324B1B957
:102DC800036A23F0010303628169036A21F0F301B6
:102DD80023F00A0341F0010142F001021A4341EADB
:102DE800041181610262836923F00C031BE004294A
:102DF8001DD1016A4FF6EF730B4003628169056AC2
:102E0800120121F473414FF65F7342F0100241F44E
:102E180080712B4092B2134341EA0431816103620D
:102E2800836923F4406383618369836130BD082922
:102E3800016A1AD14FF6FF630B400362C169036A46
:102E48009BB289B223F4206343F4807321F0F30129
:102E580043EA022241F0010192B241EA0411C16140
:102E68000262C2694FF6F37319E04EF6FF730B4026
:102E78000362C369056A40F6FF41194045F6FF73CE
:102E88002B4043F4805343EA023241F4807192B2FA
:102E980041EA0431C1610262C2694FF2FF33134053
:102EA800C361C369C36130BD6408002038B510F838
:102EB8000E2C50F8043C044652B9012200F80E2C9E
:102EC80020F80C1C997A18680222BDE838406FE790
:102ED80030F80C2C20F80A1C891A89B220F8081C32
:102EE800074A10F80F0C002522F8101004F80E5CA1
:102EF8001868997A2A46FFF75BFF04F8065C38BD24
:102F0800EC160020044B53F820301BB107289CBF57
:102F18001B681960704700BF90090020084A1368B1
:102F28009B050BD5074B00211970074908684FF618
:102F3800FE7303400B604FF400735360704700BF8B
:102F480000000240F22600203000024073B5064619
:102F58000D46002401232A88A34013421AD0AA78D8
:102F6800009302F003038DF80430EB78022B03D0B2
:102F7800032B0CBF032301238DF805303046C2F321
:102F880001136946C2F381028DF806308DF80720D7
:102F980006F000FB0134102CDCD102B070BD2DE925
:102FA800F743DFF81C9299F8004405468E460068FE
:102FB8001146164698467246631C89F8003408F094
:102FC8002BFE2B89ADF8043001A9022368688DF81F
:102FD80006308DF80730FFF7B9FFAB7A2A6809F297
:102FE80004472401274449460C2B00F2B780DFE848
:102FF80003F007B5B5B53EB5B5B56AB5B5B5930037
:10300800136ADFF8C0C123F001031362136AD2F810
:1030180004E0906920F4803020F07300624540F0AD
:10302800700012D00CF5006C62450ED00CF5406CA7
:1030380062450AD00CF5806C624506D00CF5806CB0
:10304800624502D043F0030307E023F00E032EF499
:10305800407E43F003034EF4807EC2F804E09061A2
:10306800C2F834801362936943F0080329E0136AB5
:10307800DFF850C123F010031362136AD2F804E09A
:10308800906920F0807020F4E640624540F4E0400A
:1030980006D00CF5006C624502D043F0300307E01F
:1030A80023F0E0032EF4406E43F030034EF4806EBC
:1030B800C2F804E09061C2F838801362936943F45F
:1030C800006393614AE0136ADFF8F8C023F4807361
:1030D8001362106AD2F804E0D369624523F07303DF
:1030E80043F0700306D00CF5006C624502D040F442
:1030F800407007E020F460602EF4405E40F44070B9
:103108004EF4805EC2F804E0D361C2F83C801062DD
:10311800D36943F0080320E0136ADFF8A8C023F45A
:1031280080531362106AD2F804E0D369624523F42D
:10313800E64343F4E04340F4405003D00CF5006C00
:10314800624501D14EF4804EC2F804E0D361C2F862
:1031580040801062D36943F40063D3612B7B1BB1B9
:10316800536C43F40043536413889BB243F0010348
:103178001380AB7A0C2B19D8DFE803F0071818185E
:103188000B1818180F18181813000B1902F134002F
:103198000AE00B1902F1380006E00B1902F13C00B5
:1031A80002E00B1902F14000C3F804040C4438464D
:1031B800A4F80C64C4F8082403B0BDE8F08300BF89
:1031C800600B0020002C01402DE9F04FC14BB3F9F2
:1031D8000610C14B2DED028B1F687A8991B0914280
:1031E80001930EDBB1F5FA6FFC79BDBF8B1A63430F
:1031F800A2F5FA64C4F16404BCBF93FBF4F464342C
:1032080000E06424B54AB64BB2F896A192F95E2163
:103218001868049092B20592054600220293AD4BBD
:1032280033F912300393CAEB030303F2F31640F2A7
:10323800E63086424FEA420B03D8002BB8BF5B4208
:1032480001E04FF4FA73022A049E4FF064002FD075
:1032580096F811E1BEF1000F04D07345CCBFCEEB58
:1032680003030023DFF8C0E293FBF0FC6FF063096F
:103278003EF81C809B4E09FB0C390CF1010C3EF901
:103288001CE00FFA88FCCCEB0E0E0EFB09FE9EFB31
:10329800F0FEC64426F80BE0BE1836797343924E0A
:1032A80093FBF6F364339BB2634393FBF0F02EE099
:1032B80096F812E1BEF1000F04D07345CCBFCEEBF7
:1032C80003030023DFF84C8293FBF0F06FF0630CEC
:1032D8000CFB003938F910E00130002B38F91000E8
:1032E800CEEB000000FB09F9BDF8140099FBFCF9CE
:1032F800CEEB090919FB00F97A48A0F80490B879CF
:10330800B8BF5B424343784893FBF0F064306B7876
:10331800764E4FF0640E434393FBFEF3B354744E62
:10332800EB7A434393FBFEF3B3546B7D6D4E5843E6
:10333800704B90FBFEF0022A98546F4B0FD183F824
:1033480002E0039B53450EDB644CB4F8982191428C
:1033580015DBB1F5FA6FA8BF4FF4FA6110E09C5481
:10336800039B534504DA36F80B305B4226F80B30E2
:103378000132032A05F101057FF451AFE4E7114654
:10338800891A4FF47A73DFF8A4E1564D59436FF068
:103398006303C2F5FA626427B1FBF2F191FBF7F21D
:1033A8003EF8120003FB0211013203B23EF912206B
:1033B800D21A514391FBF7F30344F3804F4B1B8818
:1033C8005B0635D54E4B4F4A1B881288DFED4E7A87
:1033D8009B1A1BB208EE103AB8EEC88A28EE278A64
:1033E800B0EE480A07F032FCF0EE408AB0EE480A28
:1033F80007F0CCFBB5F9023006EE903AB5F900308B
:10340800F8EEE66A07EE903A20EE667AF8EEE77A8A
:10341800A7EEA87A67EE807ABDEEC77AE6EEA87ABC
:1034280017EE103AFDEEE77A2B8017EE903A6B8094
:10343800364D2B689F0740F1A180354B354F1A68F0
:103448007B6945F20721D31A8B4240F397807A6152
:1034580006F08EF9304BDFF8D8901A78032A984690
:10346800B9F8003022D10A2B2AD90023282088F85D
:10347800003002F096F806F07BF9284B188806F021
:1034880061F9274B1A68D37890FBF3F001300828CC
:10349800244BA8BF08201870537980B213FB00F39F
:1034A8003B83137913FB00F0788309E00A2B07D8D4
:1034B80003231C4A88F80030002313703B837B8366
:1034C80098F80030144A012B3DD033D3022B4CD04E
:1034D80054E000BF7826002014110020481C00206A
:1034E800E8100020141500200CFEFFFF90150020A6
:1034F80066100020981500201C150020A810002038
:1035080004110020D024002035FA8E3C781B0020BE
:10351800D426002058100020A4240020CC17002016
:10352800C8170020F8000020F6140020DE14002040
:10353800581800203A8BB9F800309A421EDD012352
:1035480088F800300FE0B9F800107B8B8B4202DD61
:10355800022313700FE09C4B1B8B0133994202DD51
:10356800002313700AE0082006E07B8BB9F80020DE
:1035780001339A42E3DC072004F0B4F92F683D05D3
:103588006DD5924B904D1B68EA69C2EB030845F272
:103598000722904563DDEB618D4BB6F906B0D3F891
:1035A8000090B4F84E1199F80A308A4E012BABF509
:1035B8007A7B03D03CD3022B1AD03BE02A6A08213D
:1035C80092FBF1F3D31A00222B62AA8493FBF1F346
:1035D80040F6E4429BB25343B9F80820C2EB1333D8
:1035E8004FF47A725343B9F9062093FBF2F320E0C3
:1035F800794BB9F808A01B78C6F800A0580719D568
:10360800764804F014F920B917F0100F18BF4FF0DE
:10361800000B32220BFB0BF393FBF2F3B9F90620F4
:103628005B445A434FF47A7392FBF3F3534400E03C
:1036380000233360D5E90A013368694A03FB08F8B7
:103648004FF47A7398FBF3F810EB080041EBE8713C
:103658000023C5E90A010CF0FFF8624B1860624EBE
:103668003368D90427D53A0622D5604B1B789B07C7
:103678001ED55F4B187804281AD900225D4BD7183D
:103688000521951C4FF00A0E122AD154E9B287F889
:1036980001E004D0B0EB510F2A46EFD800E0142126
:1036A8005A18322002F8010CFF225A540F2000E069
:1036B8000A2004F017F9504D2A68002A55D04F4BBC
:1036C8004F4F18683968814298464ED84D4BDFF8FD
:1036D80040911878516808BB01201870B9F800307B
:1036E800CB5C5BB31378013B00FA03F2D4F81037D4
:1036F8001A4201D101F06EFF434B01221A700BF000
:1037080063FEB9F80030CBB92B681B78053B012B59
:1037180014D801F020FF3D4B18600FE04FF0000A6D
:1037280083F800A0B9F80030CB5C3BB1504601F0FB
:1037380051FF354B83F800A00BF046FE2A68B9F814
:10374800003052683248D25CFE2A01D100230BE0D7
:10375800FF2A02D104F0B0F807E0D8F800500A2197
:1037680011FB02523A60013303801B4D2B785F072F
:1037780004D5284B4FF480521A8561E03268D0078F
:103788005CBF43F001032B70184B1B7819075EBF11
:103798002B7823F001032B70D30242BF2B7823F040
:1037A80001032B701C4B1A88174B1AB11B4A12685D
:1037B800970702D41A4A1288A2B302221A702B78E9
:1037C80023F001032B7032E058100020D42600208B
:1037D800C817002010110020F3260020D01D00205B
:1037E800407E050008110020AC10002018110020B0
:1037F80019110020B424002010150020181B0020E7
:103808000815002004150020C82600205426002092
:103818000C15002000040048DA130020A410002032
:10382800EC2600202978CE0758BF02221A7001F032
:1038380092FEB14B1B68C01A002801DB0BF0C4FDD7
:1038480009F08CFBAD4B03931E78002E00F0AD8081
:10385800AB4F3B68002B00F09D86386801F0C9FE2D
:10386800002800F09786A64BA64C186801F0BEFE0B
:10387800092801D03F2852D14FF000092668DFF807
:10388800C4824D4636B1A048D8F8001032460FF031
:1038980019F810B9C14605B945469C4B08F11008FE
:1038A8009845EFD3EDB1D5F800C0D9F8008023686A
:1038B8001CF803E018F80300704512D15A1C92490D
:1038C80058B92D2B09D8DFF83CE2CEF800204FF08C
:1038D800200E01F803E0885403E001F803E02260B9
:1038E800E5E723680BB14D4510D089480AF0A6F9E1
:1038F8004D4507D855F8100B0AF0A0F909200AF031
:1039080095F9F5E783480AF099F9002623689E425D
:10391800A3D27D4B985D0AF089F90136F6E7236852
:10392800002B40F01C86042840F05786764806F0A5
:103938006BF800F02FBED8F80000DFF8E89101F02E
:1039480058FE40B3D9F8000001F050FEDAF8003014
:1039580093F848208346002A35D124286CD10122C7
:1039680083F84820DAF80030DFF8B49193F848B0CB
:10397800BBF1060FDFD193F8490000F0BBFE80468B
:10398800002800F081803B6898790AF0A2F83B682B
:10399800002283F84820604B93F83730002B40F022
:1039A800CC854C36982E00F0F5855C4BF21892F8D1
:1039B8004A100129F5D15A4FF3583A60594ABA4684
:1039C80013609046B7E7012A04D14D2814BF00229E
:1039D8000222C5E7022A04D13C2814BF0022032290
:1039E800BEE7032A0AD140284FF000029FBF1A7190
:1039F800DA715871987198BF0422B1E7042A08D186
:103A08009A7983F8490080EA020B83F806B0052208
:103A1800A6E7052AA6D159791A799142997906D942
:103A280041409971511C1971134418729AE78142E7
:103A38000CBF0622002293E72B783B4A590791D402
:103A48002328D9F8003012D10492039A374801216B
:103A580011702B490B6030490B630AF0EFF82D48C1
:103A68000AF0ECF8049A137843F002031370304B11
:103A78001B681B785B4501BF2E4B2F4A1A602F4BE2
:103A880004BF2F4ADA606DE7D9F8002092F8493070
:103A98004E2B00F0B18476D8352B00F05F821BD80E
:103AA800292B00F0588409D8252B00F02F84272BC8
:103AB80000F03384232B40F08C8514E22D2B00F08A
:103AC8005B84332B00F0C4842B2B40F0828509F0F3
:103AD800E3FF607100F02CBD3E2B00F0EA8033D884
:103AE800392B00F027843C2B00F0ED80372B40F079
:103AF800708500F0E1BC00BFCC260020F526002030
:103B0800A02400209418002064180020983E010882
:103B1800105901081559010858100020B01B002041
:103B2800982400209C240020F326002045590108F1
:103B38006C230020FC9F0020EFBEADDE00ED00E00E
:103B48000400FA05083D0108432B00F0928406D8CA
:103B5800412B40F03E854FF0000800F07EBC442B1E
:103B680000F0E2844C2B40F0348509F095FF84F88E
:103B7800D60109F091FF84F8D70109F097FFA4F85E
:103B8800D80100F0D5BCD12B00F07F831AD8CC2BFC
:103B980000F0228209D8C92B00F05083CA2B00F00C
:103BA800A180C82B40F0158542E0CE2B00F0398368
:103BB800C0F02E83CF2B00F06382D02B00F01D8342
:103BC80000F007BDD62B00F0948207D8D32B29D05C
:103BD80015D3D42B00F0988200F0FBBCEF2B58D003
:103BE80005D8D82B40F0F5844FF000090DE1F22BF1
:103BF80000F0D882FA2B00F01D8300F0EABC2B7885
:103C080003F0040303F0FF08002B40F0918409F04F
:103C180043FF022884F8E40640F2F582E34B83F878
:103C2800E486F0E209F042FFE14B988600F080BCA0
:103C380092F805804FEA5808B8F1120F03D909F035
:103C480015F900F075BC4FF00009C14507D209F01D
:103C58002DFF07AB23F8190009F10109F5E74246E2
:103C68000023434507DA07A931F81300D14921F8A1
:103C780013000133F5E7122A05D0CE4B002123F8B3
:103C880012100132F7E7CA4B012283F8362000F000
:103C98004FBCDFF82483D8F8009009F007FFA9F893
:103CA8005A00D8F8008009F001FFA8F8580000F081
:103CB8003FBC09F0F1FE84F8E00109F0EDFE84F85C
:103CC800DF0100F035BCDFF8F082D8F8009009F089
:103CD800E3FE89F80000D8F80030187802F0E8FA16
:103CE80000F026BCB44B1A681278022A4FF000097B
:103CF80098466FD1D8F800A009F0CEFE07EE900ADA
:103D0800F8EE677AB2EE048AC7EE887A0AEB890A77
:103D1800CAED087AD8F800A009F0BEFE07EE900AAE
:103D28009FEDA67AF8EE677A0AEB890AC7EE877ADA
:103D3800CAED0B7AD8F800A009F0AEFE07EE900A9B
:103D48009FED9F7AF8EE677A0AEB890AC7EE877AC1
:103D580009F10109B9F1030FCAED0E7ACAD1B9F117
:103D6800070FD8F800A01CD109F096FE07EE900ABC
:103D7800F8EE677AC7EE887ACAED117AD8F800A00B
:103D880009F08AFE07EE900AF8EE677AC7EE887A9D
:103D9800CAED127AD8F800A009F07EFE8AF84C0025
:103DA80012E009F079FECA448AF80100D8F800A0A8
:103DB80009F072FECA448AF80B00D8F800A009F08E
:103DC8006BFECA448AF8150009F10109B9F10A0F16
:103DD800C5D1ADE3D8F800A009F05EFECA448AF860
:103DE8000100D8F800A009F057FECA448AF80B0071
:103DF800D8F800A009F050FECA4409F10109B9F148
:103E08000A0F8AF81500E5D192E3DFF8AC819FED3F
:103E18006C8AD8F800A009F049FE07EE900AF8EE7F
:103E2800677A0AEB890AC7EE887ACAED087AD8F861
:103E380000A009F03BFE07EE900AF8EE677A0AEB5D
:103E4800890AC7EE887ACAED0B7AD8F800A009F07B
:103E58002DFE07EE900AF8EE677A0AEB890AC7EE9C
:103E6800887A09F10109B9F1030FCAED0E7ACCD1AC
:103E7800B9F1070FD8F800A01CD109F017FE07EE1A
:103E8800900AF8EE677AC7EE887ACAED117AD8F800
:103E980000A009F00BFE07EE900AF8EE677AC7EE6D
:103EA800887ACAED127AD8F800A009F0FFFD8AF8DE
:103EB8004C0012E009F0FAFDCA448AF80100D8F86B
:103EC80000A009F0F3FDCA448AF80B00D8F800A056
:103ED80009F0ECFDCA448AF8150009F10109B9F1A5
:103EE8000A0FC5D124E309F0D7FD132882463FF60F
:103EF800A6AEDFF8C490D9F800B009F0CDFD0023D4
:103F0800304A0C2101FB0322117A814222D10FFA97
:103F18008AF80BEB8808137888F8793009F0BCFD2B
:103F280088F87A0009F0B8FD88F87B0009F0B4FD3C
:103F3800254B264A1A6088F87C00254BD9F80000E2
:103F480018600021793003F061FC224B80F00100F9
:103F58001870EDE201331C2BD2D170E609F09CFDFC
:103F68000B2880463FF66BAE134BD3F8009009F050
:103F780093FD03283FF663AE0BFB089B8BF8CE003E
:103F880009F08AFD8BF8C90009F086FD8BF8CA0094
:103F980009F082FD8BF8CB0009F07EFD8BF8CC0090
:103FA80009F07AFD8BF8CD00C2E200BF481C002062
:103FB80058100020C8160020E81000200000C84251
:103FC80000007A44503B0108CC0A0020881D0020DC
:103FD800D00A0020020000205379092B7FF62FAE6B
:103FE800019BD3F8008009F057FD019B88F8000079
:103FF800D3F8008009F050FD88F8010009F04CFD65
:10400800019B64281B68A8BF6420187109F044FD4F
:10401800019B64281B68A8BF6420587109F03CFD07
:10402800019BFF281B68A8BFFF20987109F034FD89
:10403800019B6428D3F8008028BF642088F8070013
:1040480009F02AFD019B88F80200D3F8008009F0E6
:1040580023FD019B88F80300D3F8008009F026FDB2
:10406800D9F80030A8F80A005B790A2B40F2608280
:10407800D34BD3F8008009F00FFD88F8080057E209
:1040880009F014FD6FF4AF6283189BB2C62B98BF7A
:10409800A4F8960109F00AFDA4F8400109F006FD0C
:1040A800A4F8420109F002FDA4F8440109F0FEFC5D
:1040B800A4F8D80109F0F0FC84F8ED0109F0ECFC53
:1040C80009F0EAFC84F8EE0109F0E6FC84F88501C1
:1040D80009F0E2FC84F8920109F0DEFCB94BD3F850
:1040E800008009F0E3FC00EB80004000A8F85600CF
:1040F80020E109F0DBFCB44B23F8180008F10108B3
:10410800B8F1080FF5D113E253790F2B7FF497AD6F
:1041180009F0C2FC072880463FF691AD029BD3F810
:10412800009009F0C3FC0E2303FB08F8C144029B6E
:10413800A9F81901D3F8009009F0B8FCC144029B12
:10414800A9F81B01D3F8009009F0B0FCC144029B08
:10415800A9F81D01D3F8009009F09EFCC144029B08
:1041680089F81F01D3F8009009F096FCC144029B1E
:1041780089F82001D3F8009009F08EFCC144029B15
:1041880089F82101D3F8009009F086FCC144029B0C
:1041980089F82201D3F8009009F092FCC844C8F8C5
:1041A8002301C5E109F078FC0F2880463FF647ADAA
:1041B800C8EBC80809F070FC04EB080303F1D00849
:1041C80083F8D00009F068FC88F8010009F064FC65
:1041D80088F8020009F060FC88F8030009F05CFC2C
:1041E80088F8040009F058FC88F8050009F054FC28
:1041F80088F8060001F0AAFB9AE12B785B0700F12A
:10420800978109F053FF06F07BFD06F037FE8FE13A
:104218002B78580700F18C816C4B4FF4C8721A80C8
:1042280086E12B78590700F18381694A137843F0B6
:10423800040328E02B785A07E5D5CAE109F02CFCDD
:10424800634B1A7810B142F0020201E022F0020238
:104258001A7009F021FC5F4BDFF89881187009F09B
:104268002FFCC8F8000009F02BFCC8F8040009F07E
:104278001DFC594B188009F019FC584B584A1880F6
:10428800137843F00203137052E109F005FC8346EA
:1042980009F016FC824609F013FC814609F010FC6F
:1042A800804609F003FC09F001FC09F0F5FBBBF1BD
:1042B800000F14D14B4B1020C3F800A0C3F8049092
:1042C80006F0CCFC424A137843F001031370B8F1AE
:1042D800000F00F02D81444BC3F8008028E1BBF1AA
:1042E800100F40F02581414BC3F800A0C3F804909B
:1042F800B8F1000F02D03C4BC3F800803B483C4B60
:104308000222011D1A7007F019FB11E1A06009F0E3
:10431800D7FBA3681843A0600AE109F0C7FBA4F81B
:10432800580109F0C3FBA4F85A0109F0BFFBA4F82F
:104338005C01FDE009F0B0FB84F87A0109F0ACFB00
:1043480084F87E0109F0A8FB84F87D0109F0A4FB3C
:1043580084F87F01ECE009F0A9FBA4F8800109F0DA
:10436800A5FBA4F8820109F097FB84F8840109F001
:104378009DFBA4F88601DBE009F08EFB84F8900130
:1043880009F094FBA4F89A0109F090FBA4F89601AF
:1043980009F08CFBA4F8980109F07EFBD9F80030ED
:1043A80084F891015B79082B40F2C28009F07EFB0A
:1043B800A4F89C0109F07AFBA4F89E01B8E000BFBC
:1043C80014110020E81000207E240020DA130020B9
:1043D8001811002019110020241100202611002096
:1043E8002E1100203011002040110020381100202B
:1043F800D40A00201C11002092F805900323B9FB71
:10440800F3F9B9F1120F3FF61AACDFF8E4A2C84588
:1044180080F08E8009F040FB8AF8A00109F046FB85
:1044280040F2ED23984205DD40F6CA039842A8BF42
:10443800184601E040F2EE20A0F2EE20192308F120
:10444800010890FBF3F00AF1020A8AF89F01DEE7FF
:1044580009F022FB84F892016AE009F01DFB04EBE5
:10446800080308F10108B8F1080F83F88801F4D1AE
:104478005EE009F011FBC4F80880607109F020FBC8
:10448800A3681843A06009F007FB84F8900109F0BD
:104498000DFBA4F8580109F009FBA4F85A0109F02A
:1044A80005FBA4F85C0109F001FBA4F8800109F000
:1044B800FDFAA4F882013BE053794FF00709B3FBFA
:1044C800F9F9C9EBC9029B1A13F0FF0F7FF4B7ABD8
:1044D8005FFA89F909F1FF395FFA89F9B9F1FF0F34
:1044E80026D009F0D9FA5FFA80FA4FFA8AF003F079
:1044F80013F8804600283FF4A2AB80F800A009F02A
:10450800D5FAA8F8020009F0C7FA88F8040009F0FB
:10451800C3FA88F8050009F0BFFA88F8070009F01F
:10452800BBFA88F80600D5E75F4B012283F83720ED
:10453800002009F0FBFAFFF726BA5C4B985901F006
:104548004FF818B9322001F02CF8F6E701F0BEF95F
:1045580006F0ACFB564B574ADA60FFF722BA0C2834
:104568003DD00A2844D1544D544809F067FB2846E9
:1045780023210EF090F908B1401B20602368002B1E
:1045880059D14D482360002130220EF04EF9039B8B
:104598001B783BBB4A4B1B689B060FD5494B4249CE
:1045A8001B688A6B9A1A002A08DB474A1278042A81
:1045B80082BF03F5123303F5F8738B63434B9B6893
:1045C800002B6BD0424811B0BDEC028BBDE8F04F18
:1045D800184708F04BFCFFF7D6B90C2804D13D4822
:1045E80009F02CFB3C480DE07F2812D1FFF735B9C4
:1045F8000D28B8D07F2809D1013B2F4A37482360BE
:104608000021D15409F01AFBFFF727B92F2B3FF6E9
:1046180024A9A0F12002D2B25E2A3FF61EA913B93E
:1046280020283FF41AA95A1C2260234AD05409F0C2
:10463800FDFAFFF712B95A1EA95C202901D11346C9
:104648009DE71D4A23600021D154254B254DD3F801
:104658000090D5F800A0DFF8608050460EF029F9E8
:1046680006463246404651460EF02CF91E4A28B9F5
:1046780018F806304B445B78580703D0103595423C
:10468800E7D306E0954204D2701CEB684044984793
:1046980002E0164809F0D2FA002372E711B0BDEC27
:1046A800028BBDE8F08F00BF58100020B01B00201F
:1046B80000ED00E00400FA056418002036640108E3
:1046C800A4100020D4260020191100205C1300201B
:1046D800941000201A590108155901084159010878
:1046E800FC000020083D0108983E010825590108F2
:1046F800481C00202DE9F04764282DED028B044664
:1047080000F0BF8100F2D580322800F0558667D8C6
:10471800222800F07C8423D8032800F07E8114D856
:10472800012800F06E81022840F08786042009F0F5
:10473800FDF9432009F0CDF94C2009F0CAF94620CB
:1047480009F0C7F94C2000F03DBE042800F06F8145
:10475800052840F072861A2009F0E8F9002477E16C
:10476800282800F0E28515D8242800F0C5852628D9
:1047780040F06386CB4C062009F0D8F9B4F858010C
:1047880009F0D7F9B4F85A0109F0D3F9B4F85C0183
:1047980000F029BE2A2800F0DB852C2840F04D8641
:1047A800C04C0C2009F0C2F994F8900109F091F975
:1047B800B4F89A0109F0BDF9B4F8960109F0B9F90D
:1047C800B4F8980109F0B5F994F8910109F081F964
:1047D800B4F89C0109F0ADF9B4F89E0100F003BEED
:1047E8003D2800F0DE8224D8382800F08B8512D8C6
:1047F800342800F02E84362840F01F86AA4BA94C96
:1048080093F8ED00C0EBC000C0B209F08FF904F1D5
:10481800180500F0F6BD3A2800F093823B2840F0D6
:104828000C86012009F082F99F4B1B6D187800F067
:10483800C9BD452800F0EE8527D8402800F0C58579
:10484800422840F0FA85974C102009F06FF96079FA
:1048580009F03FF9A06809F075F994F8900109F09A
:1048680038F9B4F8580109F064F9B4F85A0109F0B4
:1048780060F9B4F85C0109F05CF9B4F8800109F05A
:1048880058F9B4F8820100F0AEBD4B2800F06685F7
:104898004D2800F07285462840F0CF850D2009F09C
:1048A80045F9002009F015F9002009F04BF900F04E
:1048B800BCBD722800F04B8455D86A2800F08B8460
:1048C8002ED8672800F0B2811BD8652800F0FE803A
:1048D800662840F0B285744C122009F027F9A08EA2
:1048E80009F027F9E08E09F024F9208F09F021F961
:1048F800608F09F01EF9A08F09F01BF9E08F00F016
:10490800F1BC682800F0FF81692840F09685674D62
:104918002878400000F0FE0009F008F90024FEE1C4
:104928006D2800F0078214D86B2800F075846C2875
:1049380040F083855E4C062009F0F8F8208809F0DD
:10494800F8F8608809F0F5F8574BB3F86C0000F0F8
:104958004ABD6F2800F04282C0F0F781702800F04D
:10496800678200F06ABD782800F06C8119D8752834
:1049780000F0418309D8732800F02284742840F09D
:104988005C854FF00008012690E3762800F05584F6
:10499800772840F05285444D287E09F0C7F8002456
:1049A800CDE3A42800F0738414D87B2800F0C982D2
:1049B800A02840F042850C2009F0B8F83D4B186853
:1049C80009F0C0F83C4B186809F0BCF83B4B186874
:1049D80000F02FBDF12800F07081FE2800F07E84E1
:1049E800F02840F02A85304C042009F09FF8236D08
:1049F800B3F85A0009F09DF8236DB3F8580000F099
:104A0800F2BC032009F092F8002009F062F8204671
:104A180009F05FF80D2000F0D5BC09F087F80120F7
:104A280009F057F80A2009F054F800F02EBC0620C7
:104A380009F07CF8412009F04CF8462009F049F8C3
:104A4800462009F046F8332009F043F800F052BC3C
:104A58001B4B185D013409F03CF80B2CF8D10024ED
:104A6800184B185D013409F034F8082CF8D10024EB
:104A7800154B185D013409F02CF8072CF8D100F01B
:104A8800DABC072009F052F8E72009F022F8054BB4
:104A9800587909F01EF8002009F01BF8042000F0EE
:104AA800C8BC00BF481C00209810002064230020C8
:104AB8006E1B0020ACF7FF1FB0F7FF1FB4F7FF1FF6
:104AC800745501088055010855550108BA4C0B204A
:104AD80009F02CF8208809F02CF86268B74B9A4244
:104AE8000CBF2089608980B209F023F8E368C3F31A
:104AF800C000C3F38002800040EA4200C3F34002D2
:104B08001043C3F3401240EAC20003F010031843F5
:104B180009F00FF8228A6369247E02F0080103F481
:104B2800475949EA010903F4804149EA010903F4B4
:104B3800004149EA010903F4803149EA010903F413
:104B4800003149EA010903F4802149EA010903F423
:104B5800002149EA010903F4801149EA010903F037
:104B6800007349EA0303DFF8709299F8009012F095
:104B7800010FC9F3800914BF4FF002084FF0000875
:104B880043EA090312F0020F43EA080314BF4FF087
:104B9800040C4FF0000C12F0040F43EA0C0C14BF85
:104BA8004FF0100E4FF0000E12F0400F14BF2027E8
:104BB80000274CEA0E0E12F0100F14BF4FF40076C7
:104BC80000264EEA070712F0200F14BF4FF4806545
:104BD80000253E4312F4807F14BF4FF4006000208C
:104BE800354312F4007F14BF4FF40011002128430D
:104BF80012F4806F41EA000114BF4FF08063002374
:104C0800002019430346A3420AD26D4A9D5C012243
:104C180002FA05F50D421CBF9A4010430133F2E732
:104C280008F090FF674B93F8E406CBE3102008F0F8
:104C38007DFF0024644B185D013408F04AFF102CF6
:104C4800F8D1F8E3702008F071FF00265A4D0E24C1
:104C58002B6D744323440136B3F8190108F069FF3A
:104C68002B6D2344B3F81B0108F063FF2B6D23441D
:104C7800B3F81D0108F05DFF2B6D234493F81F0165
:104C880008F027FF2B6D234493F8200108F021FF3B
:104C98002B6D234493F8210108F01BFF2B6D23444F
:104CA80093F8220108F015FF2B6D1C44D4F823015A
:104CB80008F048FF082EC9D1BDE37020414C08F028
:104CC80035FF04F1700594F8D00008F002FF94F85D
:104CD800D10008F0FEFE94F8D20008F0FAFE94F82D
:104CE800D30008F0F6FE94F8D40008F0F2FE94F829
:104CF800D50008F0EEFE073494F8CF0008F0E9FE7E
:104D0800AC42E0D197E3102008F010FF00242F4BAD
:104D1800185D013408F0DDFE102CF8D18BE32B78F8
:104D28009C4280F088832A4B33F8140008F001FF76
:104D38000134F4E7062008F0F9FE002008F002FF2D
:104D4800D8E2042008F0F2FE72E3072008F0EEFE35
:104D5800204B194C1888FF28A8BFFF20C0B208F0C4
:104D6800B8FE206F4FF6FF75A842A8BF284620EA74
:104D7800E07080B208F0DDFEB4F8740008F0D9FEE7
:104D8800104BA06F93F885313BB10A235843A842D2
:104D9800A8BF284620EAE07001E000F30F0080B2C7
:104DA80021E3084C022008F0C1FE94F8E00108F065
:104DB80090FE94F8DF0105E39810002000540040AD
:104DC800B1100020481C0020D8100020EC10002052
:104DD8007826002058180020F3260020C24C0B200B
:104DE80008F0A4FEE36F187808F073FEE36F5878B4
:104DF80008F06FFE00262546EB6FBB4C33440136A6
:104E0800187908F066FE032EF6D1E36FD87908F01A
:104E180060FEE36F987808F05CFEE36FD87808F0DE
:104E280058FEE36F588908F084FEE36F187AC9E2E8
:104E3800AD4C1E2008F07AFE236D1B78022B4FF034
:104E480000056BD1236D03EB850393ED080AB2EEE1
:104E5800048A20EE080A0DF0F7FE80F30800C0B2BD
:104E680008F037FE236DDFEDA17A03EB850393EDA0
:104E78000B0A20EE270A0DF0E7FE80F30800C0B207
:104E880008F027FE236DDFED9A7A03EB850393ED97
:104E98000E0A20EE270A0DF0D7FE80F30800C0B2F4
:104EA800013508F016FE032DCCD1072D236D23D133
:104EB80093ED110A20EE080A0DF0C6FE80F30800F3
:104EC800C0B208F006FE236D93ED120A20EE080A20
:104ED8000DF0BAFE80F30800C0B208F0FAFD236DA9
:104EE80093F84C3000EE103AB8EE400A0DF0ACFEE4
:104EF80080F30800C0B20BE02B44587808F0E9FDB5
:104F0800236D2B44D87A08F0E4FD236D2B44587D9B
:104F1800013508F0DEFD0A2DC7D18CE2236D2B4444
:104F2800587808F0D6FD236D2B44D87A08F0D1FDC7
:104F3800236D2B440135587D08F0CBFD0A2DEDD1AA
:104F480079E23C2008F0F2FD0024674D9FED688A65
:104F58002B6D03EB840393ED080A20EE080A0DF08D
:104F680073FE80B208F0E5FD2B6D03EB840393ED2F
:104F78000B0A20EE080A0DF067FE80B208F0D9FD92
:104F88002B6D03EB840393ED0E0A20EE080A0DF057
:104F98005BFE013480B208F0CCFD032CD5D1072C80
:104FA8002B6D16D193ED110A20EE080A0DF04CFE78
:104FB80080B208F0BEFD2B6D93ED120A20EE080AB0
:104FC8000DF042FE80B208F0B4FD2B6D93F84C0052
:104FD8000BE02344587808F0ACFD2B6D2344D87AB5
:104FE80008F0A7FD2B6D2344587D013408F0A1FD7E
:104FF8000A2CD4D11FE22F2008F098FD3D4C14F85C
:10500800010F002800F0178208F063FDF7E7502031
:1050180008F08CFD0025344B1C6D374B04EB8504E0
:105028000C2194F8792001FB0233013593F83800FC
:1050380008F04FFD94F87A0008F04BFD94F87B00D7
:1050480008F047FD94F87C0008F043FD142DE2D1E8
:10505800F1E1482008F06AFD0025234B1C6D06236A
:1050680003FB0544013594F8CE0008F032FD94F8AE
:10507800C90008F02EFD94F8CA0008F02AFD94F83B
:10508800CB0008F026FD94F8CC0008F022FD94F837
:10509800CD0008F01EFD0C2DDFD1CCE1002E00F074
:1050A800CA815FFA88F008F041FD002600270E4B00
:1050B8001A7E9742F2DA19330024FA5C0E4D0C235B
:1050C80005F130016343595C914207D12B44586B79
:1050D8000DF0EFFB82462EB9B1460FE001341C2CCF
:1050E800ECD118E0804416E0981000200000C84277
:1050F80000007A441F3B0108203B0108D1450ADA29
:105108000C2303FB04535B6B13F8090008F0E1FC64
:1051180009F10109F2E70137C9E701311C290DD06E
:10512800D4480C2200F1300702FB01F3DA5DB242E9
:10513800F3D1034493F8380008F0CBFC01342B7EFC
:105148009C4280F07881CC4B0021E65CE8E7CB4CB0
:10515800162008F0EBFCB4F8960108F0EAFCB4F865
:10516800400108F0E6FCB4F8420108F0E2FCB4F8AB
:10517800440108F0DEFCB4F8D80108F0DAFC94F831
:10518800ED0108F0A6FC002008F0A3FC94F8EE015D
:1051980008F09FFC94F8850108F09BFC94F89201B4
:1051A80008F097FC002008F094FCB54B1B6D0A2012
:1051B800B3F9563093FBF0F080B208F0BAFCA5E0E2
:1051C800082008F0B3FC0124E0B2013408F081FCA7
:1051D800092CF9D12FE1AA4C102008F0A7FC94F86B
:1051E800800000F0020008F074FC94F8810008F0D8
:1051F80070FCD4F8840008F0A5FCD4F8880008F006
:10520800A1FCB4F88C0008F094FCB4F88E0008F007
:1052180090FCB4F89000E6E0994C052008F086FC74
:10522800B4F8920008F085FCB4F8940008F081FC0A
:1052380094F8960000F00100C4E008F02DFC074641
:10524800122008F073FC8E4C27B9D4F89860D4F873
:105258009C5007E0102F13BF0025D4F8A060D4F8A5
:10526800A4502E46384608F034FC304608F06AFC54
:10527800284608F067FCD4F8A80008F063FC002072
:1052880008F057FC002008F054FC00209AE07C4D00
:1052980095F8AC0080000130C0B208F047FC95F8E2
:1052A800AC0008F016FC00242E4696F8AC309C4260
:1052B80080F0C180734D285D08F00BFC05F11003E8
:1052C800185D08F006FC05F120033035185D08F07C
:1052D80000FC285D08F0FDFB0134E6E7082008F033
:1052E80025FC002008F025FC002008F022FC002006
:1052F80008F01FFC002076E0042008F017FC5F4B44
:10530800986896E0042008F011FC5C4C94F87A0147
:1053180008F0DFFB94F87E0108F0DBFB94F87D01D0
:1053280008F0D7FB94F87F014CE0544C072008F0B4
:10533800FDFBB4F8800108F0FCFBB4F8820108F02A
:10534800F8FB94F8840108F0C4FBB4F886014AE03D
:10535800012008F0EBFB494B587933E0474C042017
:1053680008F0E4FB94F8D60108F0B3FB94F8D701F1
:1053780008F0AFFBB4F8D80135E0434C434D207832
:1053880000EB4000C0B208F0D1FB002623789E4213
:1053980005F102054FD215F8020C08F09AFB15F832
:1053A800010C00EB800000EB800000F2EE2080B2E0
:1053B80008F0BFFB0136E9E7012008F0B7FB2F4BE7
:1053C80093F8920108F085FB35E0082008F0AEFB61
:1053D80000242A4B2344013493F8880108F079FB10
:1053E800082CF6D127E008F0A4FB24E092F90C1071
:1053F800994224D092F918209A4220D00834AC421D
:1054080019D0234A94F8F40192F9001043B2994252
:10541800ECD114E0132008F089FB00241D4B185D23
:10542800013408F056FB0B2CF8D1002008F08AFB59
:10543800002008F087FB012018E0002016E008F0A3
:1054480048FBB4F8F60108F074FB94F8F80108F08A
:1054580040FB94F8F90108F03CFB94F8FB0108F0D4
:1054680038FB94F8FA0108F034FBC7E7BDEC028B6F
:10547800BDE8F087203B0108B1100020481C00203F
:10548800981000204511002064230020E81D00200A
:105498007023002074550108034B4FF4806208B153
:1054A8009A6170471A85704700040048034B4FF40F
:1054B800806208B11A8570479A61704700040048F5
:1054C800D0ED024A91ED016A90ED015A91ED027A10
:1054D800D0ED005AD1ED007A66EE646AE5EE076A0F
:1054E80027EE657AC2ED006AA4EEA77A67EEC57A60
:1054F80082ED017AE5EE867AC2ED027A7047D0ED48
:10550800017A91ED017AD1ED026A91ED006A37EEE8
:10551800877AD0ED027A77EEA67AD0ED006A82ED2E
:10552800017A76EE866AC2ED027AC2ED006A7047A9
:1055380090ED017AD0ED027AD0ED006A20EE077A7C
:1055480060EE277A26EE800A81ED017A81ED000A65
:10555800C1ED027A704710B5094A0A4B11689B6879
:1055680000BF12689142F7D1074A14684FF47A7065
:1055780000FB04F2D31AB3FBF4F300FB013010BDB7
:10558800181B002010E000E08811002038B5044600
:10559800FFF7E1FF0546FFF7DEFF401BA042FAD305
:1055A80038BD10B504462CB14FF47A70FFF7EEFF02
:1055B800013CF8E710BD024A1368013313607047D5
:1055C800181B0020024B5B6803B11847704700BFE7
:1055D80088110020014B1B68184700BFD8260020FF
:1055E80003681B6918470368DB68184703689B68EA
:1055F800184703685B68184703681B6818472DE954
:10560800F84FB0F90230934218BF00232DED048BF8
:1056180018BF0370057804460E469146002D40F0E9
:10562800978007EE902ADFED7D8AF8EEE77AB6EEEE
:10563800009A67EEA88ADFED7A7A68EEA78AA04614
:1056480068EE898A2746B0EE680A05F09FFAB0EE40
:10565800408AB0EE680A05F0F9FA88EE000A40F2CE
:10566800DC5363651023A4F852301823A4F8503093
:10567800DFED6C6A60EE266AB7EE006AB0EE667A15
:10568800A0EE007AD0EE006A37EE067A76EE866AE9
:10569800C6EE077A84ED046A27EE807AB0EE498A6E
:1056A80027EE007A77EE075A84ED017AC4ED025AA4
:1056B80070EE005A84ED037AB8EE007AA5EE807A8F
:1056C80027EE877A67EEA67A84ED057AC4ED067A26
:1056D800DFED557A98ED047A27EE277AF0EE678A9F
:1056E800B5EEC07AF1EE10FA4CBF77EE487A77EE55
:1056F800087A013517EE900A0AF0CAF8D8ED017A4F
:1057080067EEA87AC7E90E01F5EEC07AF1EE10FA55
:105718004CBF77EEC87A77EE887A08F1040817EE5E
:10572800900A0AF0B5F8032DC7E9080107F1080740
:10573800CED1A6F2DC531B042367E3676367C4F882
:105748008030A367C4F884300123A4F80290237042
:10575800D4F85490B4F95280636A276A206FE26FD4
:10576800D4F840C0D4F88010C4F88020C9EB0606ED
:1057780006FA08F64FEAE67B734307FB0B33266706
:10578800A7FB06671F44636C656F60674FEAE27B9F
:1057980053430CFB0B3EACFB02237344B61A67EB76
:1057A8000307E36AA26AC4F884104FEAE07B434324
:1057B80002FB0B3EA2FB00237344B6185F41E36C67
:1057C800A06CB4F95020A5674FEAE17B4B4300FB7E
:1057D8000B33A0FB01011944636B361A206B4FEAA7
:1057E800E57B05FB03F300FB0B3367EB0107A0FB2D
:1057F800050119448019794109F018FE08F1FF32B2
:1058080001239340E067C01841EBE371424609F079
:105818000DFEBDEC048B4844BDE8F88F6F12833A47
:10582800DB0F4940F404B53F0000804B2DE9F843F5
:105838000024234B93F83860E0B2B0420CD203EB5B
:105848008003204A9B6832F810101BB10B2801D83E
:10585800DB6898470134ECE71B4B1B685B032CD5CE
:1058680000242346E2B2B24227D2DFF8549009F16D
:1058780008074FEA840857F8242055689D4214D039
:10588800284606F017FAEFF31283502282F31288A3
:1058980028216A6A01FB0090013202666A6942F0B7
:1058A80001026A61DBB283F3118857F808301B687C
:1058B80000221A6001342B46D4E7BDE8F88300BF04
:1058C80088110020EC100020781B002008B50E4B32
:1058D8001B6813F4805F0D4B14BFD3F85421D3F821
:1058E800582193F8381092880023D8B2884204D2FD
:1058F800074820F813200133F7E7FFF797FF322016
:10590800BDE808404DE600BF781B00208811002044
:10591800EC1000200A4B1A680A4B30B502F480528A
:10592800D3F85441D3F8585100230AB1A18800E0B4
:10593800A988054820F8131001330C2BF5D130BD88
:10594800781B0020881100207E24002070B5124D9D
:105958000024214605F25D10702285F85C410CF0A8
:1059680064FF2146D5F8D0310B4A0B4493F9020065
:1059780080B102F25D141E680E5108199C8884805B
:105988009B79837192F85C3107310133702982F871
:105998005C31E7D170BD00BF88110020094B1A683F
:1059A8000E2303FB0020437AFF2B07D0064A127808
:1059B8009A4203D9054A32F8130000E0808800B201
:1059C800704700BF98180020642300207826002024
:1059D8002DE9F04F2DED0A8B97B011F0FD08064622
:1059E8000191A94C06D0A94B1B689A0700F1B18018
:1059F80000F03DBCD4F8D831A548DFF89492984718
:105A08000028F0D0A34F94F8E8214846494603F00F
:105A1800FDFD3B8804F50E72002B70D0D4F8EC31F4
:105A28001B7808EE103A04F5F87A04F5FE75B7F815
:105A380000B039F91800BBF57A7F02BF0023CAF815
:105A480000302B61DAF800300344CAF800302B69C3
:105A580007EE900A0133012B4FEA4801F8EEE77A86
:105A68002B6106D10023C5ED017AC5ED007AAB6044
:105A78001BE0D5ED006A07EE103A37EEE66AB8EE9D
:105A8800C77A86EE077A36EE877AD5ED026A85ED13
:105A9800017A77EEC77A85ED007AE6EE276AF0EEAE
:105AA800667AC5ED036AC5ED026A0023BBF1010FF2
:105AB80029F8013053522DD12B690392012BC3BF12
:105AC80003F1FF3300EE103AD5ED037A9FED720A29
:105AD8000291C4BFB8EEC00A87EE800A0DF08CF9B7
:105AE8000299039A18EE103A5BB1F8EEC87AB4EE50
:105AF800E70AF1EE10FA04DD4FF47A733B800023D5
:105B08001CE0DAF800304FF47A7003F5FA7393FB6F
:105B1800F0F3535208F10108B8F1030F0AF1040A2F
:105B280005F1140583D1BBF1010F04D15846029247
:105B380001F0D8FE029A3B88013BDFE739F81310E1
:105B480032F81300091A29F813100133032BF5D181
:105B580049E7019B002B00F08A8394F83E724A4D76
:105B68006FB1012F40F07B8305F52270D5EDA06A57
:105B780095EDA17A05F52573002180460FE1FFF721
:105B8800EAFCD5F848329FED457AC5F84002C31AB9
:105B980007EE903AF8EE677A414BC5F8480267EE8F
:105BA800877A5B68C5ED917A05F51370984705F516
:105BB8001378002800F0ED803A4B40461A784146A9
:105BC80003F024FDB5F85232002B41D0D5F8541219
:105BD8003B46B4F8522238F913702B4DB2F5C87F02
:105BE800314A04BF002042F823004FEA830E52F8DE
:105BF8000E00384442F80E00002028F8130021F85F
:105C080013000133032BE4D1B5F85232012B1AD11A
:105C1800D5F858324FF4C87703F1C80292FBF7F26F
:105C28000A80D5F85C22C83292FBF7F24A80D5F890
:105C38006032C83393FBF7F3A3F580738B80308011
:105C4800708005F0B7FAB4F85232013BA4F852322A
:105C5800164B1B685B0740F18880B4F864220A4B36
:105C6800322A25D1D3F854221188A3F86612518814
:105C78009288A3F86A223288A3F86C227288A3F863
:105C88006812A3F86E2215E088110020A4100020E5
:105C9800D2100020EC26002000000000BD37863519
:105CA800A8240020F4260020E0130020781B002000
:105CB800002A3BD0D4F854020023B4F8642238F9FF
:105CC80013E0C54D322AC54A04BF002142F823100B
:105CD8009F00D1597144D151002228F8132020F88F
:105CE80013200133032B1146E7D1B5F86432012B99
:105CF80017D10C2085F87C2285F87D3201F0F2FD61
:105D0800D5F85432B5F866221A80B5F868225A8058
:105D1800B5F86A229A80B5F86C323380B5F86E32DD
:105D28007380B4F86432013BA4F8643294F87E328C
:105D3800A94AD3B1D2F85402D2F8703200213225E0
:105D480082F87E1293FBF5F30380D2F8743293FB4A
:105D5800F5F34380D2F8783293FBF5F3A3F580731B
:105D680083803180718005F025FAD4F85422B4F884
:105D78004C3211885B1AA4F84C325188B4F84E3270
:105D88005B1AA4F84E329288B4F850329B1AA4F8E1
:105D9800503294F83E32013384F83E32DDE68E4DBF
:105DA8008F4F05F5137232F8112027F8112012B21F
:105DB80007EE902A8B4AF8EEE77A32F9112067EE5F
:105DC800A67A0131E0EC017A07EE902AF8EEE77A3C
:105DD800032967EE877AE3EC017AE0D105F52570AF
:105DE80005F528710246FFF78AFB05F5257005F5CC
:105DF8002B7104AAFFF783FB04A895ED910ADFF83D
:105E0800D8A10146FFF794FBDDED054ADDED047AE4
:105E18009DED065A95EDB14AD5EDB03A95EDAE3AFD
:105E2800B6EE007A64EE874A67EE875A64EEA47A83
:105E380025EE075AE5EEA57A07A80146B7EE008ACF
:105E4800E5EE057A0AAA0DAFF0EE482AE7EEC72A72
:105E58000AF5357965EE846AD5EDAF7AE2EEA36A84
:105E680025EE236AE4EE836A23EEE57AB1EE452A4D
:105E7800E2EE276AA2EEA76AA4EEA77A67EEE57AB1
:105E8800F1EE641AE2EE837AA1EE846AA2EE847AD5
:105E9800E1EEA37AA5EE836AA5EE037AE2EE047A30
:105EA80085EDAF6AC5EDAE7AB1EE466AC5EDB06A6A
:105EB80085EDB17AF1EE666AB1EE477A8DED097A31
:105EC8008DED076ACDED086AFFF719FB95EDAE0A6F
:105ED800454810A9FFF72CFB07A8434913AAFFF769
:105EE800EFFA13A810A93A46FFF709FB0AA83946A2
:105EF80013AAFFF7E5FA3A463B4813A9FFF7FFFA5A
:105F08003A4BD5EDB27A9DED0F7A1A78B4EEE77A6E
:105F1800F1EE10FACCBF42F0080222F008021A7023
:105F2800D4F8CC321B78F0EE489A0AF539753BB3B1
:105F3800DAEDB48A4846B0EE680A10A9FFF7F8FA15
:105F48009AEDB88A0AF52270B0EE480A13A9FFF74D
:105F5800EFFA4A4610A813A9FFF7D1FA2846B0EE7F
:105F6800680A10A9FFF7E4FA384613A9B0EE480A00
:105F7800FFF7DEFA10A813A92A46FFF7C0FA07E0D0
:105F880098E8070089E8070097E8070085E8070010
:105F9800D4EDA37AD4EDA26A94EDA47A0E4D67EEFF
:105FA800A77A0023E6EEA67AE7EE077A9FED107A45
:105FB800F4EEC77AF1EE10FA06DC9FED0E7AF4EEF5
:105FC800C77AF1EE10FA19D5C4F8AC32C4F8B03279
:105FD800C4F8B43225E000BF88110020F81300206F
:105FE800CC100020D2100020B43C01081811002069
:105FF800B81E8D3F3D0A673F6F12833A05F535702D
:1060080005F5397105F52B72FFF75AFAD5ED917A36
:106018001FED070A05F52B7080EE270A0146FFF7EA
:1060280087FAB4F8F032984D01339BB2B3F57A7F12
:10603800A4F8F0322ED195EDAF0AD5EDAE6A95ED04
:10604800B07AD5EDB17A20EE000AA6EEA60AA7EE40
:10605800070AA7EEA70A0CF0CFFE89EE800A0023F4
:10606800A5F8F032D5EDAF6A95EDB07AD5EDB17AF5
:1060780095EDAE6A60EE266A20EE077A60EE277A22
:1060880026EE000AC5EDAF6A85EDAE0A85EDB07A59
:10609800C5EDB17AD4EDAF8A94EDB1AA94EDAEBA5C
:1060A800D4EDB0AA9FED799A68EECA7AB7EE007A75
:1060B800EBEE2A7A77EEA77AF4EEE97AF1EE10FAA7
:1060C8000EDCFFEE006AF4EEE67AF1EE10FA24D464
:1060D800F4EE477AF1EE10FAC8BFF0EE477A01E025
:1060E800F0EE477A17EE900A09F012FB41EC100B1C
:1060F8000CF020FE51EC100B09F05EFB08EE100AC4
:10610800B5EEC08AF1EE10FA09DD78EE497AF5EEBF
:10611800C07AF1EE10FA10DC23E09FED5D8AF1EE13
:10612800487A77EEC97AF5EEC07AF1EE10FAB5EE54
:10613800C08A13DDF1EE10FA06DD38EE499ADFED7C
:10614800557AB4EEE79A03E09FED527AF4EEC77AF7
:10615800F1EE10FA4CBF0123002312E0F1EE10FA21
:1061680006DD38EE499ADFED4C7AB4EEE79A03E0A3
:106178009FED497AF4EEC77AF1EE10FACCBF01230D
:10618800002353B1B0EE4A0AF0EE4B0A04F08CFC3F
:106198009FED42CA70EE008A41E02AEE8A0A6AEE52
:1061A800AABAABEE280AB0EE6B7A30EE000AA8EE77
:1061B800A87AB5EE400AF0EE007AF0EE690AF1EE40
:1061C80010FAE7EE670AB0EE679A04D1F5EE400AD6
:1061D800F1EE10FA04D004F067FCB0EE40CA01E01A
:1061E8009FED2ECA28EEAA0AEAEE0ABAABEE0A0A10
:1061F800F0EE690A30EE000AEBEEC90AB5EE400A85
:10620800F1EE10FA04D1F5EE400AF1EE10FA04D0DE
:1062180004F04AFCF0EE408A01E0DFED208A9FEDB1
:10622800209A204D2CEE090A0CF00EFD28EE090AE2
:1062380028800CF009FDDFED1C7A1C4A688068EEA6
:10624800E78AFDEEE88ACDED018ABDF8043013F443
:10625800004F18BF03F5B4731380002300E0012337
:10626800002284F83E22002B7FF477AC06E000235E
:10627800A4F84C32A4F84E32A4F8503217B0BDEC52
:106288000A8BBDE8F08F00BF88110020DB0FC93FE3
:10629800DB0FC9BF35FA0E3C35FA0EBC0000000012
:1062A8004D3D0F446E1B0020E12E65420411002075
:1062B80001380A4B042804D8DFE800F00507090B69
:1062C8000D00074A08E0074A06E0074A04E0074AC3
:1062D80002E0074A00E0074A1A607047F000002011
:1062E80089820008F57900080DEF0008A17F0008F1
:1062F800617C000871850008284B294A1B681268D0
:1063080010B51A60274A1168596051689268DA60B6
:10631800254A996011681961516892689A61234AFF
:1063280059611168D961516892685A62204A1962A4
:1063380011881985518859859188D288DA851D4A2E
:106348009985118819865188598692889A861A4A99
:106358001188D986518819871946928821F83A2FC9
:10636800164A10780022824206DA154C34F8124098
:1063780021F8024F0132F6E7124A1288A3F8642086
:10638800114A1288A3F86620104A1288A3F86820D8
:106398000F4A5289A3F85E2010BD00BFEC240020EC
:1063A800D426002064150020701500207C150020DC
:1063B80014150020D2100020CC100020C01100209D
:1063C800EC100020CC1700207C1000200C110020BD
:1063D800D810002030B50028104C114AB8BF4042F0
:1063E8003C2590FBF2F304FB030068430D4D90FB42
:1063F800F2F22D682D7B25B903EB830303EB8303AE
:1064080001E0C3EB031302EB83030B8004FB0202DE
:106418004FF47A7392FBF3F24A8030BD806967FFCC
:10642800809698008C0700202DE9F8430E4B93E8DE
:10643800800305460E460024B44213DA7B1933F96B
:10644800140008EB050333F9142009EB050333F9AD
:1064580014301344022293FBF2F3C01A08F085F9B2
:106468000134E9E7BDE8F883EC24002070B5472043
:1064780008F0CAF8174B1B681B0307D5164B174AB9
:106488005B6810681B68C01A08F060F9144E154C58
:10649800154D307808F05AF923682868C01A08F0B2
:1064A80064F963686868C01A08F05FF90F4B1888C8
:1064B80008F04CF90E4B188808F048F90D4B18886D
:1064C80008F044F9337823742B68A3606B68E360A1
:1064D80070BD00BF40260020EC240020D4260020F8
:1064E80019110020D82400201C110020241100209C
:1064F80026110020281100207FB5264C264E274D56
:106508002749284A284B20B128480088B0F5805FE1
:1065180031D23088ADF8040028781E4D91F820104B
:1065280012788DF806008DF807108DF808201B7872
:106538008DF8093001A8294606220CF05BF930B322
:106548000198BDF808302860AB80532008F05CF84B
:10655800208808F0FBF8A07808F0F8F8E3780193B1
:106568002379029301A86379039308F055F80F4B38
:1065780000221A800BE03088208091F820102878BB
:1065880012781B78A070E17022716371DDE704B0A6
:1065980070BD00BF7C140020A81000201811002036
:1065A800A4260020200A0020860A00206026002059
:1065B800A0F17D03012B70B504460D460A4E05D89F
:1065C80030687D21FFF718F884F0200430682146F0
:1065D800FFF712F835B12B881C4404EB142404F09F
:1065E800FF042C8070BD00BF2808002010B50A4C9D
:1065F8005E280146A06805D15D21FEF7FDFFA06871
:106608003E2105E05D2903D1FEF7F6FFA0683D2194
:10661800BDE81040FEF7F0BF7C1400200A4A13883A
:1066280001331380094A136801331360084A138839
:1066380001339BB2202B01BF00231380054A138826
:1066480008BF0133138070476026002048260020C9
:106658004C2600204E26002038B53A4B1B78083BC4
:10666800012B05460C466BD8452007F0CDFF284680
:1066780007F0CAFF0C2D23D004D80A2D0AD014D84D
:1066880035B138BD0E2D4BD02ED3FF2D50D038BD8F
:10669800206849E0207807F0B7FF62796378002A1C
:1066A80014BF80200020184300E0207807F0ACFFDA
:1066B800A07807F0A9FFE07807F0A6FF20793BE073
:1066C800B4F9000008F038F8A07807F09DFFE078EA
:1066D80007F09AFFB4F9040008F02EF8B4F90600A0
:1066E800BDE8384008F028B8637820788BB180F08E
:1066F800800007F089FFA468E0B207F085FFC4F3C3
:10670800072007F081FFC4F3074007F07DFF200E44
:1067180012E007F079FF6068BDE8384008F025B856
:10672800206808F013F86068BDE8384008F00EB833
:10673800054807F047FF0020BDE8384007F064BF70
:1067480038BD00BFD2240020625A01082DE9F04F5D
:10675800B54BB64F1A888BB00193002A40F096804B
:10676800B7F80A07B24D42F20103C11A484248413C
:10677800FFF7C2FEFFF7C0FD2C68492007F044FF71
:10678800AC4B2646186807F0E1FF56F8040B07F0F3
:10679800DDFF304606F066FA04F1100006F062FAF2
:1067A80004F11C094FF01008A34E0123326803FAC4
:1067B80008F3134203D0D9F8000007F0D6FF08F118
:1067C8000108B8F1130F09F10409EDD104F128000B
:1067D80006F038FAB7F84031B4F92E00C01A07F0BD
:1067E800B5FF3368DA0408D5944BB4F864001B8805
:1067F800181AC0F30D0007F0A9FF33689B0403D5EE
:10680800B4F8660007F0A2FF3368180403D5B4F89B
:10681800680007F09BFF04F13000A04606F012FA6A
:1068280004F1360006F00EFAB7F8403138F93C0F9B
:10683800C01A07F08BFF0127814B1B789F4208DAAB
:1068480038F9020FB4F93C30C01A07F08EFF01374F
:10685800F2E73368990505D5B4F95E00A0F2DC507B
:1068680007F083FF2A6877486A60AA60121A9110B5
:10687800754A4A43531C032293FBF2F202EB42028D
:106888009A1A6C2303FB02032B60ABE16F4B704A2F
:106898001B6811688B4206D00AA9002041F8203DE8
:1068A8001360FFF7D9FE019B97F80A171B8897F822
:1068B8000B070B44013BB3FBF0F200FB12338B4296
:1068C80080F05B815A4D0120FFF716FEFFF714FD9B
:1068D80050202F686E6807F097FEAA682B6810682A
:1068E8001B686A6803441068A3EB400007F03DFF8B
:1068F80072687B689B1A0293B268BB689B1A039301
:10690800F268FB6802A89B1A049306F0ABF9326997
:106918003B699B1A029372697B699B1A0393BB6953
:10692800B26902A89B1A049307F076FE07F11C0BC4
:1069380006F11C081024404901220B68A2401A42A3
:106948008A4606D0DBF80000D8F80030C01A07F0F5
:106958000CFF0134132C0BF1040B08F10408EAD1E5
:1069680007F1260006F12601002331F9024F30F91C
:10697800022F121B02AC44F823200133042BF4D15C
:1069880003214FF000094FEA89035FFA83F902AB4C
:1069980053F821206AB102F108000F2802D849F003
:1069A800010906E08032FF2A94BF49F0020949F044
:1069B800030911F1FF31E6D2484607F025FE00240D
:1069C8000DF1080BA04609F00302022A16D0032A8B
:1069D8001DD0012A4FD1B8F1000F05D1DBF80040D6
:1069E8002401E4B2904646E0DBF8000000F00F0016
:1069F800204307F009FE4FF000083CE0B8F1000F13
:106A08000CD0DBF80000C0F3031020432DE0B8F1F0
:106A1800000F1FD19BF8010007F0F6FD9BF800005E
:106A280007F0F2FD27E000BF4C260020481C00209C
:106A3800EC24002048260020402600203C26002088
:106A4800C0110020F824002013DA4B6854260020D7
:106A580050260020DBF80000C0F30330204307F085
:106A6800D3FDDBF80000C0F3071007F0CDFDDBF81D
:106A780000402401E4B20BF1040B06AB9B454FEA3E
:106A88009909A0D1B8F1010F02D1204607F0BCFD49
:106A9800DAF8003013F480541FBFB7F86420B6F852
:106AA8006410521A029218BF01249A040AD50AAA3D
:106AB80002EB8401B6F86600B7F86620121A41F8AE
:106AC800202C013418040BD50AAB03EB8402B6F86A
:106AD8006810B7F868305B1A42F8203C013400E0CF
:106AE800FCB1012C03D1029807F03FFE19E0631EA8
:106AF800002002AA400052F82320C0B20AB140F098
:106B08000100013BF5D507F07FFD4FF0000802AB0F
:106B180053F8280008B107F028FE08F10108A0453D
:106B2800F5DB30200321FFF77FFC36200321FFF738
:106B38007BFC2F4B3C201978FFF776FCDAF8003005
:106B4800990506D5B7F95E00B6F95E30C01A07F0A8
:106B58000CFE2A6827486B686A60121A9110264A48
:106B6800AB604A43531C032293FBF2F202EB42024E
:106B78009A1A6C2303FB02032B60204B1B681A062E
:106B880030D51F4C1F4D22682B689A420BD1626882
:106B98006B689A4207D1019B1B88102B11D11A4BA5
:106BA8001B885B060DD1482007F02EFD206807F0F2
:106BB800DCFD606807F0D9FD23682B6063686B60B3
:106BC8000EE0124A0F4B11782A7C914208D1104AE4
:106BD80099681068884203D15268DB689A4201D0EC
:106BE800FFF744FC07F0E0FC0BB0BDE8F08F00BFF6
:106BF800C0110020F824002013DA4B68781B00200D
:106C080030110020D82400204E2600201911002021
:106C18001C1100202DE9F84F0C9E3A4CC2EB030BD7
:106C28000B9BF61A6368002914BF4FF0060A4FF051
:106C3800040A01330546904613D1236853455ED2B2
:106C4800314A324852F82320032B98BF294607F0CF
:106C5800C9FC6368013363602D4B002205461A7333
:106C680013E0002511E02B4A1278954240DA0B9B7D
:106C7800E3B109FB06F2995C01228A4026490968BA
:106C88000A4213D1636801336360D4F804900A9B05
:106C98001C4F9945E7DB2BD10A2007F0B5FC3B6870
:106CA80001333B604FF0FF337B6021E0184A117BD2
:106CB80021B12C2007F0A8FC013501E00121117356
:106CC800226809FB0BF308EB030752B958F80300D5
:106CD80007F078FC97F904104B1C0544D2D00F48F4
:106CE80002E03A440E48117907F07CFC0544C9E7F4
:106CF800206850452CBF00200120BDE8F88F0020F7
:106D0800BDE8F88F58260020C03C01086D5A0108DC
:106D18007C140020F9000020402600207C5A01083D
:106D28009063010830B585B004AC002524F8025DF5
:106D38000091ADF8060021461020FFF739FC9DF8B8
:106D480006002146FFF734FC9DF807002146FFF7AF
:106D58002FFC9DF800002146FFF72AFC9DF8010052
:106D68002146FFF725FC9DF802002146FFF720FC8D
:106D78009DF803002146FFF71BFC9DF80E00C04359
:106D8800C0B22946FFF714FC05B030BD10B5054C5C
:106D98002068FEF72EFC18B12068FEF727FCF6E7FE
:106DA80010BD00BF0008002010B50446C0B2FFF7B0
:106DB8001DFCC4F30720BDE8104017E4024B5E2118
:106DC8009868FEF719BC00BF7C14002038B5064C43
:106DD80005465E21A068FEF70FFCA0682946BDE8BD
:106DE8003840FEF709BC00BF7C14002013B50446E8
:106DF80001A90068FFF7EEFA1320FFF7E7FFBDF9D6
:106E08000400FFF7D1FF1B20FFF7E0FFBDF90600E4
:106E1800FFF7CAFF2320FFF7D9FF2368002BB4BF71
:106E280053204E20FFF7C0FF01A96068FFF7D2FA90
:106E38001220FFF7CBFFBDF90400FFF7B5FF1A20BA
:106E4800FFF7C4FFBDF90600FFF7AEFF2220FFF7EA
:106E5800BDFF6368002BB4BF57204520FFF7A4FF90
:106E680002B010BDF8B504460E4617460025204668
:106E780020210BF010FD0446D0B1013420460BF060
:106E88006FFDB0F5617F05DB40F634039842A8BF7B
:106E9800184601E04FF46170A0F56170192390FB6A
:106EA800F3F00DB9307000E070703B7801333B703F
:106EB8000DB90125DBE72046F8BD7FB50478064605
:106EC800E4B9364B1B6803EB8403192193F87B0064
:106ED80093F87C6093F8792093F87A304FF46175D1
:106EE80011FB005011FB0651009001912C482146DE
:106EF800013403F0BAFD142CE3D14CE00BF030FD63
:106F08001328054641DC254B701C1C6820210023F2
:106F18008DF80F300BF0BFFC1E35064670B10136F8
:106F280030460BF01DFD1A289FBF04EB85035870EF
:106F38009DF80F30013398BF8DF80F30304620216F
:106F48000BF0A9FC064670B1013630460BF008FD7F
:106F58000D289FBF04EB850398709DF80F3001330F
:106F680098BF8DF80F3004EB85043046E11C0DF115
:106F78000F02FFF777FF9DF80F30042B0BD0601C32
:106F8800002104220BF051FC05E0064806490022C6
:106F9800132303F06AFD04B070BD00BFE8100020A1
:106FA800A05A0108B55A0108D45A0108014806F048
:106FB80045BE00BFDA5A0108F0B5047887B0064626
:106FC8001CBB524B1968062303FB0411192091F8C6
:106FD800CA5091F8CB7091F8CE2091F8C9304FF48F
:106FE800617610FB056510FB07600095019091F82C
:106FF800CC000290C83146484979039121460134B2
:1070080003F033FD0C2CDCD17DE00BF0A9FC0B2840
:10701800044672DC3D4B701C1D68202100238DF84E
:1070280017300BF038FC064680B1013630460BF0BD
:1070380097FC03289FBF062303FB045383F8CE0065
:107048009DF817309CBF01338DF81730304620214A
:107058000BF021FC074680B1013738460BF080FC65
:107068000D289FBF062303FB045383F8C9009DF82E
:1070780017309CBF01338DF8173006266643A919CF
:107088003846CA310DF11702FFF7ECFE20210BF04C
:1070980002FC074670B1013738460BF061FC142832
:1070A8009FBF9DF817307619013386F8CC0098BF3A
:1070B8008DF81730384620210BF0EDFB78B1013000
:1070C8000BF04EFC0D289FBF062303FB045383F8E7
:1070D800CD009DF817309CBF01338DF817309DF80F
:1070E8001730062B0FD0062202FB04500021C930AE
:1070F8000BF09BFBFFF75AFF05E006480649002204
:107108000B2303F0B2FC07B0F0BD00BFE81000206D
:10711800E85A0108B55A0108D45A01082DE9F3477D
:10712800047807464CB9204601A905F04DFE013404
:10713800FFF7F4FF122CF6D178E00BF011FCC5B282
:10714800112D6DD8781C20210BF0A5FB394C3A4F36
:1071580005F1D006034614F8168030B9A8F10202EA
:10716800D2F1000848EB020843E000F1010A59781F
:1071780038460BF090FB60B1032D8CBF032300232E
:10718800C01B3B4453FA80F090F80490B9F1030F08
:1071980002D1FFF70BFF49E0A9F10203D3F1000880
:1071A80050464FF0200148EB03080BF074FBD8B1B0
:1071B800B8F1000FEDD001300BF0D2FB40F2ED2317
:1071C80080B2984205DD40F6CA039842A8BF184627
:1071D80001E040F2EE2004EB4603A0F2EE20192273
:1071E80090FBF2F0587002E0B8F1000FD1D104F82A
:1071F800169014F81630FA5CB8F1000F0BD00D4B4E
:107208000E4803EB46062946737840F2EE2419250A
:1072180005FB034308E02946094803F026FC05E07E
:10722800084809490022112303F01FFC02B0BDE8F9
:10723800F08700BF481C0020D83C0108085B010803
:107248001A5B0108B55A01083C66010810B50446E6
:107258002046FEF7C5F918B90A20FEF7A2F9F7E7A4
:1072680010BD0C4B5A6882421A4607D01B698342EC
:1072780006D0D36983420BD1022302E0002300E049
:1072880001230021C1620C2000FB032319725960FD
:10729800704700BF702300202DE9F04F06468B4849
:1072A80090F9004087B0B44289469DF84450114691
:1072B8001A469DF840300AD090F90C40B44209D0E3
:1072C80090F91840B4420CD14FF0020804E04FF096
:1072D800000801E04FF001080C2404FB0800047AC0
:1072E8000CB10020EEE0012E00F0DA80142E05D05B
:1072F800002E40F0E68000957548D3E0DFF814A230
:10730800DAF8183043F00103CAF81830DAF8143004
:107318004FF0904543F40033CAF814300127032294
:107328004FF4805B04A94FF090408DF8152003922C
:10733800CDF810B08DF814708DF816708DF81740D0
:1073480002F028F9A5F828B0C820FEF72AF9C5F8F0
:1073580018B0DAF81430039A43F40033CAF814303A
:1073680028464FF4C0534FF0020B04A904938DF83C
:1073780015208DF814B08DF816408DF8174002F0DE
:1073880009F96B6A23F470436B626B6A43F46043D8
:107398006B626B6A23F470236B626B6A43F460233D
:1073A8006B624C4B4C4D4FF480221A6002F18042C4
:1073B800A2F53F321223AB64082385F84D301368D9
:1073C80085F84E7023F480231360536823F48023D8
:1073D800536095F84C3003F1804303F582331A6803
:1073E80042F480221A60AA6C3C4B22F01F0002F083
:1073F8001F02C15807FA02F221EA0202C250AA6C1F
:10740800374922F01F0002F01F0250F801E007FA86
:1074180002F22EEA02024250AA6C22F01F0102F088
:107428001F02C85807FA02F20243CA502D4B2E4ACF
:107438001C60DAF81C3043F40003CAF81C302B4BEC
:1074480004A8DA608DF810608DF811B08DF812403C
:107458008DF8137005F088F92A238DF810309DF8FF
:1074680013308DF811708DF812401BB104A805F087
:107478007BF904E01E4B4FF48062C3F884201D4A58
:107488001D4B136002221A721C4A1D4B13601D4AC1
:107498001D491B68116098471C4B2B600E4806E07D
:1074A8001B480095FBF7F8FA00283FF41AAF074B82
:1074B80006710C2202FB083888F80890C8F8040006
:1074C80000E0204607B0BDE8F08F00BF7023002021
:1074D80000380140140401408C14002008040140C5
:1074E8000C040140D80042420005FA0500ED00E016
:1074F80000E100E0241B0020942300200C1B002046
:10750800A0000020081B002004000020E43C010823
:1075180000440040001002400C4B1B6893F9022005
:10752800824209D093F90A20824207D093F91220A7
:10753800824208D1022002E0002000E0012003EB93
:10754800C000023070470020704700BF6C23002045
:10755800F0B5027887B0AAB94C4C04F118064C4B28
:1075680094F9F41193F900208A4272D093F90C200F
:107578008A426ED093F918308B426AD00834B442EC
:10758800EDD180E0002204920592451C0BF0E8F949
:10759800C4B260B2FFF7C0FF074618B18DF81040BB
:1075A800012400E00446284620210BF074F9054622
:1075B80038B1013528460BF0D3F90134ADF8120083
:1075C800E4B20026284620210BF065F9B0B3451C2B
:1075D80028460BF0C5F900222E4951F82230834283
:1075E8005FFA82FE04D00132082AF5D1002300E0B8
:1075F800734651F82320824220D1022E0FD0032E49
:1076080012D05A1E012ED2B204D0042A13D88DF8F3
:1076180014300EE0042A0ED88DF8153009E0052B39
:1076280009D88DF8173004E09A1E052A03D88DF87A
:1076380016300134E4B20136042EC3D1052C03D828
:1076480007B0BDE8F040B1E404AB03CB3860796023
:1076580019E094F8F9010F4B94F8F85153F8200009
:10766800B4F8F621009094F8FB0153F8200001903B
:1076780094F8FA0153F82000029053F82530064890
:1076880003F0F3F97AE707B0F0BD00BF481C00200B
:107698007023002080450108295B010838B1438820
:1076A80011EA030003D08B420CBF0120022070476F
:1076B80030B50B4B0B491C6891F85020022A0BD8A7
:1076C800134604EBC303551CEAB29D882842F5D043
:1076D80081F85020981C30BD81F85020002030BD22
:1076E8006C2300208C140020024B002283F85020C9
:1076F800DEE700BF8C1400202DE9F047877890F86A
:1077080003C0214DBBB2C7F1640E03EB83065C4294
:10771800C3F178005FFA8EFE7600CCF16408A4B25B
:1077280080B2A3B20FFA83F9B9F1000F05DC002B80
:1077380014BFBA464FF0010A00E0F24613FB03F308
:1077480003FB0CF21AFB0AF392FBF3F3434403FB2B
:1077580009F30A2293FBF2F333449BB225F8023F64
:10776800B1F800904A880A34C9EB020AA4B21AB2E6
:1077780002FB0AF24FF47A73844292FBF3F34B4410
:107788002B80CED1BDE8F087DC14002010B54478FA
:107798000078002202FB02F3193B634303F6C4138B
:1077A800534340F6C411434393FBF1F3034921F8D3
:1077B80012300132072AEDD110BD00BFF6140020A7
:1077C8000430114B33F91000B0F5617F10B506DBBA
:1077D80040F6330398420246A8BF1A4601E04FF428
:1077E80061720C78192340F2833013FB040494422D
:1077F80007DA497813FB01039342B4BF0020012044
:1078080010BD002010BD00BF7826002010B500F183
:10781800500302788A4203D18478C278944204D310
:1078280004309842F5D1002010BD012010BD0B4B4B
:107838001B6813F4805F0A4BB3F9063005D0C08982
:10784800421A934207DD084400E0008A8342B4BF2D
:107858000020012070470120704700BF781B0020DE
:10786800782600201FB5094B1B681B030AD58DF825
:10787800040001230D2001A98DED030A8DF80530C0
:10788800FEF7EAFE05B05DF804FB00BF781B002098
:107898001FB5084B1B681B0309D58DF8040002911E
:1078A80000230D2001A98DF80530FEF7D5FE05B09F
:1078B8005DF804FB781B002010B50020FDF78AFE58
:1078C800064B00241C7007F07FFD054B83F87840B9
:1078D800DC67A3F88040C3F8844010BDC8260020A8
:1078E8008C14002010B510B9BDE81040E4E700235F
:1078F8000C225A430B4C1119125D824203D00133FA
:10790800102BF5D110BD084BD3F8840018B14A7874
:107918004078824205D20022C3F88410A3F8802060
:10792800DA6710BDA04501088C14002010B540008E
:107938001428A8BF14200023074A022199540B4495
:1079480099181424834201F8014CF5DBFF21D15426
:107958000F20BDE81040C5E7B42400202DE9F84306
:1079680007460B24013C36D01D4B4FF480529A61D8
:107978007D1C32264FF00508DFF86490B9F8143002
:107988009BB283F48053A9F814300120FDF722FE3E
:107998003046FDF706FEB9F814309BB283F48053E5
:1079A8000020A9F81430FDF715FE3046FDF7F9FD63
:1079B800B8F1000F08D0B8F10108DDD14FF4FA7022
:1079C800FDF7EFFDFA26D7E7013DD5D14FF47A70E0
:1079D800FDF7E7FDC6E7034B034ADA60BDE8F88325
:1079E8000004004800ED00E00400FA052DE9F04F1E
:1079F8002DED028B87B0074603938E4B1B889807A3
:107A0800934636D5129B8C48DC89B0F900301B1B95
:107A180003F2F31540F2E632954203D8002BB8BFC3
:107A28005B4201E04FF4FA73B0F90220121B02F234
:107A3800F31440F2E630844203D8002AB8BF524219
:107A480001E04FF4FA729342B8BF1346C3F5FA73D4
:107A5800052293FBF2F33A7F0A25643B6B43D2106D
:107A68005343642593FBF5F5643525EAE575EBB2D8
:107A780000E064230193CB1C0293B8460025029BC7
:107A8800DFF8C8A113F8016F0293022D4FEA4509E8
:107A980005D1BAF904201B365643761146E06748EB
:107AA8003AF8151030F91500022411FB0400CBF147
:107AB8000001884203DB58450146A8BF5946604883
:107AC800039B30F909400C1B33F915100C4407F0DF
:107AD80007FA88B107EE904A5A49B8EEE70AB2EEBB
:107AE800048A485D80EE080A04F088FE20EE080A41
:107AF800FDEEC07A17EE904A4E490988CA0712D49B
:107B08003AF909201B3656438B074FEA26160DD53E
:107B1800BA7C54439DF904205443642294FBF2F444
:107B280006EB241602E03E7A74432611464A0424E2
:107B380032F9092092FBF4F4444A02F10801341B9B
:107B48006E5C98F80110614371436420022D91FB2B
:107B5800F0F14FEAE11308EE103A0AD1B8EEC80A7C
:107B680002F10C001E21D2ED050A02F05FFDBDEE08
:107B7800C08A364B364803F118014FEA850C51F894
:107B88002520B2F5001FA8BF4FF400128242B8BFEB
:107B9800024641F8252003F12401521351F825002B
:107BA80041F82540201A00214FF6FF74B4FBF1F18B
:107BB80089B24143891100EE101A97F8501089B123
:107BC80003F13000B8EEC00A00EBC500D3ED050A9A
:107BD800CDF814C0049202F029FDDDF814C0049A0F
:107BE800BDEEC00A98F8151010EE103A594318EE79
:107BF800103A4E439818642196FBF1F6154936124F
:107C0800304421F8090001F1080001354CF8003032
:107C180001F114002031032D4CF800204CF80160CC
:107C280008F101087FF42BAF07B0BDEC028BBDE86B
:107C3800F08F00BFA810002078260020EE26002034
:107C48006E1B0020043D0108D210002014150020EE
:107C58000000E0FF5C1500202DE9F04F2DED028BB0
:107C680087B000260593C04B0491B3F90270B3F9AD
:107C780000300292002FB8BF7F42002BB8BF5B4292
:107C88009F42B8BF1F46B7F5FA7F8046A8BF4FF49A
:107C9800FA770090B3460196B2463446B34D2B8826
:107CA80099075AD0B04BB24A33F8143032F914203D
:107CB800022013FB0022029B5B429A424FEA4401D6
:107CC80003DB029B9342A8BF1346AA4A31F90290EC
:107CD800059A32F91420C9EB030303EB020907F0F4
:107CE800FFF888B107EE909AA34BB8EEE70AB2EE18
:107CF800048A185D80EE080A04F080FD20EE080A68
:107D0800FDEEC07A17EE909A98F80830642203FBCB
:107D180009F393FBF2F398F81C206FF0040A0AFBAE
:107D280002FA534504DB02EB820A9A45A8BF9A4639
:107D3800924A52F8241009EB010342F210718B4267
:107D4800A8BF0B468E498B42B8BF0B4642F8243079
:107D580098F8122053431B1301932D8805F0030351
:107D6800012B38D0009B804993F801C0854B31F92D
:107D780014B033F9140080EAE0731831A3EBE07310
:107D8800B3F5206F4FEA840651F824E016DC0BEBBC
:107D98008B031A0192FBFCF3042290FBF2F0181AF1
:107DA8008644BEF57A5FA8BF4FF47A5E764B9E454F
:107DB800ACBF41F824E041F8243002E0002341F848
:107DC80024308B597D2693FBF6F6009BDB7A7343B0
:107DD800402693FBF6F6AA0711D50198C7F5FA7362
:107DE80007FB0BF907FB06F54FF4FA7103FB0A9939
:107DF80003FB005599FBF1F295FBF1F505E0EB0764
:107E08004DBF019D35465A465246DFF85CE1630096
:107E180003930EF17C015B4B615C33F814004FF067
:107E2800040C03B293FBFCF909FB01F16FF04F0955
:107E380091FBF9F991440EF1800232F9141022F8FD
:107E480014005B1A98F8501093FBFCF300EE103AFC
:107E580059B10EF13000B8EEC00A00EBC400DEEDF7
:107E6800050A02F0E3FBBDEEC00A3F4A039802F19F
:107E7800840110EE103A11F804C002F1480E09EB23
:107E880005010CFB03F34FF0200C93FBFCF3C91A1C
:107E980020F80E1002F1680002F150015B4240F830
:107EA8002430009B41F8249002F15C01013341F831
:107EB800245000930CB90124F0E6049BB2F9041095
:107EC8009B79146A0F335B004B435B112D49002BE0
:107ED800B1F904104FF0040091FBF0F0A3EB00009F
:107EE800B8BF5B42322B98F80D100BDC274B01FB17
:107EF80000418B42A8BF0B4625498B42ACBF136299
:107F0800116201E00023136298F8031001FB00F3EB
:107F18002049097803294FEAA3130CD9B8F84E1061
:107F2800B1F5FA7F07D24842834203DB8B42A8BFF0
:107F38000B4600E00346116A936541F34F31B1F5F2
:107F4800807FA8BF4FF480716FF0FF008142B8BFF7
:107F5800014658180023A2F84C005166136707B071
:107F6800BDEC028BBDE8F08F14150020A81000208E
:107F7800EE2600206E1B0020043D01088815002015
:107F8800F0D8FFFFD210002080C1FFFFFEFFFF0FD7
:107F9800020000F0C01100202DE9F04F2DED028BFA
:107FA80085B080460393AA4B02911C88019204F085
:107FB8000204A4B294B1A74BB3F90240B3F900305C
:107FC800002CB8BF6442002BB8BF5B429C42B8BFCC
:107FD8001C46B4F5007FA8BF4FF40074C2460025C4
:107FE8009D4B9C4A33F9153032F8151083EAE37734
:107FF8001832A7EBE37708B2B7F5206F4FEA450BC5
:108008004FEA40004FEA850952F8256011DC042741
:1080180093FBF7F3C31A1E44B6F57A5FA8BF4FF473
:108028007A568E4B9E42ACBF42F8256042F8253006
:1080380002E0002342F8253052F809609AF80B3024
:108048009AF80170F6115E43814B1B8847439B07E2
:108058004FEAA6164FEAA71756D0814B33F90B30D3
:10806800022211FB0231019B5B42994203DB019B17
:108078008B42A8BF0B467B4A3BF902209A1A039B06
:1080880033F91530D31808EE103A06F029FF68B115
:10809800B8EEC80A744BB2EE048A80EE080A585D3E
:1080A80004F0ACFB20EE080ABDEEC08A6F4918EE5A
:1080B800102A59F8013042F2107013448342A8BFC5
:1080C80003466B4898F808208342B8BF034649F82E
:1080D800013018EE101A4A4398F81C1001EB810180
:1080E800D2114842824203DB8A42A8BF0A461046A0
:1080F80098F8122053431B13F61A3F1A6643674336
:1081080003EB662600EB6727DFF848E1524B0EF1D8
:108118007C0C3BF803101CF805C00BB2042093FB41
:10812800F0F202FB0CF2A7EBA2170EF188023BF962
:1081380002C02BF8021098F85010CCEB030393FB05
:10814800F0F300EE103A59B10EF13000B8EEC00A63
:1081580000EBC500DEED050A02F068FABDEEC00AC4
:108168003C4A02F1840110EE103A485D43435B112A
:1081780002F14800B919C91A2BF8001002F1500190
:108188005B4249F8017002F15C010AF1010A49F801
:10819800016002F1680149F801300DB901251FE7B6
:1081A800029BB2F904109B79146A0F335B004B43AE
:1081B8005B112949002BB1F904104FF0040091FB21
:1081C800F0F0A3EB0000B8BF5B42322B98F80D101B
:1081D8000BDC284B01FB00418B42A8BF0B4626490C
:1081E8008B42ACBF1362116201E00023136298F85E
:1081F800031001FB00F32149097803294FEAA3136F
:108208000CD9B8F84E10B1F5FA7F07D2484283422C
:1082180003DB8B42A8BF0B4600E00346116A936557
:1082280041F34F31B1F5807FA8BF4FF480716FF0F3
:10823800FF008142B8BF014658180023A2F84C003D
:108248005166136705B0BDEC028BBDE8F08F00BF27
:10825800A810002014150020D210002080C1FFFFB4
:10826800EE2600206E1B0020043D01088815002022
:10827800F0D8FFFFFEFFFF0F020000F0C011002042
:108288002DE9F04F2DED028B85B000260393AB4B03
:108298000292B3F90270B3F900300090002FB8BF12
:1082A8007F42002BB8BF5B429F42B8BF1F46B7F55D
:1082B800FA7F8146A8BF4FF4FA77B2460196B046D6
:1082C8003446DFF8A0B29D4DBBF8003013F0030F21
:1082D80059D0022C57D09A4935F8143031F9141076
:1082E8004FF0020E13FB0E11029B5B4299424FEABC
:1082F800440003DB029B8B42A8BF0B469149039ABB
:10830800415E5B1A32F914100B4408EE103A06F07D
:10831800E7FD68B1B8EEC80A8B4BB2EE048A80EE6E
:10832800080A185D04F06AFA20EE080ABDEEC08A51
:1083380099F8083018EE102A6421534393FBF1F39F
:1083480099F81C106FF0040808FB01F8434504DB9A
:1083580001EB81089845A8BF98467C4918EE103A69
:1083680051F82400034442F210708342A8BF034628
:1083780077488342B8BF034641F8243099F8121071
:108388004B431B130193BBF8003003F00301012991
:1083980001D1022C41D135F914A06E4D009A35F95E
:1083A80014506D4892F801E050F8242085EAE576EB
:1083B800A6EBE576B6F5206F4FEA840120DC022CA7
:1083C80018D00AEB8A00000190FBFEFE042095FB02
:1083D800F0F5C5EB0E0E02EB0E0CBCF57A5F5E48AD
:1083E8005E4DA8BF4FF47A5CAC45ACBF41F800C005
:1083F8000D5007E08AEAEA76A6EBEA76642EE0DD1D
:10840800002545505448009A09587D2691FBF6F6F8
:10841800D17A7143402691FBF6F69A0713D5022CC0
:1084280011D0019BC7F5FA7107FB06F507FB0AF0A7
:1084380001FB08004FF4FA7E01FB035190FBFEF0AC
:1084480091FBFEF508E0DB0704D5022C02D0019D64
:10845800404601E0354650463E4B384A33F9141041
:10846800042391FBF3F302F17C01022C615C03FB12
:1084780001F36FF04F0193FBF1F303444FEA440B10
:1084880008EE103A0AD1B8EEC80A02F10C001E2113
:10849800D2ED050A02F0CAF8BDEEC08A274A2D4B74
:1084A80002F18C013BF803003BF901302BF8010085
:1084B80099F850100FFA80FCC3EB0C034FF0040C32
:1084C80093FBFCF300EE103A59B102F13000B8EE1C
:1084D800C00A00EBC400D2ED050A02F0A7F8BDEE11
:1084E800C00A1F4910EE103A085D00FB03FC18EEA5
:1084F800103A4FF0200E58199CFBFEFCA1F13C0EDF
:10850800CCEB00002BF80E00A1F1340E4EF824300D
:10851800A1F128031C3943F82450CCF1000341F899
:108528002430009B01340133032C00937FF4C9AE3F
:1085380005B0BDEC028BBDE8F08F00BF141500201C
:10854800EE2600206E1B0020043D0108881500203F
:10855800F0D8FFFFD21000202C15002080C1FFFFAB
:1085680098150020A81000202DE9F04F2DED0A8B5A
:1085780085B00446039390F85030029190461BB1A1
:10858800322BA8BF322300E0012307EE903AB8EE61
:10859800E7BADFEDDB7ADB4BDFEDDBBA1B88DB4DBF
:1085A800019587EE8BBA002B08BF0123DFF8A4A33F
:1085B80007EE903AF8EEE79A2B8869EEABBA13F01B
:1085C800020F3BEE2BBA8BEE8BBA26D0BAF90030ED
:1085D800BAF9021083EAE37081EAE176A0EBE3706E
:1085E800A6EBE17686423746B8BF0746B7F5E17F86
:1085F80016DA8642DFEDC6AA05DD0029D8BF494252
:1086080007EE901A04E0002BD8BF5B4207EE903AC1
:10861800F8EEE77AC7EEAAAA04E0DFEDBEAA01E009
:10862800F7EE00AA9FEDBB9ABB4D26464FF0000B14
:10863800B0EE49AADFF8189339F91B300CEE103A5E
:10864800B8EECCCAF5EE047A3AF91B302CEE27CAFC
:1086580008EE903A019BBDEECCCA1888F8EECC7AA9
:108668009FEDAECA81074FEA4B0727EE8CCAF8EE9A
:10867800E88A00F08380AA4830F91B3007EE903A68
:10868800F8EEE77AB0EE007AE8EE877AC8F1000EE5
:10869800FDEEE77A17EE900A704503DB4045A8BF68
:1086A800404686469F48039B385EC0EB0E0E33F962
:1086B8001B00864407EE90EAB8EEE78A06F010FC45
:1086C80050B19948B2EE049A88EE090A10F80B00E6
:1086D80004F094F820EE098A237FDFED946A0AEE0D
:1086E800103A237A07EE903AF8EE677AB8EE4AAA7B
:1086F80068EE277AB1EE047A67EEA67A2AEE077A50
:10870800FDEEE77A17EE900AF1EE477ABDEEE7AA9A
:108718001AEE103A984208DBBDEEC7AA1AEE103AD4
:108728008342A8BF03460AEE103A814800EB8B004B
:10873800D0ED007AE8EE2B7ABBEE0E7AF4EEC77A2B
:10874800F1EE10FAB8EECAAA09D4B3EE0E7AF4EE36
:10875800477AF1EE10FAC8BFF0EE477A01E0F0EE82
:10876800477AC0ED007AA37C09EE103AB8EE499A30
:1087780067EE897A9FED6F9A27EE899A019B188890
:10878800C20754D439F907E0BEF1000FB8BFCEF1E3
:10879800000EBEF5206F04DD4FF0000EC5F800E0B6
:1087A80025E09FED657A737868EE877A07EE103AD0
:1087B800B8EE477A87EE877AD5ED007A37EE4C7AAD
:1087C800E7EE2B7A9FED5D7AF4EEC77AF1EE10FAB8
:1087D80009D49FED5B7AF4EE477AF1EE10FAC8BF40
:1087E800F0EE477A01E0F0EE477AC5ED007AF37AC9
:1087F800D5ED007A08EE103AB8EE488A830768EE9D
:10880800277A9FED508A27EE888A14D578EECA8A8F
:10881800F0EE4A7AEAEEA87A38EE498AF0EE678AEC
:10882800F0EE497AEAEE887AB0EE678A03E0B0EEB5
:10883800498AF0EE4A8ADFF81C919FED437A09F1E4
:108848007C0009F1A80E1BF8003007EE903AF8EE0C
:10885800E77A4FEA8B0067EECC7A8644E7EE878AA0
:10886800043501369EED007A8EED00CA3CEE477A5B
:1088780009F1B00E87EE2B7A7044D0ED007A37EE0E
:10888800677AF0EE68CAEBEE077A3CEE880AC0ED2C
:10889800007A09F184001BF8003008EE903AF8EEEF
:1088A800E88A67EEA87ADFED298A67EEA88A30EEB3
:1088B800680A0AF0C9F909F1480EFDEEECCA2EF86B
:1088C80007001CEE903A09F15000BDEEC88AF1EE9F
:1088D800688A40F82B30FDEEE88A09F15C0018EE52
:1088E800103A40F82B3009F1680018EE903A40F839
:1088F8002B30BBF1000F2FD14FF0010B9AE600BFD0
:1089080083F9223E98100020BD378635A810002034
:108918000000E14300000000A8150020CDCC4C4029
:10892800EE2600206E1B0020043D01086F12033C58
:10893800B41500200AD7A33D0000A043000040C39F
:10894800000040430AD7233CA69B443BF7CC92380F
:10895800D210002014150020029AB9F90430957934
:108968006D0028355D434B4BB3F9043000EE103AE7
:10897800BAEECF0A0AF068F96D11281A002D07EE31
:10898800900AB8BF6D42322DF8EEE76A03DD002386
:10899800C9F8203028E0FDEEE99A3F4919EE903AEF
:1089A80023F0030307EE903AF8EEE79ADFED3B7AFF
:1089B800637BC9EEA77A07EE103AB8EE477AD9F882
:1089C800203026EE877A67EE277AFDEEE77A17EEF3
:1089D800902A13448B42A8BF0B4631498B42ACBF47
:1089E800C9F82030C9F82010DAF820305B13B3F545
:1089F800807FA8BF4FF480736FF0FF018B42B8BF30
:108A08000B4607EE903AF8EEE78AFDEEE67AE17853
:108A180017EE903A4B439B1107EE903A214B1B7887
:108A2800032BB8EEE78A14D9B4F84E10B1F5FA7FE3
:108A38000FD2FDEEC87A4B4217EE900A984204DB3B
:108A4800884217EE903AA8BF0B4607EE903AB8EE68
:108A5800E78A38EE280ABDEEC00A8DED010ABDF995
:108A6800043000EE103AB8EEC00A0AF0EDF8BDEE98
:108A7800C88AFDEEE88A0023AAF84C008AED168A17
:108A8800CAED198ACAF8703005B0BDEC0A8BBDE88A
:108A9800F08F00BFD2100020FEFFFF0F00803B4583
:108AA800020000F0C011002010B5214A18B913685F
:108AB80002221A8210BD1F481468002303802178FF
:108AC80011F07F0102460DD1637A990644BF022155
:108AD800017013F0400F037814BF43F0010323F033
:108AE800010315E0012921D002291ED1637913F071
:108AF800800F03F00F034FEA830303F1804303F56C
:108B0800B8431B6806D003F03003102B07D10123AC
:108B1800137004E003F44053B3F5805FF6E7064BA7
:108B28001B681B699847034810BD184610BD00BF55
:108B3800241B0020D0150020081B002010B5064C6F
:108B480018B9236801221A8210BD044B1B689B6860
:108B5800984720680C3010BD241B0020081B0020FB
:108B680010B5064C18B9236801221A8210BD044BAF
:108B78001B681B68984720680A3010BD241B00201A
:108B8800081B002003788B4283BF034B03EB410192
:108B980048880020704700BFD015002070B500221B
:108BA8001346244914180C44A47E83EA0423082499
:108BB80013F4004F4FEA430318BF83F4815304F1C1
:108BC800FF3418BF83F0010314F0FF049BB2EFD108
:108BD8000132192AE5D100F1190200F11A050A44F7
:108BE8000D44967EAA7E02EB062292B29A421FD1CB
:108BF800104B93F83B50E2B2AA4216D2431C03EB47
:108C08004203DBB2CA1801330B44927E9B7E03EB0E
:108C180002239BB24FF4AF6253431B13064A03F57A
:108C2800487322F814300134E5E7012381F83C3019
:108C380070BD00BFD0150020D215002003788B42EC
:108C48000BD9074B1A78074B89001944086C02B1F5
:108C5800400800F5777080B270470020704700BF69
:108C680068230020D015002007299DBF034B03EB84
:108C78008101B1F870000020704700BFD0150020B6
:108C8800034B03EB4101B1F89000C008704700BFE7
:108C9800D01500200A4BDFED0B7A03EB810191ED33
:108CA8002C7AB8EE477AF6EE046AE7EE267A82B0B6
:108CB800FCEEE77ACDED017ABDF8040002B070470A
:108CC800D015002000005C44024B03EB4101B1F8D1
:108CD800F8007047D0150020024B03EB4101B1F8B2
:108CE8001C017047D015002070B5334C0546FCF7C1
:108CF80032FCD4F83431C4F83401C31AB3F5FA5F3E
:108D0800C4F8383182BF002384F83C3184F83D31FF
:108D180094F83C312BB9A12D02BF274A012182F8D2
:108D28003D1194F83D11244A29B1D118EDB201330F
:108D38008D7682F83C3194F83C5194F83E31AB4240
:108D480039D11D4B93F83F31052B02D0062B03D0A8
:108D58002CE00020FFF722FFE37E1E2B26D1002007
:108D68000246C1B26B1E994219DA21448B7E082152
:108D7800DBB283EA0206F60744BF83F01803C3F3A5
:108D8800460301F1FF3154BF5B0843F0800311F043
:108D9800FF01C2F34702ECD101301A46E1E7234450
:108DA8009B7E9A4202D10320FFF7F8FE002384F845
:108DB8003D3184F83C3170BDD015002010B5044613
:108DC800FCF7C9FB0F4BD3F84021C3F84001821AC6
:108DD80041F288318A42C3F8442184BF002283F8D3
:108DE800482193F84821074913440F2AE4B218BFD1
:108DF800013283F8494112BF81F84821012381F8E3
:108E0800593110BDD015002010B50446FCF7A3FB5E
:108E18000F4BD3F85C21C3F85C01821A41F2883108
:108E28008A42C3F8602184BF002283F8642193F842
:108E3800642107491344142A18BF013283F8654195
:108E480012BF81F86421012381F87A3110BD00BF77
:108E5800D015002038B50446FCF77DFB274A274982
:108E6800D2F87C31C2F87C01C31AB3F57A6F84BF9B
:108E7800002382F8803192F8803133B9A82C3BD195
:108E880081F88131A1F8823106E0022B02D181F804
:108E9800844101E0242B02D8D11881F8854192F849
:108EA8008411164D01330231DBB249008B4282F83E
:108EB800803118DAB5F88231E0B283EA002008235D
:108EC80010F4004F4FEA400018BF80F4815003F1BE
:108ED800FF3318BF80F0010013F0FF0380B2EFD119
:108EE800A2F8820138BD01318B4201BF002385F809
:108EF8008031012385F8813138BD00BFD0150020AD
:108F080010B50446FCF727FB104AD2F8AC3140F6FE
:108F1800AC51C31A8B42C4BF002382F8B03192F817
:108F2800B031D11881F8B14123B90F2C0DD10749BF
:108F3800C1F8AC010133DBB2192B044982F8B03116
:108F48000CBF0123002381F8CA3110BDD0150020C1
:108F58002DE9F843324F3D682A8A2E7AB2B9042E99
:108F680014D1304C30482378012B0BD12F4B196882
:108F78002F4B89B20B445B0019681A6030230380B9
:108F8800227048E010230380072644E0AC8AAB69CE
:108F9800A24294BF04260226944228BF14461FFA10
:108FA80084F840469847214A13689BB203F100535E
:108FB80003F540535B0004F1010E1B689BB203F1FB
:108FC800005303F540534FEA6E0E5B0000217145D4
:108FD80000F1020009D010F8019C10F802CC4CEA0C
:108FE800092C23F821C00131F1E71268104B92B225
:108FF80013445B001A681C602B8AC8EB03032B829E
:109008006B8A9844084BA5F8128030221A80094BC5
:109018004FF440521A803B681E72BDE8F88300BFC7
:10902800241B0020F6260020021B0020505C004074
:1090380002300020001B00200E4B0F4A1B689BB219
:1090480003EBC00002443E294FEA420209D94B090A
:10905800C80604BF03F1FF339BB29B0243F40043ED
:1090680004E04B08C90748BF01339B02116813602D
:10907800704700BF505C00400630002010B5454BDB
:109088001A68107810F07F0004D1537A23F0200377
:10909800537210BD02287AD15388002B78D11379E6
:1090A800002B75D1537923F08000840004F18041AE
:1090B80001F5B84113F0800F096814BF01F03001C1
:1090C80001F44051032862D8002960D0927A002A1E
:1090D8005DD004F1804404F5B8441906226825D50A
:1090E80002F03002102A4CD103F07F039B0003F1F9
:1090F800804303F5B8431A68510641BF196840F622
:109108000F720A4042F4004244BF42F0C0021A60A3
:109118001A6822F4E04222F0400292B282F0300251
:1091280042F4004242F080021A602AE002F44052FF
:10913800B2F5805F25D128B9174B93F82C10FFF7AB
:109148007BFF11E09B0003F1804303F5B8431A68E5
:10915800520441BF196840F60F720A4042F4404277
:1091680044BF42F080021A60236823F4804323F04E
:1091780070039BB283F4405343F4004343F08003ED
:109188002360064B1B685B699847002010BD0220CE
:1091980010BD00BF241B0020A0000020081B0020D9
:1091A80002684FF6FE7313400360002303604360B8
:1091B8008360C360284B984201D1284A27E0284B96
:1091C800984201D1254A2AE0264B984201D1234AE8
:1091D8002DE0254B984201D1204A30E0234B98429C
:1091E80001D11E4A33E0224B984204D11B4A5368EE
:1091F80043F470032EE01F4B984204D1174A53687A
:1092080043F0706326E01C4B984204D11B4A536814
:1092180043F00F031EE01A4B984204D1174A5368D3
:1092280043F0F00316E0174B984204D1134A5368F1
:1092380043F470630EE0144B984204D10F4A53680C
:1092480043F4704306E0114B984204D10B4A53682B
:1092580043F4702353607047080002400000024046
:109268001C00024030000240440002405800024006
:109278006C000240800002400804024000040240E2
:109288001C040240300402404404024058040240D6
:10929800084BDA68D10709D4DA68D20608D4DB6843
:1092A80013F0040F14BF03200420704701207047F7
:1092B8000220704700200240994A536803F00C03CB
:1092C800042B2DE9F04105D0082B06D09549016003
:1092D800B3B916E0934B036012E053685468C3F3C4
:1092E8008343991CE30349BFD36A8F4B8D4C03F02A
:1092F8000F0344BF0133B4FBF3F34B43036000E0B7
:1093080000235168894FC1F303117D5C0168EDB2F8
:1093180021FA05F444605668C6F30226BE5D24FAB5
:1093280006FEC0F808E05668C6F3C226BE5DF6B26F
:10933800F440C460D2F82C80C8F3041808F00F0C6D
:1093480007EB4C0C18F0100FBCF810C01FFA8CFC7F
:1093580007D0BCF1000F04D0B3FBFCFCC0F810C070
:1093680000E00161D2F82CC0CCF3442C0CF00F08BB
:1093780007EB48071CF0100F3F8ABFB204D01FB19B
:10938800B3FBF7F7476100E04161176BFF065ABF6F
:10939800644F87618161176BBF065ABF614FC76110
:1093A800C161176B7F065ABF5E4F07620162176B78
:1093B800FF0506D5994204D1AE4202D14F0047625B
:1093C80000E04462176BFF0406D5994204D1AE420F
:1093D80002D14F00876200E08462176BBF0506D593
:1093E800994204D1AE4202D14F00C76200E0C46284
:1093F800176B7F0506D5994204D1AE4202D14F00C2
:10940800476400E04464176B3F0506D5994204D1D0
:10941800AE4202D14F00876400E08464176BBF043A
:1094280006D5994204D1AE4202D14B00C36400E094
:109438008464156B3A4BAD0701D1046315E01C6BCE
:1094480004F00304012C01D101630EE01C6B04F04D
:109458000304022C02D14FF4004305E01B6B03F018
:109468000303032B01D12F4B0363146B2C4B14F410
:10947800403F02D1C0F834E018E01C6B04F44034DB
:10948800B4F5803F01D1416310E01C6B04F4403413
:10949800B4F5003F02D14FF4004306E01B6B03F420
:1094A8004033B3F5403F01D11E4B4363146B1C4B53
:1094B80014F4402F02D1C0F838E018E01C6B04F413
:1094C8004024B4F5802F01D1816310E01C6B04F4B3
:1094D8004024B4F5002F02D14FF4004306E01B6B83
:1094E80003F44023B3F5402F01D10E4B8363146B73
:1094F8000B4B14F4401F02D1C0F83CE020E01C6B79
:1095080004F44014B4F5801F01D1C16318E01C6B4A
:1095180004F44014B4F5001F0AD14FF400430EE0E0
:109528000010024000127A0000093D0028000020C7
:109538001B6B03F44013B3F5401F01D1134BC363F6
:10954800126B134B12F4400F03D1C0F840E0BDE892
:10955800F0811A6B02F44002B2F5800F02D1016467
:10956800BDE8F0811A6B02F44002B2F5000F02D197
:109578004FF4004306E01B6B03F44003B3F5400FC0
:1095880001D1024B0364BDE8F08100BF00127A00EC
:1095980000100240F0B500230E681C460125A540C6
:1095A80005EA060EAE452BD10F797A1E012A15D889
:1095B800856803229A4025EA020282604D79826812
:1095C8009D4015438560828892B222EA0E0282800D
:1095D8008A798588A2402A4392B28280032205684C
:1095E8009A40D2431540056005689F402F430760A5
:1095F800C7681740CA7902FA03F547EA0502C2604C
:109608000134102C03F10203C8D1F0BD38B52DED9B
:10961800048B4A4C0368C4F8CC318388A4F8D03151
:10962800013A0D46072A42D8DFE802F0040A10186A
:1096380022292F35B4F8CC310B80B4F8CE3113E0A1
:10964800B4F8CE310B80B4F8CC3105E0B4F8CC31A5
:109658005B420B80B4F8CE315B4205E0B4F8CE3102
:109668005B420B80B4F8CC316B80B4F8D0311DE08C
:10967800B4F8CC315B420B80B4F8CE3112E0B4F8C8
:10968800CE310B80B4F8CC310CE0B4F8CC310B807F
:10969800B4F8CE3105E0B4F8CE315B420B80B4F8B3
:1096A800CC315B426B80B4F8D0315B42AB80244B49
:1096B80093F83030002B3ED1B5F9003094ED780A9C
:1096C800D4ED757A09EE103AB5F9023008EE103A81
:1096D800B8EEC88AB5F90430B8EEC99A28EE000A7F
:1096E80008EE903AA7EE890AF8EEE88AD4ED7B7A7C
:1096F800A7EEA80A09F0A8FA94ED790AD4ED767ACB
:10970800288028EE000AA7EE890AD4ED7C7AA7EE15
:10971800A80A09F099FA94ED7A0AD4ED777A688064
:1097280028EE000AA7EE890AD4ED7D7AA7EEA80AEA
:1097380009F08AFAA880BDEC048B38BDD01500204A
:1097480028000020094BD3F8F821137844F6FB7160
:1097580003EB431300FB03135078C0EB0030B3FB5B
:10976800F0F39078B3FBF0F080B27047D01500208A
:1097780010B5074C00210A2204F50070A4F8FC116A
:10978800FBF73DFF80B2FFF7DDFFA4F8880210BDAC
:10979800D015002038B500240B4D6059254404F03D
:1097A8004DFA696811B1094801F05FF9A96811B16A
:1097B800074801F05AF90748103404F03FFAB4F5A5
:1097C800C87FE9D138BD00BF083D0108185C010811
:1097D8001E5C010836640108F0B585B0044609F03E
:1097E80068F8082826D1621EE01D1F4912F8013FBB
:1097F80009681944497801F00301022908BF203B90
:1098080082421370F1D1254604F1080715F8016B5F
:109818001648314609F03FF820B12846314609F08C
:109828003AF810B1FDF7C2FB1CE0BD42EED120466C
:1098380003F0ACFA0E4804F001FA00230D4A1A446A
:1098480004A992F888210A440849595C02F80C1CBA
:109858000133082BF2D1002307488DF80C3001A9F9
:1098680001F003F905B0F0BDFC000020DE6201083C
:10987800245C0108481C0020786301081E4B1F4C1B
:109888001D68206880B5FDF7E1FC2846FDF7DEFC81
:10989800206841798B0704D4036841F002015B69B1
:1098A8009847174B4FF480529A612068FBF7A1FE46
:1098B800A0B1134E4FF480533385104B1868FBF753
:1098C80095FE074601F0E5FC08B103F047FC284681
:1098D8003946FBF791FE4FF48053B3612846FBF7F6
:1098E80088FE0028E1D028462668FBF77FFE01465F
:1098F8003046FBF781FED8E7A0240020601800203E
:10990800000400482DE9F047054608F0D2FF314E23
:109918000446D6F8088090B92F4804F08FF92F4BE9
:1099280053F8241049B10123A34013EA080F02D0C9
:109938002B4801F09AF80134F1E72A4822E028463A
:109948002949224608F0BEFF58B92848284C04F097
:1099580075F954F8041F0029EFD0214801F085F863
:10996800F7E72B782D2B03BF013504F1FF344FF0B7
:10997800010A4FF0000A4FF00009184B53F82970FC
:1099880027B91C48BDE8F04704F058B928463946BD
:10999800224608F097FFC8B9012000FA09F08305AC
:1099A80001D51548EEE7BAF1000F03D001F076F9BA
:1099B800124803E040EA0800B060114804F03EF99C
:1099C80039461048BDE8F04701F04FB809F10109E0
:1099D800D3E700BF481C00202A5C0108983E010814
:1099E800345C010836640108385C01083D5C0108F4
:1099F800943E0108495C0108585C0108665C01084E
:109A08006F5C01087763010810B5084804F016F97F
:109A1800074B00241C715C63064B1C70FBF77AFF34
:109A280004F0F0FA044B1C6010BD00BF775C01081D
:109A380060180020F5260020A024002070B50646F6
:109A480000240B4BE518AA8816420AD0E1580948A9
:109A580001F00BF82846002104F07DF8064804F0D0
:109A6800EDF8143440F658439C42EAD170BD00BF6B
:109A780040470108A35C010836640108F0B5047882
:109A88008BB005460CB1002436E04B4B19680E2309
:109A980003FB041101F58C70B1F91D51B1F91921BD
:109AA800B1F91B31009591F82051019591F8215198
:109AB800029590F90700039001F590713F4891F9DC
:109AC800021004912146013400F0CFFF082CDCD1AC
:109AD80070E02D2B14D1072C1BDC284608F040FF22
:109AE8000AAB661C03EB440424F8100C15F8013F7C
:109AF800303B092BFAD934462B78002BE9D104E006
:109B0800A3F13002092A09D8E5E7082CBDF8182086
:109B180009D00BB0BDE8F040FDF748BA202BF8D1CA
:109B280001352646E7E7072AF3D8BDF81A00224B85
:109B3800A0F2EE2189B240F2DC55A9421B68E8D8B0
:109B4800BDF81C10A1F2EE24A4B2AC42E1D8BDF8D5
:109B58001E6004B237B2A742DBDB0DB2AF42D8DCDD
:109B6800A542D6DBBDF8247007F16404A4B2C82C62
:109B7800CFD8BDF826E00FFA8EF4112CC9DCBDF859
:109B88002050B42DC5D8BDF82240B42CC1D812B28B
:109B98004FF00E0C0CFB0233A3F81901A3F81B11AC
:109BA800A3F81D6183F8205183F8214183F81F71C0
:109BB80083F822E10BB0F0BDE8100020AD5C01088D
:109BC8002DE9F041047806467CB9334DB5F8C42137
:109BD800B5F8C63131482146013400F046FF042C5F
:109BE80005F10405F2D1BDE8F0812D4908F026FE03
:109BF800B0B9294B4FF47A714FF4FA62A3F8C41143
:109C0800A3F8C621A3F8C811A3F8CA21A3F8CC1158
:109C1800A3F8CE21A3F8D011A3F8D221BDE8F08192
:109C2800304608F09DFE032805462DD830462021F1
:109C380008F031FE044630B10134204608F090FEA9
:109C48000126074600E006462046202108F023FEAC
:109C580018B9BDE8F041FDF7A9B9013008F080FE58
:109C6800012EF6D1A7F2EE2240F2DC539A42F0D848
:109C7800A0F2EE229A42ECD8074B703503EB85032D
:109C88009F80D880BDE8F081064807490022032359
:109C9800BDE8F04100F0E9BE481C0020CD5C010899
:109CA800E05C0108B55A01083C6601082DE9F0415D
:109CB8002DED048BAB498AB0044608F0BFFDAA49D4
:109CC800002820460CBF0126072608F0B7FDA74943
:109CD8000028204608BF022608F0B0FD002808BF6B
:109CE8000426F10740F1E380A148A24C03F0A6FF47
:109CF800002003F0ADFDA04803F0A0FF9F4803F04B
:109D08009DFF63799E4A9F48013B254652F82310E0
:109D180000F0ABFE9C4800F0A8FE4FF00008274674
:109D280095ED048AB5EE408AF1EE10FA04D1974811
:109D380000F09BFE002570E09548D5ED059A95ED5D
:109D4800069AD5ED078A414600F08FFEB5EEC08A27
:109D5800F1EE10FA02D5202003F068FFB0EE480AB1
:109D680006A800F017FD01468A4800F07EFEF5EED1
:109D7800C09AF1EE10FA02D5202003F057FFB0EE9A
:109D8800690A06A800F006FD0146824800F06DFE4B
:109D9800B5EEC09AF1EE10FA02D5202003F046FF86
:109DA800B0EE490A06A800F0F5FC0146794800F033
:109DB8005CFEF5EEC08AF1EE10FA02D5202003F021
:109DC80035FFB0EE680A06A800F0E4FC08F10108C7
:109DD8000146714800F049FEB8F10C0F05F1100575
:109DE8009ED1A4E749B294F8D02094F8D1300091DC
:109DF80094F8D310019194F9D410029194F9D510E4
:109E0800039194F8D610049164482946013500F06E
:109E18002CFE102D04F1070403D094F8D210002969
:109E2800E0D15F485F4C03F009FFD7F8088054F889
:109E3800041F19B15C4800F018FEF8E70D465B4BAB
:109E480053F8254054B10123AB4013EA080F03D05F
:109E58005748214600F009FE0135F0E7554803F060
:109E6800EDFE21467B180AAA93F888311344524A1A
:109E78008A5C03F8102C01310829F3D1002306A9C4
:109E88004E488DF8203000F0F0FD4D4803F0D6FE26
:109E98004C48FDF75DFB4C4800F0E7FD4020FFF71C
:109EA800CDFD4A4803F0CAFE4648FDF737F9B20728
:109EB80039D5474803F0C2FE464803F0BFFE414883
:109EC80003F006FD444803F0B9FE3E48FCF7F5FFF1
:109ED800424803F0B3FE3B48FDF76EF8404800F0F7
:109EE800C4FD3848FFF76CFE3E4803F0A7FE35482E
:109EF800FFF7C4FD00270E257D4300243A4A926BE4
:109F08002A440123D2F80A20A34013421ED1013467
:109F18000E2CF3D10137082FEDD12B4800F0A5FD09
:109F28008020FFF78BFD730716D5304803F086FEB7
:109F38002F4803F083FE234803F0A4FC224800F0D6
:109F480094FD4FF48070FFF779FD05E0394622460D
:109F5800284800F08AFDDAE70AB0BDEC048BBDE8BA
:109F6800F08100BFE65C010846610108ED5C01086C
:109F7800F35C0108481C0020015D0108135D01081D
:109F8800985301081F5D01082A5D0108375D010823
:109F9800445D0108215C0108786301085C5D0108E3
:109FA8004C5D0108943E01087B5D0108983E01085C
:109FB800895D0108965D0108DE620108A25D01085D
:109FC800AB5D01084459010836640108BA5D01080F
:109FD800C75D0108DA5D0108E85D0108F25D010866
:109FE800015E01080F5E0108601800201B5E010871
:109FF8002C5E01083E5E0108F0B504468FB020468D
:10A0080008F057FCC5B225BBAF48B04C03F016FEAC
:10A0180094F8D21009B9AE4854E049B294F8D02067
:10A0280094F8D130009194F8D310019194F9D41098
:10A03800029194F9D510039194F8D6100491A5488B
:10A048002946013500F011FD102D04F10704DFD178
:10A05800E1E72046A049052208F034FC0546B8B9D6
:10A0680029469E48702208F0E0FB9D4B1968284657
:10A078000E2303FB001301300022082883F8232154
:10A0880083F8242183F8252183F82621F0D119E1CA
:10A0980020469449042208F015FC05462046002D68
:10A0A8004AD1202108F0F7FB002800F00B81461C5C
:10A0B800304608F0FEFB2C4607468B4B53F82450DD
:10A0C8002DB98A480FB0BDE8F04000F0CEBC30464C
:10A0D8002946FAB208F0F6FB01340028EDD17B4A94
:10A0E80002F170011646002382F8D63082F8D23089
:10A0F80082F8D13082F8D03007328A42F3D17C49D5
:10A1080001EBC40191F8E821934210DAD1F8EC711F
:10A11800C3EBC302B0183A4400F1D0011768C0F885
:10A12800D0709088888092798A710133E7E7294650
:10A13800704800F09AFC96E06F49072208F0C2FBCD
:10A1480005462046002D4AD1202108F0A4FB0646EA
:10A1580008F0AFFBC4B274BB684800F086FC214627
:10A168006748013400F081FC0E2CF8D1584800F003
:10A178007CFC00246348214600F077FC0025584AFF
:10A18800614811680E2202FB04120123D2F8232130
:10A198005E49AB4013425E4B05F1010508BF194605
:10A1A80000F063FC0E2DEAD14948013400F05DFC53
:10A1B800082CDFD186E03046564908F0D5FB2C46FE
:10A1C800002852D0022C55D008F0CAFB06AB5149E2
:10A1D80043F82400002008F0C7FB0134F0E74D499C
:10A1E80008F0C2FB002460B1082C3ED008F0B8FB90
:10A1F80006AB484943F82400002008F0B5FB0134B9
:10A20800F1E7082C31D1069B0F2B2ED8DDF81CE086
:10A21800BEF1070F29D8089F0D2F26D8099E06F1F1
:10A228006402C82A21D80A9DFF2D1ED80B986428DD
:10A238001BD80C99642918D8884216DA0D9C032C6F
:10A2480013D8224AC3EBC303134483F8D0E083F83E
:10A25800D17083F8D26083F8D35083F8D40083F8A0
:10A26800D51083F8D6402C4CC9E60FB0BDE8F040B5
:10A27800FCF79CBE069B072B20D807990D291DD8F3
:10A288000278722A0DD06E2A18D1154A12680E204B
:10A2980000FB032301228A40D3F8231121EA02029A
:10A2A80009E00F4A12680E2000FB032301228A40AE
:10A2B800D3F823110A43C3F8232101E0FCF776FE03
:10A2C8000D4C9CE60FB0F0BD5D5E0108481C0020F7
:10A2D80036640108885E0108E05C0108181D00204A
:10A2E800E8100020A45E010898530108495C0108A1
:10A2F800083D0108A95E0108555E0108225C0108B5
:10A30800B55E010890630108BA5E01086F6701082D
:10A3180029680108BE5E0108445901082DE9FF417A
:10A3280004780546002C39D17348744D03F086FC37
:10A33800D5ED047AF5EE407AF1EE10FA00F0D98006
:10A3480021466F4800F091FB95ED040A684600F03D
:10A3580021FA01466B4800F088FB95ED050A68462E
:10A3680000F018FA0146674800F07FFB95ED060AF1
:10A37800684600F00FFA0146624800F076FB95ED5A
:10A38800070A684600F006FA013401465E4800F004
:10A398006CFB0C2C05F11005CAD1AAE05B4905221B
:10A3A80008F090FA40B9554B03F1C002002143F878
:10A3B800101F9342FAD19CE028465549042208F020
:10A3C80081FA04462846002C40D1202108F063FA7F
:10A3D800002800F08E80451C284608F06AFA0746D7
:10A3E8004C4B53F824601EB94B4803F027FC80E01F
:10A3F80028463146FAB208F065FA01340028EFD150
:10A408003E4B03F1C0029E46002143F8101F9342C1
:10A41800FAD1424B03EBC4029846D2F804C0BCF10F
:10A42800000F04D131463E4800F01FFB57E00027DB
:10A4380018F834309F42F5DA3B010EEB030563440C
:10A448000FCB103585E80F000137F1E708F088FADF
:10A458000B28064647DC2846202108F01CFA05464A
:10A4680050B10135284600F00BF9244B03EB0613D5
:10A4780083ED040A012400E004462846202108F060
:10A488000AFA054648B10135284600F0F9F81B4B91
:10A4980003EB061383ED050A01342846202108F052
:10A4A800FAF9054648B10135284600F0E9F8134B9A
:10A4B80003EB061383ED060A01342846202108F031
:10A4C800EAF910B9FCF772FD13E0013000F0D8F892
:10A4D8000A4B032C03EB061686ED070AF2D1114846
:10A4E800FFF71CFF05E01048104901220C2300F07B
:10A4F800BCFA04B0BDE8F081C05E0108481C002029
:10A50800DB5E0108E15E010878630108E05C010890
:10A51800A45E010898530108495C0108485B0108DA
:10A52800A95E010844590108B55A0108D45A01081E
:10A53800F0B50124B0FBF4F58D4201D34C43F9E7A3
:10A548000026D4B1B0FBF4F504FB1500B4FBF1F41C
:10A558001EB9002D01DC002CF3D1092D03F1010EE9
:10A56800EFB204DD002A14BF3725572500E0302557
:10A578003D441D7001367346E3E71C70F0BDF0B52D
:10A588000124B0FBF4F58D4201D34C43F9E70026D2
:10A59800D4B1B0FBF4F504FB1500B4FBF1F41EB91B
:10A5A800002D01DC002CF3D1092D03F1010EEFB2CF
:10A5B80004DD002A14BF3725572500E030253D4427
:10A5C8001D7001367346E3E71C70F0BD2DE9F843B2
:10A5D800089E002B07468846144614BF4FF03009E2
:10A5E8004FF02009334613F8012B0AB9254603E03A
:10A5F800002CFBDD013CF6E7002D04DD384649461A
:10A60800C047013DF8E724EAE4743546A01B284416
:10A6180015F8011B11B13846C047F7E7BDE8F883C4
:10A62800014B1868FAF7E8BF8810002090ED017A0E
:10A6380007EE901AB5EE407AF1EE10FA01BFF8EE87
:10A64800E77A9FED0E7A67EE877AB7EE007A04BF55
:10A65800C7EE277AC0ED017A90ED017AD0ED007A45
:10A6680030EE877A30EE670AC0EE870AE0EE807A2D
:10A67800B0EE670AC0ED007A704700BFDB0FC94033
:10A6880010B50278202A034600F10100F9D0092A02
:10A69800F7D02D2A03D10346BFEE000A04E02B2A87
:10A6A80008BF0346B7EE000ADFED387A1A461346AC
:10A6B80012F8010BA0F13001CCB2092C0AD807EE30
:10A6C800101AB8EEC77AF2EE046AA7EEA67AF0EE90
:10A6D800477AECE72E2816D1F2EE046A1146B0EE5E
:10A6E800666A0B4611F8012B303AD0B209280AD80D
:10A6F80007EE102AB8EEC77A87EE267A66EE866AE3
:10A7080077EE877AEDE71A7802F0DF02452A35D12D
:10A718005A782D2A02D10233012004E02B2A14BFD3
:10A72800013302330020013B002213F8011F3039A6
:10A73800CCB2092C03D80A2404FB0212F5E7B2F5BF
:10A748009A7F28BF4FF49A721346B7EE007A072B08
:10A7580005D9DFED0F6A083B27EE267AF7E702F006
:10A7680007032BB1F2EE046A27EE267A013BF8E7DD
:10A77800F0EE476A20B1C7EE877A03E0F7EE006A89
:10A7880067EEA67A20EE270A10BD00BF0000000081
:10A7980020BCBE4C30B52DED028B87B0B0EE408AA0
:10A7A8000C220021054603A808F03FF8B5EEC08A40
:10A7B800DFED2A7AF1EE10FACCBF38EE278A38EEB0
:10A7C800678ADFED277A28EE278A6946FDEEC87A80
:10A7D80017EE904A84EAE470A0EBE47002F0F4FA11
:10A7E800002CACBF20232D2368468DF80C3008F0D0
:10A7F80060F8012807D130238DF80D308DF80E3020
:10A808008DF80F300CE0022805D130238DF80D307B
:10A818008DF80E3004E0032804BF30238DF80D3086
:10A82800694603A808F028F803A808F042F8033896
:10A83800C4B2224603A9284608F068F800232B551D
:10A848002846084908F018F803AB2846191908F0F3
:10A8580013F8284607B0BDEC028B30BD6F12033ADF
:10A8680000007A44B762010870B5064615460846E6
:10A87800B6FBF2F414B12046FFF7F6FF05FB1464AB
:10A88800024B1B5D00F8013B70BD00BFB9620108B7
:10A898002DE9F04F814689B08A4616461C460025A8
:10A8A8003178002900F0DD80252902D0013648469C
:10A8B80075E07278302A08BFB278A2F1300319BF68
:10A8C800B71C4FF0000BF71C4FF0010B092B4FF092
:10A8D800000819D8A2F13003D9B2092905D80A22EB
:10A8E80002FB083817F8012BF4E7A2F16103052BE6
:10A8F80002D8A2F1570305E0A2F14103052B03D8C2
:10A90800A2F137030A2BEADD6C2A31D13A78642A9E
:10A9180007F1010600F083800BD8252A3DD003D823
:10A92800002A00F09E80BBE7582A0CD0632A19D071
:10A93800B6E7732A22D002D86E2A37D0B0E7752A34
:10A948005CD0782AACD1271D2068A2F15804624255
:10A958004FF01001624155E02CD9582A32D0632AB1
:10A968002AD13E4648462178271DD04701350FE0B9
:10A97800642A64D00ED9732A14D13E462368009302
:10A988004846514642460023FFF720FE271D05444E
:10A998003C4685E7252ADFD13E4648462521D04753
:10A9A80001357DE70AD86E2A06D13E46236804346D
:10A9B8001D6075E7002A54D03E4671E7752A26D0F7
:10A9C800782AF9D1A2F1580304F1040C5A422068FC
:10A9D800CDF80CC04FF010015A4105ABFFF7A8FDA8
:10A9E800DDF80CC03E46644605AB00934846514628
:10A9F80042465B46FFF7EAFD054451E72068271DFC
:10AA08000A21002205ABFFF7BAFD3C46ECE704F14A
:10AA1800040CCDF80CC020680A210022DDE720686C
:10AA2800002804F1040708DA2D238DF81430404279
:10AA38000DF115030A210022E5E705ABFAE72068C6
:10AA4800002804F1040C0ADA2D238DF81430404252
:10AA58000DF11503CDF80CC00A210022BEE705ABA5
:10AA6800F8E7284609B0BDE8F08F0FB413B50B49D5
:10AA780004AB08680A4953F8042B09680193FFF7E7
:10AA880007FF0446074B1868FAF7AAFD0028F9D013
:10AA9800204602B0BDE8104004B070473C080020D2
:10AAA8003808002088100020B0EEE06AF0EEC05AA6
:10AAB800B4EEE56AF1EE10FAD4BFF0EE656AF0EE96
:10AAC800466AF5EE406AF1EE10FA0BD0B4EEE56A8C
:10AAD800F1EE10FA54BFF0EE657AF0EE467AC7EE62
:10AAE800A66A01E0DFED1F6ADFED1F7A9FED1F7A8E
:10AAF8009FED1F5AA6EEA77ADFED1E7AE7EE267ABB
:10AB08009FED1D7AA7EEA67ADFED1C7AE7EE267A8E
:10AB1800F4EEC65AB1EE677ADFED197AA6EEA75AB7
:10AB2800F7EE007AE5EE267AF1EE10FAC7EE277A0C
:10AB3800C8BF9FED147AF5EEC00AC8BF77EE677AF2
:10AB4800F1EE10FA48BF9FED107AB5EEC00A48BF83
:10AB580077EE677AF1EE10FA48BFF1EE677AB0EE59
:10AB6800670A70470000000039094E3DE3B59EBEF4
:10AB780069A2163E88FA16BE45FE7FBFA7DFA8B4B5
:10AB880099FB243FDB0FC93FDB0F4940FDEEC07A3C
:10AB980017EE903A2033402B43D8DFED237AB4EEFA
:10ABA800E70AF1EE10FA04DDDFED207A30EE670AED
:10ABB800F3E7DFED1F7AB4EEE70AF1EE10FA04D5F9
:10ABC800DFED1A7A30EE270AF3E7DFED1A7AB4EEF2
:10ABD800E70AF1EE10FA04DD30EE670A37EEC00A34
:10ABE8000AE09FED157AB4EEC70AF1EE10FA44BFF9
:10ABF80030EE270A37EE400A60EE007ADFED0F6A82
:10AC08009FED0F7AA7EEA67ADFED0E6AE7EE876A68
:10AC18009FED0D7AA7EEA67A20EE276AA6EE070A20
:10AC280070479FED060A7047DB0F4940DB0FC940AC
:10AC3800DB0F49C0DB0FC93FDB0FC9BF00000000B5
:10AC480092E741B99730083C15A82ABEDFED027A91
:10AC580030EE270A9AE700BFDB0FC93F064B1A8878
:10AC680022EA0000904210B518801C4602D001204C
:10AC7800FCF75CFE208810BDA8100020064B1A883F
:10AC88001043904210B518801C4602D00120FCF7F2
:10AC98004DFE208810BD00BFA8100020024A93680E
:10ACA80023EA000090607047481C002008B5104B4C
:10ACB8001A780023D9B2914207D20E4951F82310CD
:10ACC8000968002008600133F4E73220FAF769FCCC
:10ACD800094B1B685A0309D5084B9B685B0305D4CD
:10ACE80040F2DC50BDE80840FAF75BBC08BD00BF85
:10ACF800C011002090110020781B0020481C002063
:10AD08002DE9F34104F04CFB454A6C2313704FF4D2
:10AD1800E3635380BE231371EF2382F814370023B3
:10AD280082F8153719461646F25C0133B3F5E36F1E
:10AD380081EA0201F8D13A4B83F81517394B1A69A1
:10AD4800120604D5384A5A6002F188325A6004273C
:10AD58000020013F17F0FF074FD0324B3422DA6052
:10AD6800002444B1002356F80480019301F0FCFF4D
:10AD78000428EED117E001F0F7FF0428E9D1294DA6
:10AD88002B6943F002032B61284B6B612B6943F05D
:10AD980040032B6101F0E8FF2B69042823F002032C
:10ADA8002B61DFD0D5E71F4D2B6943F001032B61E1
:10ADB80004F1006303F57E331FFA88F21A8001F06C
:10ADC800D3FF042810D11A4B23440193019B4FEA67
:10ADD8001848A3F8008001F0C7FF2B69042823F066
:10ADE80001032B6105D0B4E72B6923F001032B6124
:10ADF800AFE70434B4F5E36FB3D10A4A1369042802
:10AE080043F08003136102D103F02EF910B9052035
:10AE1800FCF7A4FD04F0B0FA02B0BDE8F08100BF71
:10AE2800481C0020002002402301674500F8030861
:10AE380002F8030810B50E4C2068FCF7A7FC206840
:10AE4800047A002202FB02F3193B634303F6C4139E
:10AE58005343192193FBF1F3064921F812300132CB
:10AE6800072AEFD10449BDE81040FCF745BC00BFF4
:10AE78001411002058100020881D00202DE9F041F1
:10AE880003F0F2F810B90420FCF768FDAB4CAC4DA8
:10AE980004F086FAAB494FF4E362204607F0BAFCA7
:10AEA80094F8E436022B84BF002384F8E43694F83F
:10AEB800E4264FF4CC7101FB02F3E018234400F5BB
:10AEC8000770286093F8700203F51A73022801FBD3
:10AED800024284BF0020187292F870329A4A1370A6
:10AEE8000C2202FB0343994A03F2E6631360A3684A
:10AEF80046F209021A401AB9904A43F40053936083
:10AF0800A368D80703D54FF40050FFF7C7FEA3681E
:10AF1800590409D50820FFF7C1FE4FF40050FFF788
:10AF2800BDFE0120FFF7BAFEA3681A0706D54FF445
:10AF38000050FFF7B3FE0120FFF7B0FEA3689B04A3
:10AF480002D54020FFF7AAFE012284F80D2294F8CA
:10AF5800DE217A4B2AB193F8E22112B1002283F85C
:10AF6800E2217B4B7B4E1E604FF0000C674604EBE2
:10AF78000C03B3F8F6E14FEA5E0101F077314FEACE
:10AF88009E0303F03333C1EB0E00C11A4FEADE0310
:10AF980003F01133CB1A03EB23131EF0010803F05F
:10AFA8000F324FF0FF0392FBF3F3C3EB032318BFF9
:10AFB8000137A2EB030318BFFFB2012B0ADD022BF6
:10AFC80040F0B980B8F1000F00F0B5801EF0BC0F5A
:10AFD80000F0B1800CF1080CBCF1180FC7D1013F8B
:10AFE800012F00F2A880FFF725FF302200215A48E0
:10AFF8005A4F07F01AFC5A4BD5F800801F60594B7E
:10B00800002108F17900C3F80080FCF7FFFB564BDC
:10B0180080F001001870554B07F128021A60544B54
:10B0280007F1CC021A6098F80000FBF741F928688C
:10B03800504B00F5C5721A6000F0CAFC4E4B94F8EC
:10B04800D601DFED4E6A07F196021A6064214C4B77
:10B05800C82211FB00225A6000229A60DA601A6145
:10B068005A619A61DA6183F8202083F82120454BE0
:10B0780007F12E021A602A68434B92ED187A02F201
:10B0880019111960414B02F289111960404B07F1FF
:10B09800080119603F4B1F603F4B07F1A20119607F
:10B0A80067EE266A3D4B07F1AC01B6EE007A1960EF
:10B0B80087EE267A3A490E60B4F86411181D07EE37
:10B0C800901AB4F86611F8EE677AC3ED027A07EEC3
:10B0D800901A92F85C10197192F87810597194F8D6
:10B0E800E1111974F8EE677AB2F81611C3ED037A14
:10B0F80007EE901A2B49F8EEE77A08605A6183ED5B
:10B10800077A9FED297A1A62C7EE277A02F164015D
:10B1180099612649DF62BDE8F0419FED257A67EE27
:10B12800877AC1ED007A02F1680102F211125962C0
:10B138009A6204F021B901F0E3FD54E7481C0020AD
:10B14800E810002000F803087C24002014110020D7
:10B1580074260020D01D0020980A0020881D002099
:10B16800CC0A0020D00A002002000020741300201E
:10B17800D4090020D80A002070260020DB0F49409F
:10B18800A4260020DC130020981800203803002093
:10B19800DC120020E01200204C0200209C18002045
:10B1A80010030020541400200000614448020020CD
:10B1B8004C3D0F4408B5FFF7A3FDFFF75FFE0120E4
:10B1C800BDE80840FCF7B2BB07EE900AF8EEE77A54
:10B1D800DFED0C6A9FED0C0AF5EEC07AF1EE10FA7D
:10B1E800D4BFB1EE677AC7EEA67A08B5D8BFC7EE66
:10B1F800267A27EE800AFFF729FD044B83ED000A23
:10B2080008BD00BF8096184B35FA8E3C68000020B8
:10B218002DE9F0410369C76805460E461F40002F17
:10B2280035D0B7FA87F24FF00043D340DB432B61A8
:10B238001F40A2F11B03042BF1D8DFE803F0221F03
:10B248001C190300746A24B1013C0023A4B2736280
:10B2580001E0EC6AA4B2D6F82080B8F1000FDED085
:10B26800D8F80030404621469847D8F80480F4E7DB
:10B278003068696B07E07068A96B04E0B068E96B37
:10B2880001E0F068296C036889B29847C7E7BDE810
:10B29800F081F8B5994B1B680546187818B1012854
:10B2A80000F06181D9E2242D954C0CD006D80A2DE6
:10B2B80000F0D7800D2D00F0D4803FE12A2D06D074
:10B2C8002C2D04D03AE120706070A07047E18D4BBE
:10B2D800617827788A4A002058542FBB1978D7708C
:10B2E800472921D1597850291ED19978472907D162
:10B2F800D978472904D11979412901D10121D1707F
:10B308009978804A522903D1D1784D2900F0A78233
:10B3180099787C4A472907D1D178532904D11279E1
:10B32800562A04BF0322E270E278754E022A38D00A
:10B33800032A4BD0012A40F08380BA1E072A7FD8FF
:10B34800DFE802F004080F131A257E2A01F0F4FB47
:10B35800606075E01B78532B72D163685B42636051
:10B368006EE001F0E9FBA0606AE01B78572B67D11B
:10B37800A3685B42A36063E01B78302B624B1A78AA
:10B388008CBF42F0020222F002021A7058E000203C
:10B3980001F032FC207353E0002001F02DFCE08125
:10B3A8004EE0072F06D0082F4AD1012001F024FCD7
:10B3B800708245E0012001F01FFC41F21843584318
:10B3C8004FF47A73B0FBF3F0308239E0022F07D0E4
:10B3D800032F0AD1002001F00FFC4C4B18702FE00E
:10B3E800002001F009FC30752AE029D93A1F921093
:10B3F800337D0132D2B2013B02EB8303DBB2102B67
:10B408001ED8F91EC2F1010201EB8202D2B2012A52
:10B418000BD0042A11D100205E1E01F0EDFB3C4B3D
:10B4280098553C4B00229A5507E05E1E3A4A002088
:10B43800935501F0E1FB394B9855A3690133A3619A
:10B448002F4B2A2D18BF9A7807F101074FF00000FB
:10B458000CBF01225540277060700CBF1A779D7091
:10B468007DE0207F002846D02D4B13F8012D2D4973
:10B478005A708B42F9D1234A214D13785278402BC8
:10B4880085BF373B1B011B01DBB298BF03F0F003FC
:10B49800402A8CBF373A303AD2B21344A278DBB292
:10B4A8009A4225D121230B70E8782B6A1D4A013373
:10B4B80001282B620AD002281CD1722313701A4B60
:10B4C8002A8A1A80194B6A8A1A8013E06723137034
:10B4D8000D4B1B789F070ED5154B6A681A60AA6832
:10B4E8005A60144B2A7B1A70134BEA891A8002E0BF
:10B4F8003F230B7000200023237730E09C010020BD
:10B50800CC180020A01B0020181100204411002096
:10B5180075110020651100204511002055110020EB
:10B52800D0090020BC090020261100202811002085
:10B538001C11002019110020241100206378207F9D
:10B548000E2B9FBFAA4A591C5170AA4A98BFD554BE
:10B55800A74A18B993785D40957000E00020003044
:10B5680018BF0120F8BDA24B93F824100022082927
:10B5780000F27381DFE801F0050C101A2B3B5F7BAA
:10B588008800B52D40F0698183F8252001224FE01D
:10B59800622D08BF02224BE0032283F8242083F89F
:10B5A800265083F8275083F8285056E1042283F860
:10B5B800242093F8272093F8281083F829502A4448
:10B5C800D2B283F827200A4483F8282045E10522CF
:10B5D80083F8242093F8272093F828105D852A44BF
:10B5E800D2B283F827200A4483F8282035E10622BE
:10B5F80083F8242093F8272093F828102A44D2B2FD
:10B6080083F827200A4483F828205A8D02EB052561
:10B61800ADB2B5F5AC7F88BF754A5D8584BF0121A1
:10B6280082F8251000229A85002D40F01681072205
:10B6380083F8242011E193F8272093F828102A444E
:10B64800D2B283F827200A4483F828209A8DB2F5CD
:10B65800AC7F3CBF6649891802F1010238BF81F806
:10B668003050598D92B291429A85E0D9F5E008227E
:10B6780083F8242093F82730AB4200F0EE805C4B2F
:10B68800012283F825200FE05B4C83F8242014F86E
:10B69800012D6270594A9442F9D193F82810544AFE
:10B6A800A94206D03F232370554A5368013353609B
:10B6B800D3E0116A92F825000131116210B13E23DE
:10B6C8002370CAE02121217092F82910062941D05F
:10B6D80004D8022907D0032923D0F8BD122959D04C
:10B6E800302967D0F8BD502121704649546B4C6011
:10B6F800946B0C60116C4FF47A7491FBF4F1424C2A
:10B70800218092F88811414A19B1117841F002015B
:10B7180002E0117821F002011170012283F88921D9
:10B728008DE05321217092F83510CE0705D592F897
:10B738003420D51E6A426A4100E0024602F0010147
:10B7480083F88811002A7AD130490A7822F0020257
:10B758000A7074E04F21217092F83B10CC0705D590
:10B7680092F83A20D11E4A424A4100E0024602F0CD
:10B77800010183F8881122B924490A7822F00202CB
:10B788000A70234A93F85F101170224AB3F85C10CC
:10B79800118054E0562121701F49546C0C8042F2EC
:10B7A8001074916C91FBF4F11C4C2180012182F8FA
:10B7B8008A1144E04921217092F83410184A10295E
:10B7C80088BF10211170174914780022A24233D281
:10B7D800154D0E7A5655154D4E7A5655144DCE7A4E
:10B7E8005655144D11F80C6F56550132EEE700BF4F
:10B7F800CC180020A01B0020D0090020BC09002084
:10B808007C0100201C1100202411002018110020A8
:10B8180019110020EC00002026110020281100201A
:10B8280044110020FC18002045110020551100206B
:10B8380065110020751100209A6901329A6193F808
:10B8480089310B4A93B192F88A317BB1002182F891
:10B85800891182F88A111846F8BD0020F8BD1279BE
:10B86800432A7FF455AD0222E27051E5F8BD00BFCE
:10B87800CC1800200449054B0968187000225A6149
:10B8880099611A77704700BF181B00207C010020BF
:10B8980010B5121A07EE902A5B1A2DED028BF8EEFE
:10B8A800E78A07EE903A184B059CB8EEE78AD3ED85
:10B8B800007A28EE278A28EE080AA8EEA80A07F0D8
:10B8C8009BFADFED127A049B20EE270AF0EE480A75
:10B8D800BCEEC00A83ED000AB1EE680AFFF7E4F88F
:10B8E800DFED0B7A9FED0B7AE0EE077ABDEC028B69
:10B8F800FDEEE77A17EE903A002BBCBF03F50C4338
:10B90800A033236010BD00BF680000202C7D8E3F4F
:10B9180000A00C46A00CB34544F25063984203DDE6
:10B92800A0F50C40A0387047034B9842BCBF00F507
:10B938000C40A030704700BFB0B9FFFF73B51A4C78
:10B94800036823600B686360184D0068184EFFF7A2
:10B958003BFC184B009395E8030094E80C00019613
:10B96800FFF796FF144B32681A60686863681349DA
:10B978001B1A07EE903A124B286893ED007A236859
:10B988001B1A0B600F4BF8EEE77A1A600E4B67EE46
:10B99800877A1B68FDEEE77ADA880C4BC1ED017AED
:10B9A8001A8002B070BD00BF1C2400201C110020AA
:10B9B8002824002024240020642400202C24002093
:10B9C800680000205C240020D80A002058240020A9
:10B9D8004279DFED2A5A2A4B9FED2A5A07EE902A20
:10B9E800F8EE677AC27BC7EEA57AB2EE047AC3EDA9
:10B9F800007A07EE902AF8EE677A234ADA60C7EEF3
:10BA0800A57AC3ED017A8179204B07EE901AF8EEFA
:10BA1800677A017CDA60C7EE877AC3ED007A07EEB1
:10BA2800901A817E06EE101AF8EE677AB8EE466A2A
:10BA3800C7EEA57A86EE056AC3ED017A83ED026A40
:10BA4800C179134B06EE901A417CDA60F8EE666A0B
:10BA5800C6EE876A07EE101AC17EC3ED006A07EECC
:10BA6800901AB8EE477AF8EE677A87EE257AC7EE2D
:10BA7800857A83ED017AC3ED027A70470000C842E7
:10BA88003424002000007A440000FA4444240020B2
:10BA98006824002010B50C4C23789B0713D50B4B5A
:10BAA8001B78042B0FD90A4A0A4B106852685A604F
:10BAB8001860FFF789FB084B1A88084B1A8023780F
:10BAC80043F00103237010BD181100201911002044
:10BAD8001C110020301100200411002078240020BF
:10BAE8001C4B1B681B0307B530D51B4A1B4BD2EDFB
:10BAF800007A1B788DF80030B2EE047A67EE877A08
:10BB0800174B9FED187A1B788DF80130FCEEE77A19
:10BB18000A2017EE903AD2ED017A8DF8023067EEDE
:10BB2800877A6946FCEEE77A17EE903AD2ED027A08
:10BB38008DF80330FCEEE77A17EE903A8DF8043072
:10BB4800094B1B788DF80530FAF786FD03B05DF8D0
:10BB580004FB00BF781B00208C1B0020691B002001
:10BB6800881B002000007A446D1B0020054A1378CA
:10BB780083F001031370044A00231360034A13601F
:10BB8800AEE700BF6D1B0020841B0020801B002037
:10BB980001480249FFF73CBB00480140B4120020AD
:10BBA80001480249FFF734BB0040014064120020FD
:10BBB80001480249FFF72CBB000800403C12002056
:10BBC80001480249FFF724BB00040040141200207A
:10BBD8004FF080400149FFF71BBB00BFEC1100206C
:10BBE80010B5064C06482146FFF712FB04F1C801C0
:10BBF8000448BDE81040FFF70BBB00BFC41100208C
:10BC0800002C01400044014001480249FFF700BBF5
:10BC1800002C0140C4110020224B10B5224C5A437D
:10BC2800224BB3FBF2F203880139013AA04289B2F0
:10BC380092B29BB20ED004F50064A0420AD0B0F1D3
:10BC4800804F07D0A4F59834A04203D004F580644F
:10BC5800A04202D123F070039BB2154CA04206D03B
:10BC680004F58064A0421CBF23F440739BB2038098
:10BC78000D4BC162984202850FD003F500639842CC
:10BC88000BD003F54063984207D003F580639842D0
:10BC980003D003F58063984201D100230386012372
:10BCA800436110BD40420F00002C014000A24A042D
:10BCB80000100040134B800A984220D00AD84A3B13
:10BCC800984212D00133984211D0B0F5801F14D198
:10BCD800012070470C4B98420BD0013398420AD090
:10BCE800023B984209D10420704702207047032084
:10BCF80070470520704706207047FE2070470020D7
:10BD0800704700BF4B00100051001000F8B50468E0
:10BD1800064620460F461546FFF7CCFF06284BD8A7
:10BD2800B27A910847B902238B40D4F80CE0DB4380
:10BD38009BB203EA0E03E3600A23204A03FB0013C5
:10BD480042F82370043342F8235015463FB1B17AC4
:10BD5800E268890802238B409BB21343E3602822E0
:10BD680002FB00522032EFF31286502383F312882D
:10BD780003B203EB8303DB0003F10C011C332944FA
:10BD88002B4451F8047F17B117600A6804329942AE
:10BD9800F7D100231360F3B283F31188282303FB40
:10BDA8000050036A1BB1E36843F0010303E0E26853
:10BDB8004FF6FE731340E360F8BD00BFC4110020C6
:10BDC8000148F6F711BE00BF581A00200148F6F7DF
:10BDD8000BBE00BFAC1A0020704708B50B4B002003
:10BDE80093F82C10FDF728F9094B1B68187A0828D6
:10BDF80001BF084B4FF480521A80102208BF5A80A6
:10BE0800A0F109035842584108BD00BFA000002016
:10BE1800241B0020001B0020704770477047FEE776
:10BE2800FEE7FEE7704730B50024E3B293420DD237
:10BE3800030F092B94BF3033373301F8143001EB6B
:10BE48004403002500015D700134EEE730BD30B5D4
:10BE5800002202F1805303F5B8539B0042F40044DA
:10BE68001D6840F60F7144F08004294001322143D7
:10BE7800042A1960EDD1024B40F08000186030BDF3
:10BE88004C5C00402DE9F347884D894C2B68894E5E
:10BE98009BB2A380A28831880A40970507D54FF640
:10BEA800FF53854A2B6013780133DBB21370A388E4
:10BEB8000B40180440F100830023ADF802302B68D2
:10BEC8007B4F9AB21804A28040F1F682BB8803F037
:10BED8000F03BB71002B40F0C182784A13689BB2F4
:10BEE8003B803B8803F030037B803B8803F440535E
:10BEF8003B8011684BF6BF730B4083F4005383F00B
:10BF0800200343F4004343F080031360BB88D90641
:10BF180021D4116848F60F730B40694913600B6808
:10BF28001A7A022A884601D0042A02D1FDF710F8AD
:10BF38005AE2062A40F06B825A78052A08D11A7804
:10BF4800520605D1D878FFF782FFBB681B6A98476D
:10BF5800E3689B685AE213689BB2ADF80230BDF8FB
:10BF680002301F0540F1D0811168554F40F68F739C
:10BF78000B40544913600A68534B92B213445B0058
:10BF880088461A683B68187A092817D092B2520076
:10BF980002F1804202F5C042117819705178597047
:10BFA8009188C8B2090A41EA002159801189C8B2AA
:10BFB800090A41EA002199809289DA8001221A72DD
:10BFC800DA8893F80190002A40F0DC801A7812F0A1
:10BFD8007F024AD1B9F1090F0FD1DA78012A00F2AC
:10BFE800B8809978002940F0B4809988002940F0F9
:10BFF800B0809A72A3685B68A9E0B9F1050F10D107
:10C0080093F90320002A01DA0823B9E09A78002A74
:10C01800FAD19A88002AF7D19B7A002B00F0A280E7
:10C02800F2E7B9F1030F0ED1DA78012A40F09180D6
:10C038009A88002A40F08D805A7A42F020025A727B
:10C04800A368DB6983E0B9F1010F40F08280DA78F8
:10C05800012A7ED19A88002A7BD15B7A980678D506
:10C06800FDF70CF800287DD073E0012A2ED1B9F134
:10C078000B0F6ED1E26858799269D97890473B687E
:10C088009A7A002A65D0002863D11A79002A60D1EB
:10C098009B78002B5DD1064B9B68DB689847084B63
:10C0A8001B685A79DA72DA781A735BE0445C0040EC
:10C0B800001B0020CC240020F7260020005C004054
:10C0C800241B0020505C004004300020022A40D18C
:10C0D800B9F1010FC4D0B9F1030F3AD1587920F062
:10C0E800800E4FEA8E0202F1804101F5B84110F04E
:10C0F800800F096814BF01F0300101F44051BEF10E
:10C10800030F26D8B3F802E0BEF1000F21D101B326
:10C118009B7AF3B102F1804202F5B8420106136836
:10C128004BBF23F4E04323F4804323F0400323F080
:10C1380070034BBF9BB29BB283F0100383F4805310
:10C1480043F4004343F080031360A3689B69984756
:10C1580008E0E36848465B69984703280FD0002841
:10C168007FF452AFD8F80020A14B92B213445B0081
:10C178001A6800221A6030236380062300E009232E
:10C188003A6847E1B9F1060F12D11A78520678D108
:10C198009B78012B02D1E368DB6967E0022B02D1AF
:10C1A800E3681B6A62E0032B6BD1E3685B6A5DE0BE
:10C1B800B9F1000F38D15988002962D15A6822F4A0
:10C1C8007F42B2F5003F5CD11A7812F07F0204D1A9
:10C1D8009B88002B00F0D58153E0012A08D1E26842
:10C1E80058799269904700284BD13B689B7A17E0B1
:10C1F800022A46D15A7902F00F010BB29B0003F1D3
:10C20800804303F5B84312F0800F1B6814BF03F096
:10C21800300303F44053032933D812F0700F30D1A0
:10C22800002B40F0AE812CE0B9F1080F04D11B7847
:10C238005B0600F0A88124E0B9F10A0F21D11A7831
:10C2480002F07F02012A1CD19A7AD2B15988C1B969
:10C258005A6822F47F42B2F5803F12D1E2685879D9
:10C2680092699047002800F090810AE04BB13A6843
:10C278004FF00008A2F81280936140469847404664
:10C288000BE0E3683A681B6950789847032804D1A3
:10C29800584B1B6809221A72BDE03A68138A4FF698
:10C2A800FF718B4201D10923B4E0022800D00BB9F9
:10C2B8000823AFE092F9001000291FDAD188019114
:10C2C8000198834202D9019B138210E08B420ED25F
:10C2D800E16891F82C00834201D2002105E093FB2C
:10C2E800F0F100FB113313B90121434B1970E368D6
:10C2F80093F82C309382FCF72BFE8CE00323137207
:10C308004FF44053238086E0BDF802301BB2002B67
:10C31800BFF6D5AD116840F68F730B401360354AF0
:10C3280017683B7A022B904671D0042B6FD0032BF1
:10C3380001D0052B66D1BB693A8A8BB9398A0029A5
:10C348003BD04FF4405323802C4B1A68284B92B2B1
:10C3580013445B001A6800221A60302363802CE0C3
:10C36800002AEBD0B7F81490914528BF91461FFAE0
:10C3780089FA504698473B8ACAEB03033B827B8A7B
:10C3880053447B821D4B1A681D4B92B213445B00C9
:10C3980009F101021B689BB203F1005303F54053F6
:10C3A80052105B004FF0000E9645C7D053F82E1080
:10C3B80020F81E100EF1010EF6E7BB8A8B42D8F862
:10C3C800003001D8032201E011B105221A720BE0F6
:10C3D80006221A72094B1A68054B92B213445B0085
:10C3E8001A68196030236380D8F800301B7A0FE090
:10C3F80002300020241B0020F6260020505C00405C
:10C4080004300020072B02D1E368DB689847082333
:10C41800D8F800201372FFF7E0FC5E4B1A684BF661
:10C42800BF7313402288D704228848BF83F48053FF
:10C438009004628848BF83F40053D106628848BFDD
:10C4480083F01003920648BF83F0200343F40043AF
:10C4580043F080034F4A9BB213602DE09A0002F12B
:10C46800804202F5B842116889B2ADF80210BDF8F1
:10C47800021009B2002909DA106840F68F710140EC
:10C488001160013B444A52F823309847BDF8023006
:10C498001F067FF514ADA1798B0003F1804303F5E6
:10C4A800B84348F60F72186802401A603A4B03EB1B
:10C4B80081039B69984702E5A28833881340590590
:10C4C80005D54FF6FF332B60344B5B689847A2883D
:10C4D80031880A40920444BF4DF6FF732B60A3884D
:10C4E8002F4A0B40DB0452D54EF6FF732B60002316
:10C4F8001374137C052B41D8DFE803F0030D1418DF
:10C50800222D6369264D1BB900F0F0FC062300E0DC
:10C5180005232B743BE000F0E9FC0423237401237A
:10C52800636134E002236374032328E0637C013BE6
:10C53800DBB26374637C53BB194B04221A7426E084
:10C54800184A13689BB243F0100313600523237441
:10C558000A2363741BE0637C114A013BDBB26374FA
:10C56800637C03F0FF0093B90E490C684FF6EF7334
:10C5780023400B6006231374506108E006232374DC
:10C5880005E0094B73E6094B71E6094B6FE602B00B
:10C59800BDE8F087005C004040450108A00000208D
:10C5A800001B0020405C0040B18A0008698B00082D
:10C5B800458B0008012380F8453070472DE9F0418C
:10C5C80090F84440002380F84430002C4ED02C4989
:10C5D8000A68002A4DD00A68052A4DD12949202C1D
:10C5E800254628BF20256E1C0F6876104B688BBB2C
:10C5F800DFF89CE000F13203324613F8018C13F89F
:10C6080002CC013A4CEA082C2EF804CC03F10203C0
:10C618000EF1040EF1D11C4B1A681C4B92B2134454
:10C628005B002A46D3F800E01D604B68DFF864E041
:10C638002B444B60DEF8003023F4E04323F0400342
:10C648009BB283F0300343F4004343F08003CEF8F9
:10C65800003000E00022A24203D00B68DB1B312B24
:10C66800C4D9131B58425841BDE8F0810120BDE8E8
:10C67800F0811046BDE8F0811846BDE8F08100BFA2
:10C68800DC260020181B0020505C00400A300020E7
:10C6980084610040045C0040002280F845208DE75A
:10C6A80090F84420531C0244DBB280F8443082F8EE
:10C6B800301090F845200AB1132B00D97EE7704757
:10C6C800014B9868C0B27047181B002001207047C2
:10C6D8007047704720B9034BDB6808221A827047FD
:10C6E80001487047181B00205C000020F7B51C4B60
:10C6F8009A681D460AB99C6800E00124187C00214C
:10C70800CAB2A24201F1010107D202AE2F181644A3
:10C718003A44527C06F8042CF2E79A68121B9A6095
:10C728001A7C9D6822441A749DB903204021FCF7A5
:10C7380083FC0C4A136823F4804323F070039BB2F4
:10C7480083F4405343F4004343F080031360044BE5
:10C758001D74002CCBD09DF8040003B0F0BD00BFC1
:10C76800181B00200C5C00400C4B0D49DA6843781C
:10C77800D243C2F30222C2F10402934002781B01A1
:10C788000A44DBB282F8003303780122580903F027
:10C798001F0302FA03F341F82030704700ED00E070
:10C7A80000E100E073B50546002100680122FFF7AB
:10C7B80033FA2A6813889BB243F001031380EB7A9B
:10C7C8008DF804300124002601A88DF805408DF865
:10C7D80006608DF80740FFF7C7FFEB7A1B2B0BD1DC
:10C7E800192301A88DF804308DF805408DF80660EE
:10C7F8008DF80740FFF7B8FF02B070BDF0B5C64C22
:10C8080094F851302DED028B013B012B85B000F2DD
:10C818007E8194F85250854240F0798194F85330E3
:10C82800022B00F07481BD4B5B5D84F8543094F8A2
:10C8380055306D00F2EE048A1BB16319B3F9563016
:10C8480009E06319D4ED177AB3F95630F1EE677A37
:10C85800C4ED177A5B4208EE103A236EAE4EB8EE7E
:10C86800C88A1A0388EE288A35D5D6ED177AFDEEE0
:10C87800E77A28EE280A17EE903AD6ED197A8DF85D
:10C888000A30FDEEE77A17EE903A8DF80B3006F095
:10C8980021FAFCEEC07A96ED1A0A17EE903A20EECD
:10C8A800280AADF8083006F015FAFCEEC07A96EDC5
:10C8B8001B0A17EE903A20EE280AADF80C3006F065
:10C8C80009FAFCEEC07A0C2017EE903A02A9ADF8EE
:10C8D8000E30F9F7C1FED4ED1B7A8F4BF5EE407A96
:10C8E800F1EE10FA65D1D3ED1A7AB4EEE78AF1EEDB
:10C8F80010FA04DDDA6D83ED1A8A5A66F2E0F5EE75
:10C90800C07AF1EE10FA40F3ED8093F870204AB146
:10C91800022A00F2E7801A6883ED1B8AFA32C3F80C
:10C928008420DFE0D3ED177A38EE678AF7EE007AD5
:10C93800B4EEE78AF1EE10FAACBF01210021D3ED85
:10C948001E7A69B19FED767A27EE877ADFED757AE0
:10C95800B4EEE77AF1EE10FA58BFF0EE477A03E04A
:10C968009FED717A67EE877AC3ED1E7A236E6A4A65
:10C978001B0313D58DF8081092F85430D2F88010A4
:10C988000B440B205A788DF80920DA7A8DF80A20A2
:10C998005B7D8DF80B3002A9F9F75EFE0123D4F810
:10C9A800802084F8703094F8543013440022DA72EE
:10C9B80096E0B4EEE78AF1EE10FA48BF83ED1B8AE1
:10C9C800D4F88410236894ED1A7AD4ED1B6A591AA6
:10C9D800C943C90F77EE667A59B9B7EE006AF4EE23
:10C9E800C67AF1EE10FA7DDDB4EEE68AF1EE10FAC1
:10C9F80078DDD4ED196A484BB4EEE67AF1EE10FA18
:10CA0800CCBF0126002666B1D3ED1D7A9FED447A8E
:10CA180067EE877A9FED447AC3ED1D7AD3ED1F7ACE
:10CA28000AE0B0EE007AF4EEC77AF1EE10FA08DD0B
:10CA3800D3ED1F7A9FED3A7A67EE877AC3ED1F7AB6
:10CA480007E0D3ED1D7A9FED387A67EE877AC3ED5C
:10CA58001D7AD4ED1D7AD4F8800094F8542067EE3E
:10CA6800A87A1044FCEEE77ACDED017A9DF80430FF
:10CA78004370D4ED1F7A276EFCEEE77A3F03CDEDC5
:10CA8800017A9DF8042042750ED546EA41018DF8D9
:10CA980008108DF80930C37A8DF80A300B2002A9E6
:10CAA8008DF80B20F9F7D8FD94F870201A4B022A5C
:10CAB80013D1D3ED1E7A9FED1D7AD3F8801067EE5F
:10CAC800877A002283F87020FCEEE77A93F85420E6
:10CAD80017EE903A0A44D37202E0022283F87020DB
:10CAE800FFF744F894F855200B4B0AB1104A00E0C0
:10CAF800104ADA652544D4ED177AB5F9563000EEB8
:10CB0800103AB8EEC00A80EE280A37EEC00A05B01F
:10CB1800BDEC028BF0BD00BF181B00207C4501084E
:10CB2800EC51783F6F12833A0AD7833F00007A446A
:10CB38000000A0410000A0C12B4BF0B52B4D1E6892
:10CB480005F110002F78F3192C46597801F00401EB
:10CB5800013501F0FF0219B18542F3D10020F0BD83
:10CB6800224D631B022B0ADD1AB102EB820252002E
:10CB7800D2B215F8013B303B1A44D2B2F1E700219A
:10CB8800AC420AD919B101EB81014900C9B215F8C3
:10CB9800013B303B1944C9B2F2E72E2F16D10134BC
:10CBA800042000232578771903EB83037F785B0043
:10CBB8007F079BB244BF303D5B1900F1FF3044BF93
:10CBC80001349BB210F0FF00ECD100E000230848CC
:10CBD8004143642000FB03130620B3FBF0F3054830
:10CBE80000FB0230F0BD00BFFC000020A01B0020AD
:10CBF80040420F008096980030B500231A4610492D
:10CC08008C1894F88840BCB12E2C06D1013298B10A
:10CC18008C180444002584F8885011440A2491F89B
:10CC280088106343A1F13004092C9CBF303B5B188A
:10CC38000E2A03D80132E2E7184630BD002030BD85
:10CC4800181B002010B50446B0F9000001F08DFD56
:10CC5800B4F9020001F089FDB4F90400BDE8104000
:10CC680001F083BD10B50446006801F07EFD6068E0
:10CC780001F07BFDA068BDE8104001F076BD2DE90C
:10CC8800F74F0120FAF730FD002488B3012C2FD884
:10CC9800194E4FF04C0909FB04FA06EB0A0808F193
:10CCA800E007BD7815B10134E4B2EEE70179134B22
:10CCB80090F9002003EB810303218DE82200104640
:10CCC80001212A465B68FAF7E7FA834660B106F164
:10CCD8009800504429464A4605F0A7FD01231C4404
:10CCE800C8F898B0BB70E4B20120FAF7E1FCCCE7D1
:10CCF80003B0BDE8F08F00BF181B00207C45010879
:10CD080010B5184C00211A2204F2223005F08DFDCE
:10CD1800142384F8243305230022042184F82833BB
:10CD280084F82A3384F8303384F8323384F838337B
:10CD380084F83A335223012084F8291384F82B23EA
:10CD480084F8311384F8332384F8391384F83B23A7
:10CD580084F8223384F82C2384F83403A4F82603B7
:10CD680010BD00BF181B002010B5FCF791FA4FF456
:10CD78003024012806D11CB1FCF78AFA013CF8E7F7
:10CD8800052010BD002C08BF052010BD70B5064653
:10CD9800441E14F8011F89B1094D284605F07BFD92
:10CDA8000028F6D005F1080398423FBF054B401B09
:10CDB800C018A31B38BF80F8B832EAE770BD00BFBF
:10CDC800DE620108181B0020031EB8BF2D2210B513
:10CDD800B8BF58420C46B8BF01F8012B0A22FDF72C
:10CDE80043FD00230370204610BD07B51B4B03F617
:10CDF8004C02C3F8482893F8C0225AB1012A14D12A
:10CE0800032183F84E18072183F8502883F84F1818
:10CE18000C2208E0022183F84E18032183F85028D9
:10CE280083F84F18072283F84C280D4B0D4A9A6057
:10CE38004020FAF759FC70B10122002390F9000054
:10CE480040218DE80C00084A4FF4E133FAF724FA40
:10CE5800003018BF012003B05DF804FB181B002048
:10CE68005C000020458C0008C58D000801200021C9
:10CE780000F03EBEF0B51C4A92F85138D2F854582A
:10CE880092F8587892F8646892F870E8022B0ED8F5
:10CE980005EBC304591CA31CC9B206D02346A488B9
:10CEA80014F0010F01D0204205D10B46EEE782F8BD
:10CEB80051380020F0BD93F902307CB29C4201D178
:10CEC800002307E074B29C420CD04FFA8EF49C42C7
:10CED800EBD1022382F851180C2101FB0322D2F86E
:10CEE8005C08F0BD0123F5E7181B00200B4B10B5BB
:10CEF80019684FF6FB720A401A60094A92F88628A8
:10CF08001C46084B0AB1052200E001221A6001F014
:10CF1800FDFA4FF43643236010BD00BF405C00406B
:10CF2800181B0020DC260020022803D0431E58428C
:10CF380058417047064B1B681B7823B1054B18688E
:10CF4800C0F3C0407047044B1878C0F380007047A6
:10CF5800D4090020AC100020F3260020674B73B5DD
:10CF68001878674DFFF7E0FF2B788342044620D0FE
:10CF7800C8B1644B1B68E3B193F900000223009326
:10CF8800614B1B685B78003318BF012301930421B0
:10CF98004FF416530022FAF77FF95C4B186040B142
:10CFA80001232B7005E0594E3068FAF75AF93460BE
:10CFB8002C70574B574D1878FFF7B6FF2B788342E4
:10CFC800044618D088B1544B1B68A3B10022012431
:10CFD80093F9000000944FF4964301920821FAF760
:10CFE8005BF94E4B186028B905E04C4E3068FAF7EB
:10CFF80038F934602C704A4B4A4D1878FFF794FF83
:10D008002B78834204462E4642D0002837D0464B20
:10D018001A68002A3CD0D37992F90000434C002BBF
:10D0280008BF022302220092002254F82330019202
:10D038001021FAF731F93E4B0546186040B33D4CD4
:10D0480094F84A30022B0BD094F89620022A01D18A
:10D058004C3405E023B1002A04F14C0418BF002425
:10D06800354B1C6044B1204600214C2205F0DDFB05
:10D078000223256084F84A300123337008E02C4EDF
:10D08800306800F0E9FC3068FAF7EBF834602C708F
:10D098002A4B2B4D1878FFF747FF2B78834204461D
:10D0A80029D000B3274B1B682BB3274A93F90000FC
:10D0B80012685278002A0CBF082209220323009321
:10D0C80001924FF4614320210022FAF7E5F81F4B43
:10D0D800186080B11E4A012313702B701D4B1A680B
:10D0E8001D4B1A6007E0194E3068FAF7BAF8184B6A
:10D0F80034601C702C7002B070BD00BFDC090020C9
:10D1080081070020D80900208C0700208414002003
:10D11800DD090020910700201008002000080020E9
:10D12800E809002016080020E409002080450108CD
:10D1380018080020B01B00201C080020F40900205B
:10D1480024080020F0090020EC090020280800200D
:10D158002C080020181B0020300800202DE9F04F73
:10D16800C24BDA682DED028B1A61C14A1168D96089
:10D17800C0490B6843F020030B60BF4B19780129A5
:10D1880090460CBF002201221A70BC4B1A789107F6
:10D1980089B040F13D83BA490978042940F23883BF
:10D1A800B849097801F0040101F0FF0011B922F033
:10D1B80001021A701B78DB0702D408B1FEF76AFC7B
:10D1C800B1490A78531C052293FBF2F202EB820262
:10D1D8009A1AAE4B0A701B78039392000023AC4C4A
:10D1E800DFF8CCC2DFF8D8925CF8231091FBF9F590
:10D1F80004F1080004F1100640F82350A54844F84B
:10D20800231000FB051142F2107091FBF0F080B280
:10D2180026F813004FF0140E04F1140604F13C0A2A
:10D228000EFB036E5AF823605EF802704EF8021087
:10D23800F61B314444344AF82310052691FBF6F1D5
:10D2480009FB051144F82310039C012C4FEA830BBA
:10D25800E24605D10238B0F5797F98BF4BF80C103B
:10D268000BB90123BBE7884CD8F80030226D9FED3D
:10D278008A7A8A4E8A4D9B1A07EE903AF8EE677AB8
:10D28800D8F800302365C7EE877A7C4B1B78B7EE59
:10D29800008AF4EEC87AF1EE10FA58BFF0EE487A38
:10D2A80013F00103C4ED157A12D005AA00927D4B44
:10D2B80006AA01920CCB9AE80300FEF7E9FA64216A
:10D2C800059A069BB2FBF1F293FBF1F3328000E082
:10D2D80033802B8094F858306B48002B3BD0D0ED2E
:10D2E800157AC26DDAF80030C8EE276A9B1A026E0A
:10D2F800022507EE103AB8EEC77ADAF8043027EEBE
:10D30800267A9B1AFDEEC77AB0F9662017EE901AB6
:10D3180007EE903A644BB8EEE77AD3ED007A67EE01
:10D32800277A67EEA67AFDEEE77A17EE903A02FAC8
:10D3380083F3B0F9642093FBF5F302FA81F29BB210
:10D3480092FBF5F292B2A0F86A30A0F86820A0F833
:10D358006630A0F86420012384F85830534BDAF87B
:10D3680004101B88DAF80000474D514E216603F07F
:10D378003003E065002B00F04B8205F17403009345
:10D3880005F178030193EA6E2B6FFEF781FA726854
:10D398002B6F9B1A07EE903A434B326893ED007A55
:10D3A800EB6EF8EEE77A9B1AEB67384B67EE877AF5
:10D3B8001B78FDEEE77A012BC5ED207A03D0022B0E
:10D3C80000F0DF8024E2D5ED287A3A4BD5ED215ADA
:10D3D80095ED255A95ED156A95ED264AD5ED274A1E
:10D3E80035491D68B1EE677ABDEEC77AFDEEE77A7A
:10D3F80017EE10EA17EE90CA0020304A91ED007A35
:10D4080052F8207007EE907AF8EEE77AA2F114034A
:10D4180067EEA57A33F81060FDEEE77A283217EE4A
:10D42800903A9B1B9BB222F810301BB207EE903A41
:10D43800F8EEE77A3B4467EE857A4400FDEEE77A3A
:10D44800CDED037A07EE903AF8EEE77ABDF80C8056
:10D4580067EE847AA7EE867AFDEEC77A17EE902AF1
:10D46800724531DB6245A8BF62462EE07C01002090
:10D47800181B0020A41000202E11002018110020D5
:10D4880019110020F3260020B0230020D40A002020
:10D49800B4230020806967FF00007A442A11002025
:10D4A8002C1100203011002068000020A810002056
:10D4B8001C110020D80A0020080B00202C24002072
:10D4C80080969800DB0FC940724607EE902AF8EE66
:10D4D800E77A5FED046AC1ED007AFDEEE77A31364E
:10D4E80017EE903A43449AB2AB78D1ED027A07EE40
:10D4F800103AB8EE477A4B684F6027EE267AFB1A47
:10D5080088EE077AB6B2622E06EE903AF8EEE66A30
:10D5180037EE067AC6EE866A86EE077A76EEE76A10
:10D52800E7EE267AC1ED047AC1ED027A0FD964EEEE
:10D53800A77ABA4EFDEEE77A17EE903AB3F5FA6F8E
:10D54800A8BF4FF4FA63B342B8BF334600E00023E4
:10D5580013441BB240F6B8329342A8BF1346B04AF0
:10D568009342B8BF1346AF4AA352AF4A142303FBF2
:10D57800002351F8142B1A60002840F0498101203B
:10D588003BE7AA4BD5F874801F68D4F878903E8999
:10D59800DFEDA78A4FEA58039E4228BF1E46B5F81A
:10D5A800A8301AB29642C3BFD5ED157A9FEDA17A7D
:10D5B80067EE877AB6B2C1BFFDEEE77A17EE906ADA
:10D5C800F618B6B2C8BFA5F8A860D4F8AC50C5EB39
:10D5D80009052846FEF7A0F90028D8BF404241F2C5
:10D5E80093129042CCBF0020012088B307EE905AD6
:10D5F800B8EEE70A20EE280AFDF7C8FA07EE908A87
:10D60800F8EE677A40F6B83320EE270AFDEEC07AC6
:10D61800CDED037ABDF80C20A4F8B02012B29A42DE
:10D62800A8BF1A467E4B9A42ACBF09EB02034B4493
:10D6380048F6A042934203DDA3F50C43A03B04E067
:10D64800002BBCBF03F50C43A033C4F8B43001E091
:10D65800C4F8B490D4F8B450C5F50C53283307EE89
:10D66800903AF8EEE77A67EEA88AB0EE680AFDF716
:10D67800EDFA8DED070AB0EE680AFDF787FAD4EDEA
:10D68800317AD4ED2E4AD4ED155A94ED2F4A94ED03
:10D69800305A65498DED060AB1EE677ABDEEC77A54
:10D6A800FDEEE77A0DF1180E17EE10AA17EE90BAF4
:10D6B8000020614AFEEC016A32F91030DFF88C91E3
:10D6C80007EE903A07EE106AF8EEE77AB8EEC77AF6
:10D6D8003C32D6EE877A4FEA400CFDEEE77ACDED84
:10D6E800037ABDF90C30B3F57A7FA8BF4FF47A738B
:10D6F8004B45B8BF4B461FFA83F922F810900FFA32
:10D7080089F207EE902AF8EEE77A27EEA47ABDEEC2
:10D71800C77A8DED037A27EE847AD1ED007ABDF8C9
:10D728000C90E7EE257AFDEEE77A17EE902A52453F
:10D7380003DB5A45A8BF5A4600E0524607EE902A36
:10D74800F8EEE77A9FED3D6AC1ED007ABA7891ED7F
:10D75800027A06EE902AF8EE666A4A684B6066EE30
:10D76800866A9A1AC8EE266A143106EE102AB8EEAE
:10D77800C66A76EEA56A86EE256AC5EEA66A36EE14
:10D78800476AA6EE867A01ED017A01ED037A25EE65
:10D79800077ABDEEC77A17EE103ABDEEE77A4B442A
:10D7A80017EE102A13441BB240F6B8329342A8BFB2
:10D7B80013461B4A9342B8BF13461A4A2CF8023044
:10D7C8001F4A142303FB0023C3ED007A08B9012084
:10D7D8006FE73B7923B1642395FBF3F5194B1D8063
:10D7E8003B8898450DD9D4F8AC30A06FC01AFEF725
:10D7F80093F880EAE072A2EBE07242F210739A4268
:10D8080006DD114B01221A700E4BB4F8C8201A809D
:10D8180009B0BDEC028BBDE8F08F00BF30F8FFFF08
:10D8280048F4FFFF5C0B0020300B0020D80A0020D2
:10D83800D30237390000C84218240020DB0FC94042
:10D84800080B00208C100020D40A002018FCFFFFD1
:10D8580007B5064B0093064B01930649064A074B4A
:10D868000748FDF702F903B05DF804FB805501088D
:10D87800555501081663010820630108745501080D
:10D88800F362010808B5037833B90C4B0C481978D2
:10D89800BDE80840FDF7E9B805F062F802280CD8A1
:10D8A800064B1870074B0C2202FB0030064B063063
:10D8B8001860FDF7BFFA0548E5E708BD7C2400209D
:10D8C8002763010828230020141100204459010867
:10D8D80008B503783BB90B4B0B4893F8E416BDE841
:10D8E8000840FDF7C2B805F03BF8022808D8054BF8
:10D8F80083F8E406FDF704FAFDF7C0FA0348E8E701
:10D9080008BD00BF481C00202B63010844590108CA
:10D9180038B5037803BB214B1B6801330F2B07D89D
:10D928001F490C2202FB03121C4695682DBB00E020
:10D938001C4601340F2C01DD002400E005D81849ED
:10D948000C2202FB04129568BDB99C42F1D115481E
:10D95800BDE83840FDF789B805F002F80F280446FD
:10D9680005D80F4A0C2303FB00239D682DB92146D7
:10D978000D48BDE83840FDF778B8084B1C60F9F74A
:10D988009BFF21462A460948FDF76FF80C235C43A4
:10D99800034B185DBDE83840F9F7A4BF6C000020C0
:10D9A800A0450108386301084E6301086663010851
:10D9B80073B5037813B9F9F7F9FA3FE001AA2049DA
:10D9C80005F02FF800240246264625469AB134B1C0
:10D9D800012C08D1104604F0C3FF064603E01046A8
:10D9E80004F0BEFF054601AA0020154905F019F804
:10D9F80001340246EAE70B2D03D9124812490C23D9
:10DA08000CE0022C11D1A6F57A73B3F57A7F08D908
:10DA18000C480E494FF47A724FF4FA63FDF725F873
:10DA28000CE00B4B03EB45035E80094B094803EB05
:10DA380045032946B3F90220FDF717F802B070BD77
:10DA4800BE5E0108B55A0108D45A0108776001087A
:10DA58007C2400207D63010838B50D4C236883427F
:10DA6800054606D1F9F7FDFB204600214C2204F0BB
:10DA7800DCFEE36CAB4209D12846F9F7F2FB054816
:10DA880000214C22BDE8384004F0CFBE38BD00BFAD
:10DA9800B01B0020FC1B0020034BDA69D379591C0A
:10DAA8001344D171187A70477C24002010B5FFF711
:10DAB800F3FF84B2FFF7F0FF04EB002080B210BD43
:10DAC80010B5FFF7F3FF0446FFF7F0FF04EB004043
:10DAD80010BD38B5054D04462146286AF7F78CFD78
:10DAE800EB6998796040987138BD00BF7C240020AC
:10DAF80038B5044624200D46FFF7EBFF4D20FFF70D
:10DB0800E8FF002C084C14BF21203E20FFF7E1FF5E
:10DB1800E369002228469A71FFF7DBFFE36993F86F
:10DB28004900BDE83840D4E77C24002001460020A5
:10DB3800DEE710B50446C0B2FFF7CBFF200ABDE808
:10DB48001040C6E710B5044680B2FFF7F2FF200C7C
:10DB5800BDE81040EDE737B58288836804461006B3
:10DB68000D4641BF2B4991F8E4164FF4CC7000FBE9
:10DB78000133D10544BF2849097802F03F0244BF68
:10DB880001EB410103EB8103042A12D006D8012AD4
:10DB98000DD0022A32D193F9001030E0102A0AD0B1
:10DBA800202A0AD0082A29D1B3F9001027E01978C9
:10DBB80025E0198823E0196821E093ED000A6846FA
:10DBC800FCF7E8FD01461548FCF74FFF05B3D4ED17
:10DBD800037A6846B8EEE70AFCF7DCFD0146104810
:10DBE800FCF743FF94ED040A6846B8EEC00AFCF758
:10DBF800D1FD01460A48FCF738FF09E00021094831
:10DC0800FCF733FF25B10848E1682269FCF72DFFCE
:10DC180003B030BD481C00207C240020215C010892
:10DC28001A5C0108906301088C630108024B0146E5
:10DC3800586AF7F7E1BC00BF7C24002010B5441EE9
:10DC480014F8011F21B1034B586AF7F7D5FCF7E721
:10DC580010BD00BF7C2400202DE9F3412B4E2C4B36
:10DC680096F828002B4D1C682B4B05EB80001A8872
:10DC78002A4BD0F8C0101B78294800914FF47A71CC
:10DC8800B4FBF1F1FCF7F1FE26484821FCF7EDFE64
:10DC9800254BD3F800800027FBB205EB8302D2F8AE
:10DCA800D010E9B101249C4014EA080F16D02207CD
:10DCB80014D01E4AD25C0B2000FB0323154A1C48D3
:10DCC80002EB8303D3F8F020FCF7CFFE022C05D13A
:10DCD80096F8341011B11748FCF7C7FE0137DBE797
:10DCE8001548FFF7ABFF154B15481A68154B9A42B4
:10DCF8000CBF154B154B1A88154B198892B24FF467
:10DD0800E36302B0BDE8F041FCF7AFBE7C2400201D
:10DD1800181B0020A045010858180020F800002012
:10DD280093630108D6630108A4100020F4000020C2
:10DD3800E6630108EE630108366401089C100020C0
:10DD4800F263010800540040A0100020A210002037
:10DD5800981000202DE9F0410024804625460F4EFA
:10DD6800A7594146384604F0E3FD58B139460C48F6
:10DD7800FCF77BFE30190021FFF7EDFE0948FFF79D
:10DD88005DFF0135143440F658439C42E7D11DB974
:10DD98000548BDE8F04151E7BDE8F081404701087A
:10DDA800A75C010836640108495C01082DE9F04FB9
:10DDB8002DED028B83B0054604F07BFD064620B1AD
:10DDC800012818D12B782A2B15D15C48FFF736FF8C
:10DDD80000245B4D5B486159FCF747FE2819314622
:10DDE800FFF7B9FE5848FFF729FF143440F65843A7
:10DDF8009C42EED19CE028463D2104F04CFD0028D1
:10DE080000F08F800346994613F8012D202AFAD096
:10DE1800441C204604F0A4FD80462046FCF730FC54
:10DE2800C5EB0909B0EE408A0026DFF834A11422B8
:10DE380002FB06F40AF5D07B54F80B70384604F060
:10DE480038FD03461A4628463946019304F03AFD40
:10DE5800019B00285BD15FFA89F29A4257D10AEBFD
:10DE68000402D2ED6B7AF8EEE77A0BEB0405B4EE18
:10DE7800E78AF1EE10FA48DBD2ED6C7AF8EEE77A31
:10DE8800B4EEE78AF1EE10FA3FD8B2F8A431D2F82E
:10DE9800A82113F0200F08BF08EE108A1C0641BF06
:10DEA8002A4991F8E4164FF4CC7404FB0122D905F1
:10DEB80044BF2749097803F03F0344BF01EB410100
:10DEC80002EB8102042B18EE100A0BD004D8013B98
:10DED800012B0ED810700CE0102B05D0202B06D08B
:10DEE800082B06D1108004E082ED008A01E082ED63
:10DEF800008A39461748FCF7B8FD2846002103B0C8
:10DF0800BDEC028BBDE8F04F25E6134803E001366F
:10DF18009E2E8AD1114803B0BDEC028BBDE8F04FAC
:10DF28008CE6284603B0BDEC028BBDE8F04F11E744
:10DF380003B0BDEC028BBDE8F08F00BF246401087C
:10DF480040470108A75C010836640108481C002006
:10DF58007C2400203964010844640108495C0108F4
:10DF6800A045010870B50546284604F0A2FC0646FF
:10DF780058B9194B19485A79194B03EB8203BDE874
:10DF88007040D3F8F41DFCF770BD28461549324699
:10DF980004F098FC60B91448144CFFF74FFE54F88D
:10DFA800041F19B11248FCF760FDF8E7114805E0B5
:10DFB8000024114B53F8241019B91048BDE87040DB
:10DFC8003CE62846324604F07DFC01340028F0D1B6
:10DFD800014B0B4D5C71C7E7481C002064640108C5
:10DFE800A0450108385C01087064010894530108D1
:10DFF800345C01083664010898530108495C01083B
:10E008004459010808B50748FFF718FE064B586A37
:10E01800F9F71CF9F7F75AFCFCF748FE034B044ADA
:10E02800DA6008BD836401087C24002000ED00E06C
:10E038000400FA0508B50548FFF700FE00F036F8B9
:10E04800FCF75EFEBDE80840DCE700BF8F6401080E
:10E0580008B50448FFF7F2FDFCF752FEBDE808409A
:10E06800D0E700BFA56401080E4B1A786C2A16D1B8
:10E078005A88B2F5E36F12D11A79BE2A0FD193F8F4
:10E088001427EF2A4FF000000BD113F8012B504052
:10E09800054A9342F9D1B0FA80F040097047002050
:10E0A8007047704700F8030818FF03082DE9F04F80
:10E0B8002DED028BEB4D00214FF4E36285B028462D
:10E0C80004F0B3FBE84B05F507721A60E74A002332
:10E0D8001370E74A05F2E66111606C222A70032288
:10E0E8006A714FF48072AA604FF41672A5F8642121
:10E0F800FA22A5F866214FF4FA722021A5F86C21BE
:10E10800012285F85E2185F8681185F869216E215C
:10E1180085F86A2185F87C2185F88421052285F80F
:10E128007A1185F81B220A2140F2DC5285F87B110E
:10E13800A5F896212B2140F24C4285F87D11A5F8CF
:10E148009821212140F26C7285F87E11A5F89A2158
:10E15800232140F2753285F87F11A5F89C214FF4F0
:10E16800C87140F64302A5F89E21A5F880112A46F9
:10E178002C46032BCCBF0121002103F1010382F8B7
:10E18800A01114BF1E210521122B82F8A11102F142
:10E198000202EED140F27E414FF4FA63A4F8401136
:10E1A80040F23A71A4F8C631A4F8CA31A4F8CE31C5
:10E1B800A4F8D231A4F84211052340F27E5184F824
:10E1C800E031A4F84811C82340F2EA5101274FF47E
:10E1D8007A794FF0320A40F2DC50A4F8E431A4F81E
:10E1E8004A114FF4C87340F2B4511E224FF0190B74
:10E1F800A4F8E831A4F84601A4F84C11A4F84EA1FB
:10E20800A4F8C491A4F8C891A4F8CC91A4F8D0912A
:10E2180084F8E27184F8E37184F8E671A4F8449113
:10E2280084F89321019284F8E1B10390A4F8503165
:10E23800A4F852A184F8DF7184F8EC7184F8EF71C6
:10E24800FEF75EFD8849019A0B6802910026267345
:10E25800DA721A735522DA700F225A7122229A71D1
:10E268000E221A7435229A7621225A7453224FF0BC
:10E278002D0EDA765A224FF0280883F80DE083F83D
:10E2880007B01A724FF0640B0A2283F814E04FF0BB
:10E29800780C4FF4FA7E83F804A09A74019283F8FC
:10E2A8000AC01E7083F8018083F8158083F8028005
:10E2B80083F81680DE759E731E76DE735E7683F8AD
:10E2C8001CB083F809809F77A3F84EE0DFF8BCE123
:10E2D800C3F838E0C3F83CE0DFF8B4E1C3F828E05D
:10E2E800DFF8B0E1C3F834E0DFF8ACE1C3F848E0A8
:10E2F800DFF8A8C19FED5F8AC3F82CC04FF04B0E22
:10E30800C3F830C083F84CE0F7EE087ADFF890C124
:10E31800039883F850804FF0460EC3ED087AC3ED9A
:10E32800097A83ED108AC3F844C084F8E7E6A4F8B4
:10E33800F0064FF0140E042084F8E8A684F8EEE600
:10E3480084F8E6B684F8E96684F8ED6684F8EA6647
:10E3580084F8EB6684F8EC6683F85C00152083F893
:10E3680068004548A3F85860A3F85A60A3F85660B7
:10E37800C3F860C083F8648083F86580D8663F4836
:10E3880018673F48586783F878703E48FEF7FEFCE8
:10E398000299019AD1F800A04FF44873AAF81631EF
:10E3A800C8238AF811618AF812618AF813818AF8F9
:10E3B80014718AF8186184F8D62184F8D731A4F842
:10E3C800D89184F8DA61A4F8DCB152460E2303FB35
:10E3D80006A36FF0170183F81911032183F81A11A6
:10E3E8006FF02F0183F81B11072183F81C116FF0C0
:10E3F800230183F81D11052183F81E1101365A21C6
:10E4080082F8201182F821116423FF21082E82F856
:10E418001F3182F8221102F10E02D7D100228AF8A8
:10E428008921C822AAF88A21AAF8903114224FF427
:10E4380096738AF88C21AAF892311E2228238AF82A
:10E448008D21AAF8943101220F4B8AF88E2118EEFB
:10E45800102A45F8102F9D42F9D1024C00230125BE
:10E4680051461FE0481C0020E81000207C240020B2
:10E4780014110020000000009A99193FF6287C3FEB
:10E488003D0A773F526F0108081D00208FC2F53CF6
:10E49800000060406666663F00004040CDCCCC3E40
:10E4A8000000A04004F56D704FF4CC7284F80C376E
:10E4B80084F80A5784F80B5704F0ACF904F24C506E
:10E4C80051464FF4CC7204F0A5F90F4B1B681A683B
:10E4D800C4F8F2265A68C4F8F6269A68C4F8FA26E8
:10E4E8001A68C4F8FE265A68C4F802279A68C4F85D
:10E4F8000627022384F8085484F8A03505B0BDEC3B
:10E50800028BBDE8F08F00BF141100201549D1F827
:10E51800883043F47003C1F88830134B1A6842F00E
:10E5280001021A605868114A02405A601A6822F0BB
:10E53800847222F480321A601A6822F480221A60E7
:10E548005A6822F4FE025A60DA6A22F00F02DA628E
:10E55800186B074A02401A6300229A604FF0006362
:10E568008B60704700ED00E0001002400CC07FF89F
:10E57800CCFC00FF38B5094B93F80C5765B9084C2B
:10E588002068F8F76EFE074B25601B78022B03D135
:10E59800BDE83840FEF773BB38BD00BF481C0020FB
:10E5A800D4240020D3240020044B93F80C371BB943
:10E5B800034B1868F7F714B800207047481C002070
:10E5C800D424002038B505460446204614F8011B1B
:10E5D80021B1034B1868F7F70FF8F6E7401B38BD71
:10E5E800D42400200FB407B504AB064953F8042B14
:10E5F80001930020FCF74CF903B05DF804EB04B07C
:10E60800704700BF7BE70008024B01461868F6F721
:10E61800F3BF00BFD4240020F8B5011F064600232D
:10E62800083051F8042F02F120043F2C3AD802F1A7
:10E6380008040F2C06D80232032A04D9002B08BF7D
:10E64800012300E002238142EBD1012B30680ED078
:10E65800022B1AD0736803F003039B0000F0030039
:10E6680043EA0010B36803F00303184317E000F00F
:10E678000F0040F04000FFF7C7FFB068736800F074
:10E688000F0040EA0310C0B209E000F03F0040F07C
:10E698008000FFF7B9FF3079FFF7B6FF307ABDE8A1
:10E6A800F840B1E706F10C0734463A46002552F81F
:10E6B800043D03F18001FF294FEA850510D903F5D0
:10E6C8000041B1F5803F02D245F0010508E003F5AD
:10E6D8000003B3F1807F34BF45F0020545F0030520
:10E6E800B242E4D165F03F00C0B2FFF78DFF05F0FC
:10E6F8000303022B207807D0032B0CD0012B13D156
:10E70800FFF782FF60780FE0FFF77EFF6078FFF782
:10E718007BFFA07808E0FFF777FF6078FFF774FFCA
:10E72800A078FFF771FFE0780434FFF76DFFBC4273
:10E738004FEAA505DBD1F8BD10B50446C0B2FFF716
:10E7480063FFC4F30720BDE810405DE710B5044639
:10E758007F2C06D964F07F00C0B2FFF755FFE409AB
:10E76800F6E7E0B2BDE810404EE7430083EAE07008
:10E77800ECE7084648E700BF20B9034B1B680822AE
:10E788001A82704701487047241B00205C00002053
:10E7980021B901288CBF0220002070470220704751
:10E7A80010B50A4B1968CA78042A0CD84C8A084B49
:10E7B80028B903EBC2039B881B1B0B8210BD53F8BF
:10E7C8003230181910BD002010BD00BF241B0020D6
:10E7D80070000020054B1968054B4A8A18B99B8CB4
:10E7E8009B1A0B827047186A10447047241B00203C
:10E7F80070000020054B1968054B4A8A18B99B8D93
:10E808009B1A0B827047986A10447047241B00209B
:10E8180070000020074B1B681B7803F07F03212B37
:10E8280006D100F0DF00022814BF02200020704744
:10E8380002207047241B0020212810B508D1114B55
:10E848001B681B7803F07F03212B10D0022010BD1A
:10E858002028FBD10B4B0C4A1B6810701B7803F067
:10E868007F03212B094B18BF00230BB9EEE7084B98
:10E87800044A12680024936154822046984720462F
:10E8880010BD00BF241B0020F8260020DDC60008AC
:10E8980081E700087047034B1A78202A04BF00223A
:10E8A8001A707047F8260020014B04221A6070473E
:10E8B800DC260020034B9B7A13B1034B05221A6018
:10E8C800704700BF94230020DC2600200D4B0E4922
:10E8D8001A680E4B92B213445B000D4A1B68C3F3CF
:10E8E800090310B5136013689BB201335B10002253
:10E8F8009A4206D0074851F8044B20F812400132DA
:10E90800F6E710BD505C0040206200401E30002039
:10E91800201B0020291B0020014B00221A60704791
:10E928001C1B00202DE9F843664B674E1B68DFF877
:10E93800B881664A00254FF0C0099D7283F8099096
:10E94800DD723560D8F8003023F4EC4323F070030F
:10E9580043F400739BB2C8F80030D8F8003023F4B1
:10E96800E04323F040039BB248F2800483F0100395
:10E978002343C8F80030336812FA83F35B0040275A
:10E988001A681F6033689BB203F1005303F54053C4
:10E998005B0028461A6880221A60D8F8003023F4F1
:10E9A800F8731B051B0D2343C8F80030484B93F838
:10E9B8005C10FAF741FBD8F80030464A464923F480
:10E9C800804323F070039BB283F440532343C8F879
:10E9D8000030136823F4EC4323F070039BB21360F8
:10E9E800336811FA83F35B0003201968C3F80090B9
:10E9F80013683A4923F4E04323F040039BB283F0C1
:10EA0800200323431360136823F4804323F0700327
:10EA180023439BB21360536823F4EC4323F0700341
:10EA280043F4C0639BB25360336811FA83F35B000D
:10EA380019684FF480711960536823F4804323F0F8
:10EA4800700323439BB25360536823F4E04323F0DD
:10EA580040039BB283F0200323435360D8F80C3063
:10EA68001F4A23F4EC4323F070039BB2C8F80C3020
:10EA7800336812FA83F35B0039461A684FF48872D8
:10EA88001A60FAF7D9FAD8F80C3023F4804323F047
:10EA980070039BB283F440532343C8F80C30D8F872
:10EAA8000C3023F4E04323F040031C43A4B2C8F81D
:10EAB8000C402846FDF7CBF90A4B01221A60BDE845
:10EAC800F88300BF241B0020505C00400430002065
:10EAD80070000020045C0040083000201030002046
:10EAE8001C300020DC260020005C0040134A144B38
:10EAF80050681B68181810B5146808D01149082206
:10EB0800FDF791F9204610490422FDF78CF90F4BC7
:10EB18001A68002393720E4A012111600D4913608F
:10EB28004FF4E0500B6010600B480B604FF4364117
:10EB380001801160094A136010BD00BFB0F7FF1FC4
:10EB4800ACF7FF1FD2000020E2000020241B0020A9
:10EB5800405C0040445C0040CC240020DC260020BF
:10EB6800024B4FF480221A60704700BF1404014022
:10EB78002DE9F04FAD490B7813F0010F85B003F084
:10EB8800040200F04581002A40F07281A848076815
:10EB980017F0806740F06C81980700F1398143F0E5
:10EBA80004030B70A34BA44C1B882380A34B1A6847
:10EBB80012F4002F984600F00C81A14B80201F70A2
:10EBC800FEF758F908B1FEF747FFA678012E40F086
:10EBD80000819C4D95F80A2722B195F80B370BB1A7
:10EBE8009A4203D3012385F80A370FE018461146E5
:10EBF80030B191FBF0FE00FB1E1E01467046F7E7A0
:10EC080092FBF1F285F80A2793FBF1F385F80B37AD
:10EC180095F80C371BB18B4B002283F80C278A4BD5
:10EC280095F80CA71B6841F6690203EBC3039342EE
:10EC380084BF40F2E242B3FBF2F3844A8CBFDBB2FA
:10EC480004231370BAF1000F1FD18020F8F74CFD90
:10EC58008146D0B18021F8F721FD99F806207C4B38
:10EC6800E07053F8223099F90000DFF8CC91B3F541
:10EC7800613F0CBF0222002202218DE8060080219C
:10EC88005246F8F709FB606008B90023A0E0514636
:10EC980009F10800142203F0C8FD09F12803C9F896
:10ECA8001C3009F19403C9F8203009F58073C9F8BC
:10ECB8002430684BD8F800101B88A9F86C3195F8F7
:10ECC8009231654895F884910390002B6B79A3F1F4
:10ECD800190BC1F3C03C18BF4FF0010CDBF1000E5B
:10ECE8004EEB0B0E95F80AB7012B95F80B37056814
:10ECF80008BF4FF0010E9B45584B1B780293C1F398
:10ED0800400A28BF4FF0000B01F4006138BF4FF0F4
:10ED1800010B721ED2B2531E132B35D8DFE803F055
:10ED28000C0C0C0C0C0C0C0C0A37377F2737811293
:10ED380012123137734675E0029B9342B4BF002329
:10ED4800012320E02B78022B0BD105EB820353ED36
:10ED5800027AF5EE407AF1EE10FA14BF012300238F
:10ED680011E0AB185B79003318BF01230BE021B128
:10ED780009F1FF304342434100E00B4603F0010331
:10ED880050E05B464EE013B1012393401F43142E1D
:10ED980002D80136F6B2BCE7039BC4F87071186854
:10EDA80019217930F8F732FD0023C4F87831A4F836
:10EDB8007C31A4F87E31C4F88831294BD4F88421F9
:10EDC8001B68C4F88C3184F87401C4F880210223CC
:10EDD800A370234B1B4A1B6892F8E0214FF47A7109
:10EDE80001FB02331F4A1360D8F800301A0609D510
:10EDF8001D4B1B789B0705D51C4B1B78042B01D991
:10EE0800062000E0052005B0BDE8F04FF8F76ABD20
:10EE180072BB012005B0BDE8F04FF8F787BD534637
:10EE280000E06346002BAFD1B3E700BFF326002014
:10EE3800AC10002004110020D0240020781B0020F2
:10EE480069230020481C0020CC150020F900002070
:10EE580080450108CC170020E8100020C0110020D0
:10EE6800181B0020900A00201811002019110020FA
:10EE780005B0BDE8F08F10B5154A1378590725D5A8
:10EE880023F004031370134B1B681B0319D5124C92
:10EE9800A378A3F10802012A0BD8FF200021F7F775
:10EEA800DBFB0E4B1B68C4F88C31FFF77DFB0A2394
:10EEB80006E0012B05D90A2B03D0FFF75BFB0123E2
:10EEC800A3700420BDE81040F8F70CBD10BD00BFCA
:10EED800F3260020781B0020D0240020181B0020D7
:10EEE800064B1B7803F0040303F0FF001BB1044B2F
:10EEF8001888C0F3C01000F001007047F326002006
:10EF0800A81000202DE9F04F2DED088B83B00AEEF4
:10EF1800102A0093D14B01931A8812F0020F05466C
:10EF2800F7EE009A4CD0149BCD48DC89B0F900303C
:10EF38001B1B03F2F31640F2E632964203D8002B6D
:10EF4800B8BF5B4201E04FF4FA73B0F90220121B1C
:10EF580002F2F31440F2E630844203D8002AB8BF24
:10EF6800524201E04FF4FA7295F84C0058B39342BC
:10EF7800B8BF1346C3F5FA7307EE903A9FEDB97A16
:10EF8800F8EEE77A6423C7EE877A93FBF0F307EE8F
:10EF9800103A77EEE97AB8EEC77AB0EE699AA7EE3A
:10EFA800879AF7EE006AB5EEC09AF1EE10FA0AD425
:10EFB800B4EE669AF1EE10FAC8BFB0EE669A04E0B5
:10EFC800B0EE699A01E09FEDA89AA84ECF1C2C4696
:10EFD8004FF00008B8F1020F17F801BFDFF8DC9214
:10EFE8004FEA480AF2EE04AA0ED1B9F904109FEDCF
:10EFF800A07A0BF10A0B01FB0BF307EE903AF8EE3F
:10F00800E77AC7EE877A68E0F8EE4A7A9FED956A64
:10F0180039F91830C7EE867A06EE903A954B33F9EF
:10F02800183007EE103A1AEE103AF8EEE66AB8EE23
:10F03800C77A5B42A6EEA77A07EE903AF8EEE77A2F
:10F04800B4EEE77AF1EE10FA08D4F8EECA7AB4EE24
:10F05800E77AF1EE10FAD8BFF0EE477A864B33F92B
:10F068000A3008EE103A009BB8EEC88A33F9183017
:10F0780077EEC87A08EE103AB8EEC88A37EE888A72
:10F0880088EE2A8AFFF72CFF40B17C4B13F8080062
:10F09800B0EE480AFDF7B2FBB0EE408A019B198832
:10F0A800CA0704D5D5ED117A68EE277A15E039F943
:10F0B8000A309FED6F7A0BF1140B03FB0BF307EE8D
:10F0C800903AF8EEE77A8B07C7EE877A42BF95ED5C
:10F0D800127A28EE078AE8EE097A694BDFF8E0B180
:10F0E80033F90A3094ED08BA9FED668ADFF8D491B7
:10F0F80007EE103A644BB8EEC77AD3ED046A18F8F5
:10F108000B30E7EE667AB8F1020FF0EE48BAF0EE8F
:10F11800678A67EE8B7A0BEE103AB8EECBBA27EE19
:10F128008BBA8BEE08BA09D1B0EE4B0A5748D9ED25
:10F13800000A1E21FBF77AFAB0EE40BAD9ED000AB0
:10F1480094ED0B7A68EEA07A67EE877A96ED007AEE
:10F15800A7EEAA7ADFED4E7AB4EEE77AF1EE10FA6E
:10F16800F0EE47AA09D4DFED4B7AB4EE677AF1EEF8
:10F1780010FAC8BFF0EE67AA01E0F0EE67AA89EEC0
:10F18800A08A45494FEA8809494491ED000AC6ED2D
:10F1980000AAC1ED008A38EEC00A95F8501020EE9A
:10F1A800080A21B13D4800EBC800FBF73FFAD4ED4F
:10F1B8000E7A1BF8083060EE277A00EE103AB8EEA7
:10F1C800C00A27EE800ADFED367A80EE2B8AB4EE8D
:10F1D800E78AF1EE10FA09D4DFED327AB4EE678AE5
:10F1E800F1EE10FAC8BFB0EE678A01E0B0EE678AA8
:10F1F8003BEE2A0A08F1010830EE080A03F024FD64
:10F208002949B0F57A7FA8BF4FF47A708842B8BF11
:10F218000846BDEECBBA25491BEE103A21F80A0084
:10F22800FDEEEAAA2249BDEEC88A49F80130214913
:10F238001AEE903A49F801301F4918EE103AB8F121
:10F24800030F49F8013004F1040406F104067FF4C1
:10F25800C1AE03B0BDEC088BBDE8F08FA81000204C
:10F26800782600200000FA4300000000A8150020BE
:10F2780000004842EE2600206E1B0020043D0108D5
:10F28800D21000200000C8425C1300202015002086
:10F2980000007AC300007A43642600204415002049
:10F2A800000096C30000964318FCFFFF5C15002081
:10F2B80064150020701500207C150020141500200E
:10F2C8001C15002028150020044B00221A605A60E3
:10F2D800034B00221A605A60704700BF881500204F
:10F2E800B415002010B50B4C0123E3704FF4806077
:10F2F800022384F82030FBF7C1FC074A074BD26889
:10F308001B685178642212FB01336361238801333F
:10F31800238010BDA426002064260020181B00208E
:10F32800014B33F811007047EC160020002070479D
:10F338000F4B10B51A6802EB40010C7E2CB1022C61
:10F348000DD003EB4003988810BD032805D1094B65
:10F358001B68DB0401D4908A10BDD08910BD487E9B
:10F3680000EB800000EB800000F2EE2080B210BDC0
:10F3780074260020781B002008B5F6F7ECF8064B39
:10F38800022283F82C20054A986212689A630122A7
:10F3980083F8512008BD00BF74260020181B0020E8
:10F3A80008B5F6F7D8F8074B022283F82C209A6B99
:10F3B80000F5B71000F5587002F2DC5298629A63B3
:10F3C80008BD00BF74260020104B93F85420012A72
:10F3D80010B51C460ED008D3022A0FD10C4A938AC6
:10F3E8009BB283F48053938208E0094B4FF4805218
:10F3F8009A6103E0064B4FF480521A85F6F7ABF892
:10F4080000F5F42000F59070A06510BD742600206A
:10F418000004004808B5044B1B7803F00503052BCE
:10F4280001D1F6F753FAFEE7D0260020D0400B1C96
:10F438001141203A03D49C46134118436346524273
:10F4480093401843704700BF81F0004102E000BFBD
:10F4580083F0004330B54FEA41044FEA430594EA8C
:10F46800050F08BF90EA020F1FBF54EA000C55EAC7
:10F47800020C7FEA645C7FEA655C00F0E2804FEA98
:10F488005454D4EB5555B8BF6D420CDD2C4480EA7A
:10F49800020281EA030382EA000083EA010180EAAA
:10F4A800020281EA0303362D88BF30BD11F0004FF8
:10F4B8004FEA01314FF4801C4CEA113102D040422E
:10F4C80061EB410113F0004F4FEA03334CEA133369
:10F4D80002D0524263EB430394EA050F00F0A78081
:10F4E800A4F10104D5F1200E0DDB02FA0EFC22FA7C
:10F4F80005F2801841F1000103FA0EF2801843FA70
:10F5080005F359410EE0A5F120050EF1200E012A60
:10F5180003FA0EFC28BF4CF0020C43FA05F3C0189E
:10F5280051EBE37101F0004507D54FF0000EDCF117
:10F53800000C7EEB00006EEB0101B1F5801F1BD3C0
:10F54800B1F5001F0CD349085FEA30004FEA3C0CC4
:10F5580004F101044FEA445212F5800F80F09A80BA
:10F56800BCF1004F08BF5FEA500C50F1000041EBBE
:10F57800045141EA050130BD5FEA4C0C404141EBC2
:10F58800010111F4801FA4F10104E9D191F0000FE9
:10F5980004BF01460020B1FA81F308BF2033A3F16C
:10F5A8000B03B3F120020CDA0C3208DD02F1140C63
:10F5B800C2F10C0201FA0CF021FA02F10CE002F19E
:10F5C8001402D8BFC2F1200C01FA02F120FA0CFC97
:10F5D800DCBF41EA0C019040E41AA2BF01EB0451E0
:10F5E800294330BD6FEA04041F3C1CDA0C340EDCDE
:10F5F80004F11404C4F1200220FA04F001FA02F321
:10F6080040EA030021FA04F345EA030130BDC4F1DE
:10F618000C04C4F1200220FA02F001FA04F340EAD3
:10F628000300294630BD21FA04F0294630BD94F084
:10F63800000F83F4801306BF81F480110134013D6B
:10F648004EE77FEA645C18BF7FEA655C29D094EADC
:10F65800050F08BF90EA020F05D054EA000C04BF5A
:10F668001946104630BD91EA030F1EBF0021002045
:10F6780030BD5FEA545C05D14000494128BF41F0E4
:10F68800004130BD14F580043CBF01F5801130BD48
:10F6980001F0004545F0FE4141F470014FF00000D3
:10F6A80030BD7FEA645C1ABF194610467FEA655C84
:10F6B8001CBF0B46024650EA013406BF52EA033526
:10F6C80091EA030F41F4002130BD00BF90F0000F14
:10F6D80004BF0021704730B54FF4806404F1320450
:10F6E8004FF000054FF0000150E700BF90F0000F09
:10F6F80004BF0021704730B54FF4806404F1320430
:10F7080010F0004548BF40424FF000013EE700BFFF
:10F7180042004FEAE2014FEA31014FEA02701FBF8F
:10F7280012F07F4393F07F4F81F06051704792F061
:10F73800000F14BF93F07F4F704730B54FF46074DB
:10F7480001F0004521F0004120E700BF50EA010226
:10F7580008BF704730B54FF000050AE050EA0102D3
:10F7680008BF704730B511F0004502D5404261EB43
:10F7780041014FF4806404F132045FEA915C3FF484
:10F78800DCAE4FF003025FEADC0C18BF03325FEA1D
:10F79800DC0C18BF033202EBDC02C2F1200300FAD2
:10F7A80003FC20FA02F001FA03FE40EA0E0021FAF7
:10F7B80002F11444C1E600BF4FEA4102B2F1E0434E
:10F7C80024BFB3F5001CDCF1FE5C0DD901F0004C40
:10F7D8004FEAC0024CEA5070B2F1004F40EB830090
:10F7E80008BF20F00100704711F0804F21D113F1BC
:10F7F8003872BCBF01F00040704741F480114FEAF5
:10F808005252C2F11802C2F1200C10FA0CF320FA7D
:10F8180002F018BF40F001004FEAC1234FEAD3239A
:10F8280003FA0CFC40EA0C0023FA02F34FEA430304
:10F83800CCE77FEA625307D150EA01331EBF4FF08D
:10F84800FE4040F44000704701F0004040F0FE40A8
:10F8580040F40000704700BF7BB972B90029BEBFF1
:10F8680000204FF0004106E008BF00281CBF6FF0E1
:10F8780000414FF0FF3000F073B882B0EC462DE93C
:10F88800005000F03DF8DDF804E002B00CBC704711
:10F8980007EE900AF5EEC07AF1EE10FA01D400F006
:10F8A80009B808B580F0004000F004F8404261EB68
:10F8B800410108BDD0B5FFF72BFF00220E4B0646CD
:10F8C8000F4600F04FF800F05FFA0446FFF7FEFE1F
:10F8D80000220A4B00F046F802460B4630463946ED
:10F8E800FFF7B6FD00F050FA2346002242EA000274
:10F8F80010461946D0BD00BF0000F03D0000F041A1
:10F908002DE9F041069C154606460F46984600F03C
:10F918005BFA05FB01F300FB0838A5FB0023B21ACC
:10F92800434467EB0303C4E90023BDE8F08100BF4B
:10F938002DE9F041069C904606460F461D4600F00C
:10F9480091FB00FB05F5A0FB082308FB0155B21A43
:10F958002B4467EB0303C4E90023BDE8F08100BF33
:10F96800704700BF70B54FF0FF0C4CF4E06C1CEA18
:10F9780011541DBF1CEA135594EA0C0F95EA0C0F9D
:10F9880000F0DEF82C4481EA030621EA4C5123EA10
:10F998004C5350EA013518BF52EA033541F480113F
:10F9A80043F4801338D0A0FB02CE4FF00005E1FBF2
:10F9B80002E506F00042E0FB03E54FF00006E1FB3C
:10F9C80003569CF0000F18BF4EF0010EA4F1FF047F
:10F9D800B6F5007F64F5407404D25FEA4E0E6D41BF
:10F9E80046EB060642EAC62141EA55514FEAC520D0
:10F9F80040EA5E504FEACE2EB4F1FD0C88BFBCF54C
:10FA0800E06F1ED8BEF1004F08BF5FEA500E50F1FC
:10FA1800000041EB045170BD06F0004646EA0101C2
:10FA280040EA020081EA0301B4EB5C04C2BFD4EBF4
:10FA38000C0541EA045170BD41F480114FF0000EED
:10FA4800013C00F3AB8014F1360FDEBF002001F05B
:10FA5800004170BDC4F10004203C35DA0C341BDCD5
:10FA680004F11404C4F1200500FA05F320FA04F0A7
:10FA780001FA05F240EA020001F0004221F00041DB
:10FA880010EBD37021FA04F642EB06015EEA430E4E
:10FA980008BF20EAD37070BDC4F10C04C4F120057E
:10FAA80000FA04F320FA05F001FA04F240EA020031
:10FAB80001F0004110EBD37041F100015EEA430E02
:10FAC80008BF20EAD37070BDC4F1200500FA05F222
:10FAD8004EEA020E20FA04F301FA05F243EA0203A1
:10FAE80021FA04F001F0004121FA04F220EA0200B0
:10FAF80000EBD3705EEA430E08BF20EAD37070BDF6
:10FB080094F0000F0FD101F00046400041EB0101D5
:10FB180011F4801F08BF013CF7D041EA060195F0B7
:10FB2800000F18BF704703F00046520043EB030371
:10FB380013F4801F08BF013DF7D043EA060370475E
:10FB480094EA0C0F0CEA135518BF95EA0C0F0CD069
:10FB580050EA410618BF52EA4306D1D181EA0301AF
:10FB680001F000414FF0000070BD50EA410606BFA9
:10FB78001046194652EA430619D094EA0C0F02D1EE
:10FB880050EA013613D195EA0C0F05D152EA033633
:10FB98001CBF104619460AD181EA030101F0004151
:10FBA80041F0FE4141F470014FF0000070BD41F09A
:10FBB800FE4141F4780170BD70B54FF0FF0C4CF474
:10FBC800E06C1CEA11541DBF1CEA135594EA0C0F93
:10FBD80095EA0C0F00F0A7F8A4EB050481EA030EE0
:10FBE80052EA03354FEA013100F088804FEA0333C7
:10FBF8004FF0805545EA131343EA12634FEA022295
:10FC080045EA111545EA10654FEA00260EF0004155
:10FC18009D4208BF964244F1FD0404F5407402D2A7
:10FC28005B084FEA3202B61A65EB03055B084FEA38
:10FC380032024FF480104FF4002CB6EB020E75EB35
:10FC4800030E22BFB61A754640EA0C005B084FEA5D
:10FC58003202B6EB020E75EB030E22BFB61A7546DA
:10FC680040EA5C005B084FEA3202B6EB020E75EB25
:10FC7800030E22BFB61A754640EA9C005B084FEA9D
:10FC88003202B6EB020E75EB030E22BFB61A7546AA
:10FC980040EADC0055EA060E18D04FEA051545EA99
:10FCA80016754FEA06164FEAC30343EA52734FEA42
:10FCB800C2025FEA1C1CC0D111F4801F0BD141EABB
:10FCC80000014FF000004FF0004CB6E711F4801F20
:10FCD80004BF01430020B4F1FD0C88BFBCF5E06F00
:10FCE8003FF6AFAEB5EB030C04BFB6EB020C5FEA10
:10FCF800500C50F1000041EB045170BD0EF0004E65
:10FD08004EEA113114EB5C04C2BFD4EB0C0541EA96
:10FD1800045170BD41F480114FF0000E013C90E693
:10FD280045EA060E8DE60CEA135594EA0C0F08BF57
:10FD380095EA0C0F3FF43BAF94EA0C0F0AD150EA56
:10FD480001347FF434AF95EA0C0F7FF425AF1046E9
:10FD580019462CE795EA0C0F06D152EA03353FF411
:10FD6800FDAE1046194622E750EA410618BF52EA8E
:10FD780043067FF4C5AE50EA41047FF40DAF52EA62
:10FD880043057FF4EBAE12E74A0011D212F50012D8
:10FD980011D20DD56FF47873B3EB62520ED44FEADB
:10FDA800C12343F0004343EA505323FA02F070475B
:10FDB8004FF00000704750EA013002D14FF0FF3099
:10FDC80070474FF00000704700292DE9F043C0F25A
:10FDD800A6800026002BC0F29C80884694469E464A
:10FDE800154604460F46002B3DD18A4259D9B2FA2E
:10FDF80082F33BB1C3F120029F4020FA02F29D40FA
:10FE080017439C40290C220CB7FBF1FEA8B201FB5A
:10FE18001E7742EA074700FB0EF3BB420AD97F1957
:10FE28000EF1FF3280F00581BB4240F20281AEF153
:10FE3800020E2F44FF1AA4B2B7FBF1F301FB1377AC
:10FE480044EA074700FB03F0B84208D97F1903F1D9
:10FE5800FF3280F0F080B84240F2ED80023B43EA86
:10FE68000E43002203E08B420FD900221346341CB4
:10FE780018BF012460424FF0000565EB450158406A
:10FE8800514000196941BDE8F083B3FA83F2002AB2
:10FE980040F086808B4202D3844500F2DB80012348
:10FEA800E5E712B90123B3FBF2F5B5FA85F00028AE
:10FEB8003BD1781B4FEA154E1FFA85FC0122B0FB97
:10FEC800FEF8210C0EFB180741EA07470CFB08F364
:10FED800BB4207D97F1908F1FF3102D2BB4200F2B9
:10FEE800BD808846FF1AA4B2B7FBFEF30EFB13775A
:10FEF80044EA07470CFB03FCBC4507D97F1903F10B
:10FF0800FF3102D2BC4500F2A7800B4643EA084302
:10FF1800ADE752426FEA060663EB43035DE74042F2
:10FF280061EB41014FF0FF3654E7C0F1200224FA9B
:10FF380002F107FA00F385404FEA154ED7401943FE
:10FF4800B7FBFEF20B0C0EFB12771FFA85FC43EA97
:10FF580007430CFB02F79F4204FA00F407D95B1928
:10FF680002F1FF3074D29F4272D9023A2B44DF1B50
:10FF780089B2B7FBFEF80EFB187341EA03430CFB8A
:10FF880008F79F4208D95B1908F1FF315CD29F42FC
:10FF98005AD9A8F102082B44D81B48EA02428EE736
:10FFA800C2F120032CFA03F10EFA02FE20FA03F73D
:10FFB80041EA0E0E08FA02F028FA03F14FEA1E454C
:10FFC8003843B1FBF5F8030C05FB18111FFA8EF73F
:10FFD80043EA014107FB08F38B420CFA02FC09D9FA
:10FFE80011EB0E0108F1FF3930D28B422ED9A8F15E
:08FFF80002087144C91A80B22D
:020000040801F1
:10000000B1FBF5F305FB131140EA014107FB03F7D0
:100010008F4208D911EB0E0103F1FF3016D28F4247
:1000200014D9023B714443EA0843C91BA3FB0C8962
:10003000494509D305D000221DE79646FEE6134642
:1000400011E794404445F6D2013BF4E70346EAE762
:100050008846A5E7C846D1E702468CE713460AE77B
:10006000023B57E7A8F102082F443FE72DE9F04192
:10007000002B44D18A42154604464FD9B2FA82F782
:100080000E464FB1C7F12003B94020FA03F602FA39
:1000900007F50E4300FA07F44FEA154E230CB6FBA2
:1000A000FEF0AFB20EFB106143EA014307FB00F123
:1000B000994209D95B1900F1FF3280F0EC80994236
:1000C00040F2E98002382B445A1AA4B2B2FBFEF384
:1000D0000EFB132244EA024207FB03F7974208D9BA
:1000E000521903F1FF3180F0D880974240F2D58059
:1000F000023B43EA004000263146BDE8F0818B42D6
:1001000047D8B3FA83F6002E48D18B4202D38242FD
:1001100000F2CD8001203146BDE8F08112B9012501
:10012000B5FBF2F5B5FA85F8B8F1000F77D14A1BA7
:100130004FEA154EAFB20126B2FBFEF0230C0EFBC8
:10014000102143EA014107FB00F38B4207D949190B
:1001500000F1FF3202D28B4200F2BA801046C91A77
:10016000A4B2B1FBFEF30EFB131144EA014407FBFA
:1001700003F7A74208D9641903F1FF3280F08F809A
:10018000A74240F28C80023B43EA00403146BDE882
:10019000F081002630463146BDE8F081C6F12004EA
:1001A00022FA04F5B3402B4320FA04FC01FA06F7C7
:1001B00021FA04F54FEA134E4CEA0707B5FBFEF8A7
:1001C000390C0EFB18551FFA83FC41EA05450CFB60
:1001D00008F1A94202FA06F204D9ED1808F1FF3439
:1001E00067D3A0466D1ABFB2B5FBFEF40EFB1455E3
:1001F00047EA05410CFB04FC8C4504D9C91804F1FD
:10020000FF355CD32C4644EA0844CCEB0101A4FB47
:100210000223994248D344D0204600266CE7C8F117
:10022000200401FA08F305FA08F520FA04F7E14082
:100230004FEA154E1F43B1FBFEF63A0C0EFB1611AA
:100240001FFA85FC42EA01430CFB06F29A4200FACF
:1002500008F407D95B1906F1FF3137D29A4235D934
:10026000023E2B449B1ABFB2B3FBFEF00EFB1033D1
:1002700047EA03430CFB00F1994207D95B1900F1EF
:10028000FF3221D299421FD902382B445A1A40EA30
:100290000646674650E7104616E70B4629E7134621
:1002A00072E7B0409042B7D2601E002624E7304685
:1002B00022E7A94295D9A8F102081D4492E78C458E
:1002C000A0D9023C19449EE71046DFE70E46C9E775
:1002D0000238294443E700BF4FF0FF3C06E000BF6F
:1002E0004FF0010C02E000BF4FF0010C4DF804CDBF
:1002F0004FEA410C7FEA6C5C4FEA430C18BF7FEA7F
:100300006C5C1BD001B050EA410C0CBF52EA430CAC
:1003100091EA030F02BF90EA020F0020704710F12C
:10032000000F91EA030F58BF994208BF90422CBFBB
:10033000D8176FEAE37040F0010070474FEA410CB4
:100340007FEA6C5C02D150EA013C07D14FEA430CD2
:100350007FEA6C5CD6D152EA033CD3D05DF8040B43
:10036000704700BF8446104662468C461946634675
:1003700000E000BF01B5FFF7B7FF002848BF10F14C
:10038000000F01BD4DF808EDFFF7F4FF0CBF012091
:1003900000205DF808FB00BF4DF808EDFFF7EAFF0D
:1003A00034BF012000205DF808FB00BF4DF808EDC8
:1003B000FFF7E0FF94BF012000205DF808FB00BFBD
:1003C0004DF808EDFFF7CEFF94BF012000205DF847
:1003D00008FB00BF4DF808EDFFF7C4FF34BF012054
:1003E00000205DF808FB00BF114812490268006058
:1003F0008A4218D0002103E00F4B5B584350043170
:100400000E480F4B42189A42F6D30E4A02E00023E0
:1004100042F8043B0C4B9A42F9D3FEF77BF800F00C
:1004200019F87047FEE70948D0F800D04068004747
:10043000FC9F0020EFBEADDE9070010800000020A0
:1004400068010020680100200027002000D8FF1F5D
:10045000FEE700002DE9804891B0EFF795FEB24C21
:10046000B24D2378296833B1B14B1B68CB1A002BEE
:10047000A4BF00232370DFF810A3DAF8000042F2D3
:10048000010303400BB9AB4A1370070740F1928197
:10049000A94B1B681B7A062B00F27C81DFE813F066
:1004A000070007003400D40010013C013C01A34BBD
:1004B0001A78002A00F06E8100221A70A04B93F87F
:1004C00000E0A04B1B6893F800C09F4B93F800809E
:1004D00002229E4FBB5C43FA0EF303F00F03634509
:1004E00002F101090CD20B2B9FBFBE5C17F80970FB
:1004F00006EA080607EB06269CBF954F47F82360DF
:100500000232102AE5D10CE1924B1A78002A00F051
:10051000418100221A70904B904A93F802C093F8E0
:1005200003E05E780CF0070746EA07260EF03F0767
:100530007F0147EADC0716601E7957605F7993F800
:1005400006C0B60046EA9E1607F0010E46EA8E2661
:10055000966093F807E00CF00F06F60146EA57069E
:100560000EF07F07D6603F011E7A47EA1C1793F80A
:1005700009C0176176000CF0030746EADE1646EA6A
:10058000472693F80AE05661DE7A0EF01F07BF0196
:10059000F60047EA9C0746EA5E1693F80DC093F80A
:1005A0000EE0D6611E7B97610CF0070746EA07262E
:1005B0000EF03F077F0147EADC071662DE7B5762D9
:1005C0001F7C93F811C0B60046EA9E1607F0010E94
:1005D00046EA8E26966293F812E00CF00F06F601BA
:1005E00046EA57060EF07F073F0147EA1C17D6621E
:1005F000DE7C176393F814C0760046EADE160CF032
:10060000030746EA472693F815E056639E7DDB7D97
:100610000EF01F07F60046EA5E16BF01D66347EAF2
:100620009C07DE074CBF40F21476AD2697639F0708
:1006300016644CBF40F21476AD2613F0080F5664D2
:1006400014BF03230123A6E0454A1378002B00F0D2
:10065000A18000231370434ADFF830E11778424E3F
:100660000EEB470CB6F800809CF803909CF80460F1
:1006700046EA0926B04540F08D809EF80160012EC3
:1006800004D0812E40F08780032300E03346102FF2
:1006900084BF10261670354E92F800E00022D7B2C3
:1006A000774506F1020676D216F802CC16F8017CE0
:1006B00047EA0C27DFF8D8C02CF812700132EEE7B9
:1006C0002B4B1A78002A65D000221A70294B1A7811
:1006D000A82A1F465ED1DA7C002A5BD107EB4206CE
:1006E0009FED257A96F803E0337903EB0E2307EEAE
:1006F000903AF8EEE77A214BC7EE877A9FED207AA1
:1007000077EEC77AFCEEE77A17EE906A43F822603C
:100710000132082AE2D104E01A4B1A78D2B300223F
:100720001A70012337E000BF200A0020D4260020E1
:1007300068010020210A00207426002029170020CB
:100740006623002060230020672300201917002063
:10075000101600209A170020811700208016002014
:10076000511700205417002052170020581700205E
:100770004A17002035170020CDCCCC404016002071
:100780000080BB430C160020781B0020551700206A
:10079000601600200023DE070CD5A64A83F0020372
:1007A000C3F34003012616702370A34A01F5C33337
:1007B000A033136042040FD5A04A13780BB1002672
:1007C00016709C4A13703BB1012323709A4A01F5BD
:1007D000433303F5A0731360C3070CD5964B5A79C6
:1007E0001E79B2421FBF0122227001F5C332A0322E
:1007F0001CBF1A605E71870409D50023904A32F845
:100800001320002A40F0518701330C2BF6D1894B7D
:10081000894C1B7823B98B4B1B68CB1A002B0ADB46
:10082000A368C91A11F15A0F05D5F0F759FE824B8A
:1008300001221A7324E123697F4A0133002BC8BFC8
:1008400000230606136140F11B817F4F3B683E4643
:10085000A3B9237D013B042B00F21281DFE813F0E2
:100860001400140014000001CC00774B1868F4F752
:10087000C1FEFAF712FD08B1FCF774FC3068F4F71A
:10088000BCFE0028F1D1E4E7626B6B4E92F8008069
:10089000B8F1000F03D0B8F1010F10D0F0E0012B38
:1008A00000F2EE80727D694B38680C2101FB023347
:1008B0005A78674B53F82210F4F799FE5DE03868D8
:1008C000DFF88491F4F790FE002800F0D980337DA2
:1008D000022B40D0032B4DD0012B40F0D1805D4B3B
:1008E0001968F36ACB1AC72B40F2CA80B36A042B8B
:1008F0002FD8564AF1620C20D9F8006000FB032380
:10090000B0685F7896460023514A52F8231081421E
:100910005FFA83FC04D00133082BF5D1002300E0FB
:100920006346BB4205D0304652F82710F4F75FFE0D
:10093000A6E0627D0C2303FB02E35F6817F8011B4E
:1009400019B13046F4F75CFEF8E7A36A0133A362FD
:1009500096E0022092E0727D3C4BD9F800000C2119
:1009600001FB02335A783A4B53F82210F4F73FFE5A
:10097000032083E0736B9B780BB904207EE096F82C
:1009800030300BB986F8308094F830302A4E012B85
:1009900012D1B36AB22B0AD82C4A3868134493F8A0
:1009A0003C10F4F72DFEB36A0133B36204E0002378
:1009B000B362022386F8303094F830301E4E022B9A
:1009C00015D1B26A0F2A0FD8736B20495B7838684B
:1009D00003EB03130B44134493F8F010F4F710FEE9
:1009E000B36A0133B36202E0032386F8303094F82F
:1009F0003030022B44D9C0E7E3690F490133E3618A
:100A0000636BDB784BB14B7D0133DBB20522B3FB6B
:100A1000F2F202EB82029B1A4B750E4B1B682362AB
:100A20000D4B00221A700D4A137823F00203137045
:100A3000012023E0210A0020680100208E10002000
:100A4000EC160020F8090020601800205C36010830
:100A500080450108181B00201911002018110020E2
:100A6000A14B226A1B689B1A40F6C412934207D915
:100A70009E4A136823F0200313600520FAF7FEFE58
:100A8000F4F76DFD9A4B286009AEDB683046984755
:100A90009DF824302BB9974BA2681B689B1A642BD6
:100AA00037D4954BDFF884B21B680493049A2B6803
:100AB0001344A360914B1988002940F01B86DBF892
:100AC0000000583000F01ABE9AF80430002B01F0F4
:100AD0002F8469890020F2F719FA01263B689906EC
:100AE00001F16184B9F1050F01F05D843B68DA0220
:100AF00001F1668498F818360BB1F4F79BFE7F4B32
:100B00001B88002B01F0E9857D4B1B78002B01F041
:100B100065847B4B1B78002B7FF4A1ACDFF810922F
:100B2000D9F8002012F4806F4F463FF498AC754A14
:100B3000754DB2F84EA195F819266B4E002A00F0BB
:100B40002C823168D5F81C268A1A7C2A40F225822C
:100B500095F82026C5F81C16013285F820269846FF
:100B600008F12400C0B2F6F735F9684B9FED687ABA
:100B700033F9183007EE903AFAEECC7A08F1010812
:100B800067EE877AFDEEE77ACDED047ABDF91000C5
:100B9000F6F70EF9B8F1030FE2D13020F6F71AF9A3
:100BA0000020F6F705F9F6F70DF994F8208618F00D
:100BB000030822D1544BD3F81C2641F288339A42C1
:100BC0000BD91020F6F706F94046F6F7F1F8212088
:100BD000F6F700F94046F6F7EBF81420F6F7FAF8C6
:100BE0004C4BB3F90000F6F7E3F81C20F6F7F2F8E7
:100BF0000020F6F7DDF8F6F7E5F894F820365A0706
:100C000040F0A5810220F6F7E5F8434BB3F9000068
:100C10000A2390FBF3F0F6F7CBF8404B0320B3F92F
:100C20000680F6F7D7F83E4B1B785B074FF0050BB5
:100C300098FBFBF81FFA88F80ED53A485146F6F7AC
:100C4000FAFD30B9D9F8003013F0100F18BF4FF08B
:100C500000080FFA88F005E0334B1B689889B0FB59
:100C6000FBF000B2F6F7A4F8D9F80030980740F18D
:100C7000BF80DFF8C0B0B4F82296DFF8BC809BF8E4
:100C80000030B8F800204FEA09194FF0640A1FFA43
:100C900089F90AFB02325B00B2FBF3F349EA03294C
:100CA0001FFA89F9C3F3032349EA03090620F6F77B
:100CB00091F80FFA89F0F6F77BF8B4F822369BF832
:100CC000001001339BB293FBF1F201FB1233A4F845
:100CD0002236D4F824369B7B012B2FD13920F6F70E
:100CE00079F8B8F900004AE0181B0020A410002091
:100CF0005C130020D4260020CC150020A810002072
:100D0000F5260020481C002068010020CC1000209F
:100D100000007A44041100209410002014150020D3
:100D2000F3260020D01D0020C8170020E810002066
:100D3000781B0020F800002058180020B8F8008028
:100D40006E233A2003FB08F84FF01509F6F742F836
:100D500098FBF9F81FFA88F9B9FBFAF80FFA88F04E
:100D6000F6F726F80AFB18983B20F6F733F81FFA37
:100D700088F000F105080A2098FBF0F000B2F6F7C1
:100D800017F82820F6F726F8B24B0A201B6893FBC9
:100D9000F0F000B2F6F70CF80420F6F71BF8AE4BB3
:100DA000AE491B6808689A894FF6FF739842A8BF3E
:100DB0001846C2B10028ACBF131A134607EE903A8A
:100DC0009FEDA77AF8EEE77A67EE877A07EE102AAA
:100DD000B8EEC77AC7EE877AFDEEE77A17EE900A8B
:100DE0006428A8BF642020EAE07000B2F5F7E0FFB5
:100DF0009C4B1B68990640F19F80DFF8A09299F800
:100E000000309A0721D5DFF898A21120F5F7E2FF0C
:100E1000BAF80000944B4FF4F36808FB00F090FB25
:100E2000F3F000B2F5F7C4FF1920F5F7D3FFBAF8D5
:100E3000000008FB00F8642098FBF0F898FBF0F342
:100E400000FB138000B2F5F7B3FF884BB3F80080C6
:100E500099F8003013F0020F08BF4FF0000801208E
:100E6000F5F7B8FF0FFA88F0F5F7A2FF0920F5F7BC
:100E7000B1FF0020F5F79CFF7D4B93F800807D4B80
:100E80001A88B2F5967F0AD994F8203603F00F033A
:100E9000072B04D842F20F78904528BF90460520D2
:100EA000F5F798FFD5F824365B7B13B90FFA88F075
:100EB0001CE0A8F1200307EE903A9FED6F7AF8EE60
:100EC000E77AF6EE006AC7EE877ABEEE007AF5EEB4
:100ED000C07AF1EE10FA58BFB0EE667A77EE877AF4
:100EE000FDEEE77ACDED047ABDF91000F5F760FF6D
:100EF00099F800309B0703D495F82836012B04D1CC
:100F0000012385F828365D481DE05D4BDFED5D6A05
:100F1000D3F8243693ED017AD3ED027A27EE267AC0
:100F200067EEA67ABDEEC77AFDEEE77A8DED097A17
:100F3000CDED0A7A09A806E0534A92E8030009AB0E
:100F400083E803001846F5F755FFF5F73BFF95F8E2
:100F50002036282B21D14A4B3068002283F82026E6
:100F60004FF03C0A4FF47A73B0FBF3F91720F5F712
:100F700031FFB9FBFAF8B8FBFAF00AFB1080000267
:100F800000B2F5F715FF1820F5F724FF0AFB1890BB
:100F900000B2F5F70DFFF5F715FF95F82936DFF8E4
:100FA000E090002B00F08181F4F7D9FAD9F82C36C3
:100FB000364AC31A9342804640F2EF80002389F8F4
:100FC000323689F83436324B1B88DAB21B0A89F87C
:100FD0004E2689F84F3689F8442689F84536D9F8DF
:100FE0005C2633689A1AD9F86036D97B4FF47A7345
:100FF0004B439A420ED3274B1B68C9F85C36264BED
:101000001B78013B012B9FBF102389F83236022346
:1010100089F834360F4B1A481A68104B0A2192FB94
:10102000F1F284F84C26121284F84D261B4A1B68F4
:1010300093FBF1F384F850361B1284F85136127882
:101040000B4B95071B7884F87E362BD42D2380F824
:101050007F369FE010110020C817002008110020E3
:101060000000C842A4100020A08601002411002026
:1010700019110020EC0000206666E63F1C110020DC
:10108000680100208096184B283A01083F0D0300A4
:1010900058180020181B0020A4240020181100203C
:1010A00026110020042B8CBF3323322380F87F3697
:1010B000CF4BDFF86C93D3F800A05D68CD4ACE4BE0
:1010C0009AFBF3F04FF0060C09FB00A195FBF3F33C
:1010D00009FB035903EB83030CFB01F103EB8303CF
:1010E00091FBF2FE642602FB1E119B0091FBF6F1C0
:1010F00084F8701609120CFB09FC84F871169CFB2D
:10110000F2F143FA81F39BB284F873361B0A84F838
:101110007436BA4B02FB11C292FBF6F284F87526C4
:10112000121284F876261A882423534393FBF6F68A
:10113000B34B84F86B661B8884F877361B0A84F8F7
:101140007836B04B00EB80001B880A22B3FBF2F329
:1011500003F5FA739BB200EB8000800084F87936C7
:101160001B0A40FA8EF084F87A36A74B80B24FEA19
:10117000DA7A84F86E06ED0F000AC6F307261B889C
:1011800084F86DA684F86F0684F8725684F86C664D
:1011900084F880369D4BC3F82C869C4E96F890A61A
:1011A0003546BAF1000F0FD1D6F89806F4F725FAB4
:1011B000012809D90228DFF86C9201F09682F5F730
:1011C000E9FD012389F80130D6F89C068F4D0028EF
:1011D0006BD095F89096B9F1000F08D0D5F8A436E9
:1011E00040F6B732C3EB0803934219D85DE0012300
:1011F000D5F8980685F89036F6F737F8D5F8A8367A
:1012000093F9000002238DE8080208214A464FF4B2
:101210009643F6F745F885F8AC96C5F8980642E08F
:1012200095F8A096B9F1000F19D1D5F89806C5F830
:101230009C9685F89096F6F718F8D5F8A83693F9A5
:10124000000001238DE8080208214A464FF4964326
:10125000F6F726F8C5F89806F5F79CFD23E009F1A6
:10126000FF32D2B285F8A02695F8AC1695F8AD36C7
:1012700042B94A1C013385F8AC2685F8AD36D5F85D
:1012800098060EE00246013312F801EBC5F89C26E1
:101290000EEB010085F8AC06D5F8980685F8AD365A
:1012A0007146F4F7ADF9C6F8A486584D95F8AE36F8
:1012B0002E460BB3D5F8B036F3B1D5F8B436DBB162
:1012C000DFF864811A68C8F80030514B1A60514A3F
:1012D000D5F8B836134493F8D403F3F70FFAD8F8D7
:1012E00000309879FCF7F9FBD5F8B8360133092BB3
:1012F00088BF0023C5F8B836DFF830B195F8BC26B2
:10130000DBF800300493D846404B002A3FF4A7A8EE
:10131000D3F8C026002A3FF4A2A893F8C436013BB4
:10132000012B3FF69CA8D4F8C006DFF8E0A0F4F744
:1013300064F9F0B1DAF8C006F4F75CF99AF8C5166A
:10134000D8F800207E29814610D102211B288AF876
:10135000C4160BD1DAF8C0060592F4F74EF928B995
:10136000059ACAF8C82601228AF8CC2686F8C596BE
:10137000D9E7DAF8C826DBF800309B1A41F6583274
:10138000934220D903238AF8C436FFF768B8224A6B
:1013900032F8130010B903464FF403600133B0F57F
:1013A000C06FDBB200F0978042D9B0F5006F00F05B
:1013B0009B8056D9B0F5036F64D184F8CD36174BB6
:1013C0001B689A0665D496F8CC1696F8CD36002997
:1013D00000F06781D8F800200498121A012AD6D9A3
:1013E00085F8CD36002385F8CC36FFF738B800BF36
:1013F0001C11002040420F0080969800261100200A
:101400002A110020241100202C1100206801002046
:101410009C2400205C36010800550108A41000201F
:10142000806967FF0000002098240020181B00201E
:10143000B0F5007F43D008D8B0F5807F00F08880F9
:10144000B0F5887F00F08480C1E7B0F5806F00F0D0
:10145000A480B0F5826F00F0E380B0F5047FB6D1D0
:1014600024E0B0F5E26F00F08480B0F5E46F00F0A6
:101470008680B0F5E06FAAD184F8CD368F4BB3F9F2
:10148000001081E0B0F5046F6BD0B0F5026F9ED113
:10149000F0E08B4B1B789B0795D58A4B198824234A
:1014A0004B431233642193FBF1F1F3E084F8CD3622
:1014B0003B68990787D5844B0A211B88E9E084F8AB
:1014C000CD363B681A057FF57EAF804B19680A233D
:1014D00091FBF3F1DEE084F8CD363B681B057FF528
:1014E00072AF7B4B1968D5E07A4A84F8CD36126822
:1014F00091067FF568AF724A127892077FF563AF65
:1015000013F0010F744B11D05A6882EAE273A3EB17
:10151000E273002A4FF0190103EB5303B3FBF1F31D
:1015200043F0004111DA43F040410EE01B6883EACA
:10153000E371A1EBE371002B01EB51014FF01902B4
:10154000B1FBF2F1B8BF41F080414FF4006080E0A0
:1015500084F8CD365F4B1B685B077FF534AF002105
:1015600098E084F8CD365D4BB3F9001064235943FD
:101570000DE084F8CD36514BB3F9021004E084F845
:10158000CD364E4BB3F904102C2391FBF3F1F5F754
:10159000CDFB002384F8CC3615E784F8CD3694F8DB
:1015A000CE364F4A0133DBB2032B88BF012382F8CA
:1015B000CE3694F8CE1642F210735943494B1B783D
:1015C000D80748BF01319A0748BF02315807464B38
:1015D0001B8848BF0431DA0748BF0A31980748BF63
:1015E00014311A0648BF2831D80548BF28315A0798
:1015F00048BF6431180748BFC8319A0548BF01F594
:10160000C871980648BF01F57A71DA0648BF01F53E
:10161000FA61580648BF01F57A614FF4806018E01E
:1016200084F8CD362B4B1B6813F0200A17D0244BBF
:101630001A7812F0020F14BF4FF47A71002112F0E1
:10164000010F2A4A14BF4FF4FA6300230B441178A8
:101650001944F5F76BFB002386F8CC36B3E63B68FC
:1016600019067FF5B0AE5146F5F760FB1C4B83F8C9
:10167000CCA6A8E684F8CD36164B1B689A067FF5F3
:10168000A2AE0F4B1B789B077FF59DAE184B1B88B6
:1016900064215943F5F74AFB114B002283F8CC260D
:1016A00091E685F8CD36FEF7DABE012323700C4AA9
:1016B00001F5C333A0331360FFF7A9B8CC100020A5
:1016C00018110020261100205818002010110020A9
:1016D00008110020A41000201C110020041100207B
:1016E00068010020F3260020A81000201911002016
:1016F00024110020DBF8000002215830F4F76CF9C7
:10170000F3F72DFFA26BDDED047ABC4BDFEDBC0AD5
:101710002860821AF8EE677A92B21A8067EEA00A01
:10172000B84BA063C3ED000AB74B354603F1080E72
:10173000186859682F4603C7083373453D46F7D1EB
:1017400018689B883860BB80BDF830E0AF4F00253B
:1017500000213846884630F802CF735A20F802CC70
:1017600002310C291CFB0388F5D1A94931F8153049
:10177000BB814FF4807013FB0E8393FBF0F321F8D1
:1017800015300135032D07F10E07E1D107EE902A40
:10179000A04FB4F86650B8EE670A07F1680001215F
:1017A000F8F748FFBCEEC00A8DED040ABDF8103012
:1017B000B5FBF3F5237B6E1CB6B2A4F8706013B3CF
:1017C000B7F8728000239348934A00F17C0700F138
:1017D000740C32F813E037F813203CF8131027F894
:1017E00013E0C2EB0E0911FB08F132B291FBF2F2E9
:1017F0004A442CF813200133042BE4D10023037353
:10180000A0F8725004E0B7F87230013BA7F87230CC
:10181000B4F872007F4A03B2002B4FF0000313DDCF
:10182000B2F970507D4931F81320083112FB00F2F3
:1018300031F8131092FBF5F28A1A774921F8132038
:101840000133042BEED101E0A2F87230F1F7C0FCB5
:10185000734B744D1B68744E13F4801300F0938027
:101860002B88180600F11981704B1B7803F00403D4
:1018700003F0FF08002B72D06D4A6E4B117811B146
:1018800094F8841039B16C49002008600121197066
:10189000002184F884101B7837681370032B05D15E
:1018A00038466649542200F0B9FF51E0012B06D1B9
:1018B00054226248394600F0B1FF002202E0022BB8
:1018C00002D101225E4B1A705E4A012313705E4AF8
:1018D00013705E4A002313605D4A13605D4B1F6006
:1018E0005D4B3A781A70564B5C4A1B78D05C5C4B67
:1018F0005C4A1870504B38441A6042785A4B07EED5
:10190000902AF8EEE77AB2EE047AC7EE877AC27AC6
:101910009FED567AC3ED007A07EE902AF8EEE77A4B
:10192000427DC7EE877A9FED527AC3ED017A07EECA
:10193000902AF8EEE77A67EE877AC3ED027AFCEE3A
:10194000E77A17EE903A43750023C372FAF7CCF8A2
:101950008020F9F797F9012384F8DC309DE0364FB9
:10196000D7ED007AF5EE407AF1EE10FA00F09580AE
:10197000F9F724FC00233B602D4B83F800802D4BAE
:1019800001221A7089E02A8811067BD5284A11782D
:10199000481E012827482CD8334F2E4BD7ED017A0B
:1019A0009FED327A1A682E4B67EE877A19789FED91
:1019B000317AFCEEE77A114417EE903ACB72D7ED0C
:1019C000027A67EE877AFCEEE77A17EE903A4B756B
:1019D000537807EE903AF8EEE77A77EEA77AFCEEC6
:1019E000E77A17EE903AD370D37A5373537DD37559
:1019F00042E0032940D1137001233FE098100020FA
:101A0000BD37863528150020A0370108A401002025
:101A1000D21000206801002078260020DC01002080
:101A2000AC100020A8100020E8100020F3260020B1
:101A3000691B002000000020741B0020F001002022
:101A40006A1B00206D1B0020881B0020841B0020C7
:101A5000801B0020981B00206B1B00207C45010888
:101A60006C1B00200000A0418C1B002000007A4469
:101A70005555553F9A99993F03780133037080205B
:101A8000F9F7F0F8C14B1B785A0706D494F8DC300C
:101A90001BB1BF4B012283F88420BE4BDFF8589363
:101AA0001B78BD4FABB1BD4BB3F90620B9F89831E7
:101AB0009A420EDC99F80530012B01D0192B02D186
:101AC00099F8E6212AB90E2B03D0082B1CBF00235E
:101AD000BB80336893F81861002E46D02B889B0793
:101AE00043D09FEDAF8ADFEDAF7A88EE088AB4EE7F
:101AF000E78AF1EE10FA34D9B7EE000A30EE480A60
:101B000001F07EF99FEDA87ADFEDA87AE8EE077A7A
:101B10009FEDA77AA8EE277ADFEDA67AE8EE077A9E
:101B200020EE270AD4ED387A20EE270A01F090F84B
:101B3000B0F5617FA8BF4FF4617007EE900AB8EE70
:101B4000E70ADFED9D7A80EE270AF9F723F807EE22
:101B5000906AF8EEE77A27EE800A01F079F880B211
:101B600000E00020FB881844F880944B1B689E0618
:101B700040F19F802B8803F03003002B00F0998008
:101B80008F4B1B78D80740F194808E4BDFED8E7A17
:101B9000B3F9003008EE103AB8EEC88A28EE278A6A
:101BA000B0EE480AF8F7F6FFF0EE408AB0EE480AC9
:101BB000F9F750F8854B864A1B6893F803C0854BAC
:101BC000B0EE409AB2EE048ABCF1000F4FD08249C9
:101BD000B2F902604D88079328B2301ACDF818C0C8
:101BE00005910492F9F79CFEDDF818C0049A059956
:101BF000079BCCF10008404503DB6045A8BF604669
